:1000000000800020BD010000F9E00000B1E0000028
:10001000B1E00000B1E00000B1E00000B1E000009C
:10002000B1E00000B1E00000B1E00000F9E0000044
:10003000F9E00000B1E00000F10A0100F50A01005A
:10004000F9E00000F9E00000F9E00000F9E000004C
:10005000F9E00000F9E00000F9E00000F9E000003C
:10006000F9E00000F9E00000F9E00000F9E000002C
:10007000F9E00000F9E00000F9E00000F9E000001C
:10008000F9E00000F9E00000F9E00000F9E000000C
:10009000F9E00000F9E00000F9E00000F9E00000FC
:1000A00089B7000095B70000F9E00000F9E0000012
:1000B000F9E00000F9E00000F9E00000F9E00000DC
:1000C000F9E00000F9E00000F9E00000F9E00000CC
:1000D000F9E00000F9E00000F9E00000F9E00000BC
:1000E000F9E00000F9E00000F9E00000F9E00000AC
:1000F000F9E00000F9E00000F9E0000041EF000045
:10010000F9E00000C5F40000F9E00000F9E00000AB
:10011000F9E00000F9E00000F9E00000F9E000007B
:10012000F9E00000F9E00000F9E00000F9E000006B
:10013000F9E00000F9E00000F9E00000F9E000005B
:10014000F9E00000F9E00000F9E00000F9E000004B
:10015000A10E0100B50E0100C90E0100DD0E010067
:10016000F9E00000E1F70000F9E00000F9E000002C
:10017000F9E00000F9E00000F9E00000F9E000001B
:10018000F9E00000F9E00000F9E00000F9E000000B
:10019000F9E00000F9E00000F9E00000F9E00000FB
:1001A000F9E00000F9E00000F9E00000F9E00000EB
:1001B000F9E00000F9E00000F9E00000564B4CF2D5
:1001C000205210B51A804DF628121A8000BF00BFC9
:1001D0000DF096FF514B4FF010621A60504A9A6032
:1001E000504ADA60504A136813F4807304D14F49BF
:1001F0000B604FF4A85313604D4B1A78110703D5C9
:100200001A7842F008021A704A4B4B492A221A7097
:100210004A4A4B4B8B4204D252F8040F43F8040B6A
:10022000F8E7484B484900228B4202D243F8042B9E
:10023000FAE74649464A002352F8230041F82300D2
:1002400001336F2BF8D1434B434A802103F8011B44
:100250009342FBD1414B3D4A1A60414B8A221A70AE
:10026000A3F5805324225A70A0221A709A7992071B
:10027000FCD59A79D406FCD43A4A937903F00C035E
:10028000082B384BF9D103221A7140225A719A79FE
:100290009006FCD5334A9179324B4906FBD5324A58
:1002A000324911600221516020221A709A7902F0BD
:1002B0000C020C2AFAD12E4B2E4A1A602E4B2F4AD2
:1002C0001A6000225A60072243F8042C2C4AC3F813
:1002D0000C2D62B60EF09EFA144B1B68DA0705D59A
:1002E00028480EF06BF8284B284A1A60284B1B78D8
:1002F0005B0609D5244C254B22689A4204D121483B
:100300000EF05CF80023236012F056F90DF0FEFEAB
:1003100010F05CFEFEE700BF0E2005403080044078
:10032000823F04000100002B10D0034014D0034092
:1003300002D0074000E00740949CFF1F646001006A
:100340004088FF1F949CFF1F48A4FF1F0082FF1FCF
:100350000000000000E400E05FE400E008ED00E0E1
:100360000050064000400640448004400000030165
:1003700004800440C010050014E000E0FF76010096
:10038000000020201C1FEF5F1CE00340A5C3945A0F
:1003900000F00740FFFFFFFFFFFFFFFFFFFFFFFF32
:1003A000FFFFFFFFFFFFFFFFFFFFFFFFFFFFFFFF5D
:1003B000FFFFFFFFFFFFFFFFFFFFFFFFFFFFFFFF4D
:1003C000FFFFFFFFFFFFFFFFFFFFFFFFFFFFFFFF3D
:1003D000FFFFFFFFFFFFFFFFFFFFFFFFFFFFFFFF2D
:1003E000FFFFFFFFFFFFFFFFFFFFFFFFFFFFFFFF1D
:1003F000FFFFFFFFFFFFFFFFFFFFFFFFFFFFFFFF0D
:10040000FFFFFFFFFFFFFFFFFFFFFFFFDEF9FFFF23
:1004100010B5054C237833B9044B13B10448AFF33E
:1004200000800123237010BD949CFF1F000000007A
:1004300060600100084B10B51BB108490848AFF3D4
:1004400000800848036803B910BD074B002BFBD0A0
:10045000BDE81040184700BF00000000989CFF1F37
:1004600060600100949CFF1F0000000038B5044646
:10047000104621700A491D4611F086FE01464FF0D4
:100480007E5011F035FF074911F07EFEE560606097
:10049000256165610EF04EF9E061204638BD00BF70
:1004A000DB0FC9400024744938B50446104621705A
:1004B00009491D4611F068FE01464FF07E5011F0CB
:1004C00017FF064911F060FEE56060602561656117
:1004D0000EF030F9E06138BDDB0FC94000247449EB
:1004E00038B503780446032B20D8DFE803F01A1848
:1004F0001002C168406911F03DFD0D490546606874
:1005000011F0F6FE0146284611F0F2FE38BD08490A
:10051000406811F0EDFEE16811F036FE38BDC068AC
:1005200038BDC168406911F025FD38BD002038BDD7
:100530000024744970B504460E460EF0FBF80546DB
:10054000E069281A11F0CCFDE3682361E56166617A
:10055000A0610146606811F0CBFE0146A060104822
:1005600011F0C6FE11F09CF910F036FE11F0AEFC51
:10057000054601464FF07E5011F0FCFC616911F018
:1005800003FE21690646284611F0FEFD014630466D
:1005900011F0F2FCE0602046BDE87040FFF7A0BF1C
:1005A000000080BF38B50E201C4C0DF05BFC21888C
:1005B0001B4B884205461A881DDA0023511AB1F5F3
:1005C000805FAABF1B03C3EB03330131142093FBED
:1005D000F1F10DF005FF134B1988F1B923889D4205
:1005E00010DAC3F57F630F33282091FBF3F1BDE8E8
:1005F00038400DF0F5BE9042D4BFC1EB0003C1EB13
:100600000203DBE740F6FF718D42D4BFC3EB050167
:10061000C3EB0101C1EB0131E3E738BD9C9DFF1F36
:10062000649FFF1F049FFF1F10B5044610F016FCC7
:10063000204610BD70B44C88A04220D9012301335C
:10064000DBB21CB2660031F8144084421D46F6D37A
:10065000A04211D005F10045013D965B31F815101F
:1006600032F81530401AF21A00FB02F0641A90FBBF
:10067000F4F4E01870BC7047905B70BC70470226C1
:100680000125E5E700280CDA064A434282FB0320F5
:10069000DA17C2EB600000EB4000A3EB8000C0F172
:1006A0000C007047ABAAAA2A38B5234B1B78002B45
:1006B0002CD015200DF0D6FB204B1860204B1B884A
:1006C000984203DA1F4C237863BB38BD1E4A148856
:1006D000A042A4EB0302A8BF20467F2A1CDDC01A5B
:1006E000C001541C90FBF4F4002CEBD0154B1A788D
:1006F0000AB901221A70154D2B689C4204D0144B84
:10070000E1B2187809F030F92C6038BD11200EF0F4
:1007100045FF0A4B1860D1E7C01AC0EBC01090FB30
:10072000F2F4E1E70A4B0021187809F01DF90023E3
:10073000064A2370136038BDB89EFF1FC09CFF1F80
:10074000429DFF1F909FFF1F309FFF1F889FFF1F2D
:10075000189DFF1F38B50F200EF020FF1B4A1C4BC1
:1007600012881860C0F53B600830904220DB194BBE
:100770001B889842A3EB0204A8BF1846801A7F2C5E
:10078000C6BFC0010134C0EBC01090FBF4F47CB1D3
:10079000114B1A780AB901221A70104D2B689C422D
:1007A00004D00F4BE1B2187809F0DEF82C6038BDA8
:1007B000094C237803B938BD094B0021187809F09A
:1007C000D3F80023054A2370136038BDA09DFF1F96
:1007D000D89CFF1F1C9FFF1F409FFF1F509DFF1FA6
:1007E0003A9DFF1FF0B40E8886420DD203F10043FC
:1007F000013B31F81350854202D9F0BCFFF71ABF14
:1008000032F81300F0BC70471088F0BC704700BF8E
:10081000094B1B880C2B09D8084A80B252F82320B8
:1008200028B143F6FE73984203D9108C70471088A4
:1008300070470349FFF7FEBEEE9CFF1F043A01001C
:10084000A03B01004B4B4C4A2DE9F0471E88146831
:100850004A4BB442B3F80080494B33DB4445A8BF50
:100860004446A6421C60C8BF00202DDDC6EB080729
:10087000B7F5804F33DB80037B1C90FBF3F0FFF771
:10088000C7FF404A404B15881B88C0F3C61909FBB7
:1008900005F57F2D8246A8BF7F252BB3A64253DCEA
:1008A0004445D4BFC6EB0404C6EB08049F42CCBF4A
:1008B00003FB04445C43354BC8BF013794FBF7F797
:1008C0001F6013E034461E60C6EB0807A045D4BF86
:1008D000C6EB0800C6EB0400B7F5804FCBDAC0EBDF
:1008E000803090FBF7F0CAE7284A1360284C236851
:1008F000994508D0274B1B88002B34D1264B1B88E9
:100900006BBBC4F80090254C23689A4506D0214B58
:100910001B885A1F032A19D9C4F800A0204C236849
:100920009D420FD01F4B188848B11A4B1E4A1B8896
:10093000D35C834203D0C0B2E9B209F015F8256058
:10094000BDE8F087BDE8F0870024AFE7164AD05C29
:100950002030C0B20AF07F0109F006F8DCE7484613
:1009600009F0A2F8CDE7104A4946D05C08F0FCFF38
:10097000C4E700BF9C9DFF1F009FFF1F649FFF1FD8
:10098000B89CFF1FC89CFF1FCA9CFF1F689FFF1FCA
:10099000349DFF1FE89EFF1F8E9DFF1FE89CFF1FD9
:1009A000909DFF1FF69EFF1F208AFF1F2DE9F04F2D
:1009B00001208BB00EF0F2FDDFF870B3DFF870A30A
:1009C000CBF8000000200EF0E9FDBA4BCAF8000099
:1009D0001B880C2B00F05E82B74EB84A3188B84BAA
:1009E00052F8214000221A70B64BB74A1B88B7490B
:1009F0001288013B012A31F91330059300F0AE81D2
:100A0000B34B0193B34B0293B34FDFF8288300231A
:100A10000093B24B1B88012B00F0F481DFF8189390
:100A2000AF4B0393D9F80050AE4B04930023AE4A6A
:100A30001288013A032A00F24982DFE812F0A50089
:100A4000ED000400C9002846059311F049FBA749B1
:100A500011F09AFB059B0546184611F041FBA4498D
:100A600011F092FB0146284611F086FA11F052FD72
:100A70000546C9F80050386811F032FB9B4911F067
:100A800083FB8146009811F02BFB994911F07CFB08
:100A90000146484611F070FA11F03CFD3860954A65
:100AA000954B17881988954BDBF800201B88DFF8D9
:100AB0008CE2C7EB050C3D44039FC7F800C0471A02
:100AC000084404990D6001990F600299BEF8007006
:100AD00008609A4280F2E7800025C3EB070E744558
:100AE000DAF8000080F2D380611C984205FB01F522
:100AF0000EF1010E95FBFEF5C0F25F838742A8BFA1
:100B00000746FF1A01FB07F494FBFEF49A4200F338
:100B1000A780984200F3A480794C206811F0E0FA95
:100B2000784911F031FB784911F026FA11F0F2FC06
:100B3000A0F5FF531C3B082B98BF4FF40050D8F88A
:100B40000030184400282060C0F29F80B0F5804F2C
:100B500080F2F6806D4B1B781BB1B0F5005F40F062
:100B6000F7806B4D2B78002B40F0AB81694D2068EE
:100B70002B68634C984204D080B208F0C5FE23680D
:100B80002B600BB0BDE8F08F2846059311F0A8FA52
:100B9000614911F0F9FA059B0546184611F0A0FAD3
:100BA0005E4911F0F1FA0146284611F0E5F911F01D
:100BB000B1FC0546C9F80050386811F091FA564961
:100BC00011F0E2FA8146009811F08AFA53495DE784
:100BD0002846059311F084FA4A4911F0D5FA059B8D
:100BE0000546184611F07CFA4D4911F0CDFA014640
:100BF000284611F0C1F911F08DFC0546C9F80050E6
:100C0000386811F06DFA3F4911F0BEFA814600983C
:100C100011F066FA424939E72846059311F060FA67
:100C2000404911F0B1FA059B0546184611F058FAF3
:100C30003D4911F0A9FA0146284611F09DF911F03D
:100C400069FC0546C9F80050386811F049FA354981
:100C500011F09AFA8146009811F042FA324915E7EC
:100C60003388002B3FF458AF2B1B002BB8BF5B42DF
:100C7000092B00F32D81D8F80030214C4FF400509F
:100C8000184400282060BFF661AF00225AE0984265
:100C900005FB04F5B8BF002195FBFEF580F28482C8
:100CA00091FBFEF432E7BA42D4BFC3EB0205C3EBBB
:100CB000070512E7329FFF1F289DFF1F9C89FF1F1A
:100CC000BE9CFF1F3689FF1F069FFF1FE03E0100ED
:100CD0008C9FFF1F609DFF1FB09CFF1F989EFF1FF2
:100CE000249FFF1F9C9EFF1F7289FF1FCDCC4C3F8E
:100CF000CDCC4C3E2C8AFF1F7089FF1FFC9EFF1F2E
:100D0000D489FF1F9A99193FCDCC4C4546A0FF1FAF
:100D10008C9DFF1F3889FF1F3333733FCDCC4C3D73
:100D2000CDCCCC3E6666663FCDCCCC3D209DFF1F32
:100D3000E49CFF1F3C9FFF1F209FFF1F049DFF1F80
:100D400043F6FF72C04B22601B78002B3FF409AFC3
:100D500005F05AFFBD4B01221A7007E7BC4BBD4A94
:100D60001B88BD491278013B31F91350002A40F02D
:100D7000C78011200EF012FC0090B84B0193D3F8FD
:100D80000080009B984540F3C080B54BB54F1B8851
:100D9000B54A012B3B68B2F80090B44A0292204653
:100DA000A3EB050500F0E28011F09AF9029A52F8DF
:100DB000291011F0E9F90146002011F0DBF811F0DB
:100DC000A9FB009BC8EB05029D42B8BF1D4690429F
:100DD000C8EB050580F2DE8000FB0555013295FB6E
:100DE000F2F5A34BDFF8B4820293D8F800302B441D
:100DF00003EBD3735B10C8F800309E4B1B88012BAC
:100E00007FF40CAE9C4B03931D460F200EF0C6FBE7
:100E10002A6804929042034680F2CC80904A12885D
:100E2000012A00F03F81904A079012888F4D069268
:100E3000204611F055F9069ADFF8649255F8221011
:100E4000D9F8005011F0A0F90146002011F092F8F5
:100E5000059BEA1A059211F05DFB059A079B049920
:100E60009A42C1EB020EB8BF1A46704580F2448127
:100E7000521A00FB02220EF1010192FBF1F2D8F8A6
:100E800000107E4804900A4402EBD2725210C8F857
:100E90000020CCE57A4B1B78002B3FF49DAD794EBA
:100EA000794A3188794B52F8210001221A7011F0E9
:100EB00017F94FF07C5111F067F911F02BFB044644
:100EC00092E505F09DFE00232B704FE63868E6E5BD
:100ED00005F500500130001B11F002F96C496D4C12
:100EE00011F052F90546206811F0FAF86A4911F03C
:100EF0004BF90146284611F03FF811F00BFB1EE6B6
:100F000015200CF0AFFF009037E7594B0293D3F850
:100F10000080009B984542DA514B524F1B88524A41
:100F2000012B3B68B2F80090504A039220461D44C2
:100F300000F0E98011F0D4F8039A52F8291011F06A
:100F400023F911F0E7FA009B9D42C8EB0502A8BF08
:100F50001D46C8EB05059042BABF00FB055501329E
:100F6000454395FBF2F5DFF834813EE711F0B8F820
:100F7000029A52F8291011F007F911F0CBFA009BF0
:100F8000C8EB05029D42B8BF1D468242C8EB05056D
:100F90003FF722AF00FB05F595FBF2F521E7DFF8FF
:100FA000FC80304FD8F8003003EBD3735B10C8F8E7
:100FB00000302EE5314A049212680692904237DDE5
:100FC000274A1288012A00F0BC80274A099011881C
:100FD000264A08912046079211F082F8079A08994C
:100FE000DFF8BC9052F82110D9F8005011F0CCF87D
:100FF000059B2B44059311F08DFA0599099B069AE0
:101000009942C2EB010EA8BF1946704580F2BE801E
:10101000891A00FB01110EF1010291FBF2F2D8F8DE
:1010200000100A4402EBD2725210C8F80020FEE40D
:10103000D8F80020DFF8689002EBD2725210D9F88D
:101040000050C8F80020F2E446A0FF1F8C9DFF1F4F
:10105000788AFF1FB89EFF1F583B01008C9FFF1F1F
:10106000729DFF1FB09CFF1F0C9DFF1FF83E0100EB
:10107000609DFF1F989EFF1F249FFF1F9C9EFF1FC8
:10108000D49CFF1F289DFF1F9C89FF1FBE9CFF1F34
:10109000CDCCCC3ED489FF1F9A99193F3C9FFF1FAE
:1010A000209FFF1F464A08901188464A0791204614
:1010B000069211F015F8069A0799DFF80C9152F88C
:1010C0002110D9F8005011F05FF8059BE91A05913D
:1010D00011F020FA0599089B049A9942C2EB010E7F
:1010E000B8BF1946704558DA891A00FB01110EF194
:1010F000010291FBF2F2C2E60499521A00FB02F2DD
:1011000092FBFEF2BBE610F0EBFF039A52F82910B7
:1011100011F03AF80146002010F02CFF11F0FAF916
:10112000009A9542C8EB0503A8BF1546C8EB050514
:101130009842BABF00FB05550133454395FBF3F5D3
:1011400011E71F491F4A089020460D88079210F0AA
:10115000C7FF079ADFF8709052F82510D9F80050B1
:1011600011F012F80146002010F004FF059B2B44FB
:10117000059311F0CFF90599089B069A9942C2EBA5
:10118000010EA8BF19467045FFF642AF069A891AAC
:1011900000FB01F191FBFEF241E7049A891A00FB82
:1011A00001F191FBFEF26AE6B842D4BFC3EB000145
:1011B000C3EB070104FB01F172E51F46A1E400BF88
:1011C0000C9DFF1FF83E0100209FFF1F08B5244B18
:1011D0001B88FBB1234B1B78FBB1234B1B78E3B17E
:1011E000224B1B78CBB1224B1B78B3B1214B224849
:1011F0001A78C2B9214A2249008812880968024433
:10120000B1EB620F09DD01221A706420BDE80840CD
:1012100005F00EBD174A117801B908BD1370BDE87D
:10122000084008F015BC154A16490088128809685C
:101230000244B1EB620FF0DD00221A7008F008FCE6
:10124000642005F0F5FC642005F0F2FC642005F054
:10125000EFFC4FF41670BDE808400DF08DBA00BFEA
:10126000AA9EFF1F609FFF1F619FFF1F629FFF1FBE
:10127000639FFF1FEC9CFF1F049DFF1FFC9EFF1F31
:10128000209DFF1FE49CFF1F38B5114C23202578BB
:101290000CF0E8FD0F4A42F82500131F02F1C400CC
:1012A000002253F8041F83420A44FAD123780A49E2
:1012B00007480A4C0133DBB2322B81FB025108BFD5
:1012C0000023D217C2EB21120370226038BD00BF89
:1012D000CC9CFF1FAC9DFF1F1F85EB51F89EFF1F8D
:1012E0002DE9F04FB84CB94D2068B94F83B010F0DC
:1012F000F7FEB84910F048FF064610200EF04EF9F0
:1013000010F0EEFEB44910F03FFF314610F034FE0D
:1013100011F000F92988206088423B8843DA9E4614
:101320005B1A7F2B4FF0000247DDD2015E1C92FB5F
:10133000F6F2AA4EDFF8C882B6F800C0C8F800205E
:10134000BCF1190F00F0DF80BCF11A0F00F017811B
:10135000BCF11E0F00F020810126B146A04A128880
:10136000002A00F09D808842C0F207817045D4BFFA
:10137000C1EB0000C1EB0E009A42BABF02FB0000B5
:101380000133504390FBF3F3964A1360964B188851
:10139000C0B9964A1288AAB9954B197801B11A704A
:1013A00003B0BDE8F08F9842D4BFC1EB0002C1EB9F
:1013B00003029E465B1A7F2BB7DCC2EBC21292FB84
:1013C000F3F2B6E72988D4F800E0DFF80082DFF80E
:1013D000F8A171456CDCDFF818C29CF80020002AE7
:1013E0002ED14FF0010B04288CF800B028D1002E2C
:1013F00040F094817D4B18880028D1D0B9F1000FBE
:10140000CED023682C883A88A34280F265810023DD
:10141000141B7E2C774DD5BFC3EB8313C3EBC313D3
:101420005B00013493FBF4F42B680134A34203D036
:10143000C0B2E1B208F098FA2C6003B0BDE8F08FBA
:10144000012800F0F680022800F0EB800328D1D1BB
:10145000694B1B88092BCDD0002ECBD023682E885A
:101460003A88B34280F27B810023961B7E2EDFF800
:101470008CA1D5BFC3EB8313C3EBC3135B00013651
:1014800093FBF6F6DAF800300136B34203D0F1B23E
:101490004A2008F069FACAF80060ABE716469146A0
:1014A000BCF11E0F7FF472AF0022DFF858817EE09E
:1014B0004F4B1A78002A3FF473AF002401281C70A8
:1014C00000F0A480022840F00E81002E00F0A380DE
:1014D0004A4D2B68002B00F09E800420214608F026
:1014E00043FA424B2C60188800283FF459AFB9F1F9
:1014F000000F3FF455AFC0B2002108F035FA3D4B64
:1015000000221A604CE7DFF8FC8098F80020C2B196
:10151000DFF8D890B9F800A0BAF1000F11D0DFF8C9
:10152000E89099F800B0934578D05FFA8AF07F216F
:1015300008F01AFA98F80030B6F800C089F80030C0
:1015400010E0DFF8C49099F800A0924566D0274BD0
:101550000021187808F008FA98F80030B6F800C0B2
:1015600089F800301E4B1A88002A97D0BCF11E0F54
:1015700040F006810026B14619E00020FCE6DFF8C5
:10158000848098F80020002A0BBF012600264FF027
:1015900000094FF00109E1E6DFF86880104B98F888
:1015A00000601A88B6FA86F676094FF0000998F8B6
:1015B0000030002B3FF4E8AE2988B7F800E020683F
:1015C000C1EB0E03CFE600BF149DFF1FB09EFF1FAF
:1015D000AC9EFF1F9A99193FCDCCCC3E329FFF1F86
:1015E0006C9FFF1FA49DFF1F1C9DFF1F449FFF1F9B
:1015F000389FFF1FF89CFF1FE89EFF1FA89DFF1F3D
:10160000189FFF1FD49CFF1FD09CFF1F1EB1614D70
:101610002B68002B7BD1604B188865E70026B1460C
:101620009CE6002E3FF4E6AEDFF868A1DAF8002071
:101630002EE0002E3FF4DEAEB7F80080F045D4BFB8
:10164000C1EB0802C1EB0E02C1EB0808B8F17E0F36
:10165000DFF840A1D5BFC2EB8212C2EBC21252002A
:1016600008F1010892FBF8F8DAF8002008F1010807
:10167000424506D05FFA88F10120009308F074F922
:10168000009B1888CAF8008002287FF4DFAE42462B
:101690002168B5F800803888414559DA0021C8EB47
:1016A0000008B8F17E0FD3BFC1EB8111C1EBC111AE
:1016B00008F10108490091FBF8F808F1010890458C
:1016C00006D05FFA88F10420009308F04DF9009BE2
:1016D0001888CAF80080B9E69342D4BFC4EB03036C
:1016E000C4EB020394E6032827D12C4B1B88092B5B
:1016F00091D0002E8FD0274D2B68002B8BD04A2005
:10170000214608F031F9244B2C601888ECE621467C
:1017100008F02AF9204B2C601888E5E640207F214C
:101720008DE80C0008F020F9019B009A18885845B4
:101730001CD002287FF48AAE76E704287FF46BAFD2
:10174000002E3FF468AF2146402008F00DF962E713
:101750008142D4BFC8EB0101C8EB00019FE793426F
:10176000D4BFC6EB0303C6EB02037EE6B8F8001055
:10177000DAF800E0B7F800808E45FFF665AF5DE768
:101780002988B7F800E020680026C1EB0E03B146B7
:10179000E9E500BFA89DFF1F449FFF1FE89EFF1FB4
:1017A00008B5114B1B88022B09D0052B07D0032B42
:1017B00015D0042B0BD00D4B01221A7008BD7F21D0
:1017C000412008F0D1F8094B01221A7008BD7F2191
:1017D000092008F0C9F8054B01221A7008BD402104
:1017E000092008F0C1F8E6E7A29DFF1F469DFF1FF4
:1017F00038B5074B074D1B88052B044606D02B68D0
:10180000834203D0C1B2052008F0AEF82C6038BD89
:10181000A29DFF1F4C9FFF1F38B5124D124C2B8805
:10182000052B12D022684AB9022B0ED0033B012BA4
:1018300013D90E4A00231370236038BD0021052000
:1018400008F092F82B88022B04D10021412008F0E7
:101850008BF8EEE7052BE9D1F7E70021092008F026
:1018600083F8E6E7A29DFF1F4C9FFF1F469DFF1FC9
:10187000464B1B881D2B70B541D0454D0024454B70
:101880001B88022B16D0444B1B88022B54D028886F
:10189000424B002C1B780ADB8442A8BF044634B1BB
:1018A000002B3AD02046BDE87040FFF7A1BF002BC7
:1018B0002FD170BD3A4B1B78002B37D015200CF080
:1018C000D1FA384B1860384A1288002ADBD0374AE0
:1018D000186811888142D6DC354B2A881B888342E0
:1018E000A3EB0106A8BF03465B1AB242BABF02FBD4
:1018F00003330136534393FBF6F31C44C3E72A4BEF
:101900001C888CB12B4B224D1C78002CB7D02C8816
:10191000B5E7BDE87040FFF77FBFFFF741FF204606
:10192000BDE87040FFF764BF194DA8E711200DF026
:1019300035FE1C4B1860C6E70F200DF02FFE1A4B2A
:101940001D4A1B881060002BA1D01C4AC0F53B63C8
:10195000118808338B429ADB194A288812889342EF
:10196000A2EB0105A8BF1346A842A3EB010306DAC8
:1019700000FB0333013593FBF5F31C4488E700FBC0
:1019800003F292FBF5F31C4482E700BF329FFF1F76
:101990003A9FFF1F069FFF1F989EFF1F469DFF1F38
:1019A000B89EFF1FC09CFF1FA29DFF1F429DFF1FEF
:1019B000309FFF1FD49CFF1FD89CFF1FA09DFF1FBF
:1019C0001C9FFF1FF8B510200DF0E8FDC830B0F5E2
:1019D000FA7FC0F29680B0F57A6F0146A8BF4FF447
:1019E0007A6101F51673B3F57A6FA8BF4FF47A6385
:1019F0009BB289B2914A924C11802220238008F038
:101A000035F921888F4D904C242008F02FF90E20B5
:101A10000CF028FA40F6FF71C8308842A8BF08468B
:101A200020EAE07000F2DC5283B28A42A8BF0A4684
:101A30000220194622802B8008F018F92188042002
:101A400008F014F901200DF0A9FD044600200DF066
:101A5000A5FDA042B8BF204600F1C801B1F5FA7F4C
:101A6000C0F2D180B1F57A6FA8BF4FF47A6101F569
:101A70004873B3F57A6FA8BF4FF47A639BB289B20B
:101A8000724A734C11800A20238008F0EFF82188F5
:101A90000C2008F0EBF80F200DF080FDC0F53F6141
:101AA0000431B1F5AF6FC0F2AB80B1F5FA6FA8BFEA
:101AB0004FF4FA6189B2674BC0F54360B0F5AF6F80
:101AC0001980C0F29A80B0F5FA6FA8BF4FF4FA609F
:101AD00083B2614CA420238008F0C8F82188A62096
:101AE00008F0C4F815200CF0BDF900F59671B1F5B9
:101AF0002F7F0BDB41F25C23994240F3898019462A
:101B000008E040F24C434FF4FA7173E740F214538B
:101B10004FF42F71514A1180514C524D23800620B1
:101B200008F0A4F82188504E082008F09FF80027FC
:101B30004FF4AF74F9B24D4809F05CFE55F8043B20
:101B4000C3F5967300FB03F086FB0023C017C0EBC0
:101B50006310844207F10107A8BF0446062FE9D1AC
:101B6000434F414E0025E9B2424809F043FE57F881
:101B7000043BC3F5967300FB03F086FB0023C017FC
:101B8000C0EB6310844205F10105A8BF04460C2D8B
:101B9000E9D1394F344E0025E9B2384809F02AFE20
:101BA00057F8043B304AC3F5967300FB03F086FBFD
:101BB0000013C017C0EB6310844205F10105A8BFF4
:101BC00004460C2DE8D1A4F11401312931DD40F295
:101BD0003A73A4F5B97403FB04F482FB0432E417EE
:101BE000A4EB621289B232322548264B01801A607A
:101BF0002A20BDE8F84008F039B84FF4AF6368E731
:101C00004FF4AF6157E740F214534FF4FA7137E7DE
:101C1000124A00F5617089B2B0F52F7F1180B8BF0C
:101C20004FF42F73FFF678AF8342A8BF03469BB2F1
:101C300072E740F26C723221D6E700BFB09EFF1F00
:101C4000AC9EFF1F9C9DFF1F649FFF1FFC9EFF1FFC
:101C5000049DFF1FA09DFF1F1C9FFF1F429DFF1F94
:101C6000309FFF1F608AFF1FB5814E1BF09CFF1F36
:101C7000308AFF1F249DFF1F4089FF1F949DFF1F77
:101C80005E9FFF1F1C8AFF1F2DE9F04F0C2083B0C1
:101C90000CF0B4F80C200CF0A1FCC949DFF8A8A3A3
:101CA00014200CF0ABFCC749C74809F073FA0221B5
:101CB00003200CF039FD022104200CF035FD022137
:101CC00005200CF031FD022106200CF02DFD012134
:101CD0000A200CF029FD012109200CF025FD01212D
:101CE0000D200CF021FD012128200CF01DFD01210B
:101CF00014200CF019FD012116200CF015FD012116
:101D000017200CF011FD012121200CF00DFD022106
:101D10001C200CF009FD01211B200CF005FD002109
:101D20001B200CF0EDFC1C200CF0F0FCB0FA80F352
:101D30005B091A208AF800300CF036FF1F200021C2
:101D40000CF0F8FE04200CF0E1FC002800F0878184
:101D500005200CF0DBFC002800F0B28100239B4C36
:101D6000062023700CF0D2FCB0FA80F35B094FF030
:101D7000000B974A137006F01FFB2478002C40F0EC
:101D80006981584607F09CFF924B934A1B88934801
:101D9000128802709249934D40F23A72A3F5AF73E4
:101DA00002FB03F381FB0312DB17A3EB6213323355
:101DB00001210D202B600CF0A3FC64200CF0DCFC56
:101DC00006254FF416710A200CF00AFB00950C232F
:101DD0007D4A85485D2109F075FD002800F0AD8140
:101DE00064200CF0C9FC21460A200CF0F9FA4FF4EB
:101DF000967109200CF0F4FA00950C23724A7B4886
:101E00005C2109F05FFD002800F0848164200CF063
:101E1000B3FC214609200CF0E3FA4FF4967116202A
:101E20000CF0DEFA00950C23674A71485B2109F03B
:101E300049FD002800F04B8164200CF09DFC2146F8
:101E400016200CF0CDFA4FF4967117200CF0C8FA5A
:101E500064200CF091FC214617200CF0C1FA64209C
:101E60000CF08AFC21460D200CF04AFC614A6248C5
:101E70001268DFF8D891614F614D624EDFF8D08172
:101E800000230121FEF710FB01233C602C6034602D
:101E900089F8003004240F200DF080FB33680344E0
:101EA0000E2033600BF0DEFF3B6899F800201844E9
:101EB0003860002A7DD015200BF0D4FF2B68184421
:101EC000286004F0010080F0010004F0A1FEB8F8E1
:101ED0000030002B14BF4B20DC200CF04DFC013CEB
:101EE000D9D133683968454A2868474F002BB8BFB5
:101EF00003330029B8BF0331891011604349444AB4
:101F0000098814889B1000283360B8BF0330414E05
:101F10008210581A19442A60316038603E4D3F489B
:101F20003F49161B22442E6002600B60BBF1000F7C
:101F300040F0AE80B8F80030002B00F09C80394BA8
:101F4000012404201C600CF0E1FB18B9364B234A35
:101F50001C701070354B1B881C2B00F0A180344C7A
:101F600004F1C80523200BF07DFF44F8040F012085
:101F70000CF002FCA542F5D19AF8003023B12D4BAC
:101F80001B78002B40F09780002121200CF0B8FB3B
:101F9000294A2A4B1078187007F02EFE04F030FE04
:101FA0002749284845F6BF5203B0BDE8F04F0EF070
:101FB0000BBF11200DF0F2FA2B681844286080E75F
:101FC000001B374640420F007091FF1FF69CFF1F19
:101FD000A09EFF1F5E9FFF1F349FFF1F5C9DFF1F82
:101FE000B5814E1B1C8AFF1FF09CFF1F949DFF1F95
:101FF000249DFF1F3C89FF1FC49EFF1FC49CFF1F21
:10200000B09CFF1F209FFF1F249FFF1F2C8AFF1FD4
:102010007089FF1F9C9EFF1F8C9FFF1F609DFF1FED
:10202000749FFF1F2C9FFF1FDC9CFF1F329FFF1F11
:10203000A89DFF1FB29EFF1FB49EFF1F979EFF1F0C
:10204000A5050000549FFF1F9A9EFF1FB89EFF1F0B
:10205000F29EFF1F03B0BDE8F04F08F0AFBF0620AF
:102060000CF054FB00287FF473AE374C034620700D
:102070004FF0010B7DE64FF4FA7004F0D9FD04F047
:10208000C3FD06F0C3FC4FF4AF600CF075FB56E7E0
:10209000FFF798FCB8F80030002B7FF450AFEAE768
:1020A0002A4B188800283FF45AAF294BC0B2197840
:1020B00007F05AFC53E7012121200CF021FB67E7D0
:1020C00003200CF023FBB0FA80F35B0947E6032002
:1020D0000CF01CFB0028FAD104200CF017FB0028A0
:1020E000F5D105200CF012FB0028F0D106200CF0F1
:1020F0000DFB0028EBD10DF071FB04200CF006FB6A
:1021000040B905200CF002FB20B906200CF0FEFAC5
:102110000028F0D003200CF0F9FA0028FAD1ECE7FF
:1021200004200CF0F3FA40B905200CF0EFFA20B9C6
:1021300006200CF0EBFA0028DDD003200CF0E6FAC4
:102140000028FAD1ECE700BFF69CFF1F649DFF1F3B
:10215000109DFF1F2DE9F04FAD4C2678012E95B054
:1021600000F05582C0F00B82022E00F0D880A94901
:10217000A94A91F800801178A84ADFF83CE3A84DFD
:10218000A84FA948A94B0292A94A0092A94A9EF8D1
:1021900000B001922D78A84A3F7890F800E01B78B3
:1021A000DFF818A3DFF818C3DFF818930392012EA5
:1021B00084BF00222270A14AA1481370A14A80F86E
:1021C00000B01570A048A14A077082F80080A048AE
:1021D000A04A03709CBF013626701170BEF1000F3B
:1021E00040F074819C4A10880D2800F0B9819B4C06
:1021F00000202070024604462DB197480088002830
:1022000040F0BA810546964806882544002E40F0E5
:1022100067819448944C019E007836782478013088
:10222000A0EB4600002C40F05682039C94F800E09E
:10223000CEEB0004BEF1000F40F076820026DFF8FE
:1022400074E202989EF800E00078A41BA4EB4E0410
:102250003C44CBEB040410B1B7FA87F040099CF87A
:1022600000602718BC1B1EB11EF1000618BF012616
:10227000009F99F8000097F800909AF800C07B4FF3
:10228000C6EB040EC0EB0E00A0EB49008044C3EB8C
:102290000803A3EB41010C2313FB0C113960744BB1
:1022A000744F754C75481B880088D7F800C0744E71
:1022B0002788744C3688D4F800E0033BC0EBC00498
:1022C00003EB4303C7EBC70001EB830364446E4F8A
:1022D000334470446D4E57F8244056F820000C3BB0
:1022E0001D44254405440AB1694B1960694A1368C5
:1022F0009D4200F03181684B684819680791079941
:1023000001601B6808936648089B008815605B1A8B
:10231000834284BF634B1D6015B0BDE8F08FDFF8CA
:10232000A881614E08AF0025E9B2604809F062FA61
:1023300058F8043BC3F5967300FB03F086FB0023BB
:102340000135C017C0EB63100C2D47F8040BEBD11F
:10235000574B384D0195384DB3F800C00395109D8B
:1023600009980F99404EDFF8C0A0DFF8B490DFF86D
:10237000BC80654511AA8CCAAE46ACBF4FF0000EBA
:102380004FF0010E8445D4BF0020012030708C45F1
:1023900028480B9D1F4E8AF800E0D4BF0021012180
:1023A000017094452449DFF814A1D4BF0022012212
:1023B0000A709C453F4AD4BF00230123BC45AB466D
:1023C000D4BF002701271370AC45164B0C9D1F701E
:1023D000D4BF4FF0000B4FF0010B374B0F4A029266
:1023E000AC45DFF834C0124A83F800B0D4BF0025F2
:1023F000012589F8005098F800309CF8001096F8F4
:102400000080DFF8BCC02678DFF8B8900092CEE6F6
:10241000969EFF1FE49EFF1FE69EFF1F749DFF1FF9
:10242000EB9EFF1F449DFF1F989FFF1FE59EFF1F10
:10243000369FFF1F499FFF1F4A9FFF1F929FFF1F4D
:10244000939FFF1F949FFF1F959FFF1F969FFF1F46
:10245000979FFF1F379FFF1F9A9FFF1FD49CFF1F4F
:10246000BC9CFF1F2E8AFF1F809FFF1FEC9EFF1F3B
:102470000A9FFF1FA49DFF1F489DFF1F289FFF1F4E
:10248000CE9CFF1F689FFF1FF43C0100A036010097
:10249000789FFF1F3C9DFF1F64A0FF1F2C9DFF1F07
:1024A000429FFF1F849FFF1FB5814E1B949DFF1FFE
:1024B0005E9FFF1F4B9FFF1F459DFF1FA19EFF1F9C
:1024C000919FFF1F5C9FFF1F4089FF1FAF4AB048CD
:1024D00014880122182C027040F2058100248BE63A
:1024E000012E00F08F81022E00F0EE81032EA94B09
:1024F00000F01F811E78009B9CF800E01C78019B77
:1025000099F800C01878029B93F80080039B1F780D
:10251000A6EB4E03A4EB8404CCEB030CC0EB80765B
:102520000CEB0403C0EB8600034403EB480303EB0E
:10253000810327B198490978002940F0608201267B
:102540009AF800109548C1F1060101EB41013344AE
:1025500003EB81010160A2E69149924B0968D0E644
:10256000002D3FF444AE894A894E14880122182C6C
:10257000327040F2B8807446A0F10D0543E6DFF8F2
:102580007092894F0DF120080025E9B2874809F0C3
:1025900031F959F8043BC3F5967300FB03F087FB50
:1025A00000230135C017C0EB6310062D48F8040B5B
:1025B000EBD17F4BDFF83CA219880D9B00228B42A8
:1025C0008AF8002080F2A2807A4B8AF800507A497B
:1025D0007A4A7B4891F8008011787A4A1D700292FD
:1025E0000378794ADFF810C2DFF810920092774A38
:1025F000774E784D784892F800E0784A0192784A10
:1026000096F800B02D78077826780392CFE5DFF8AA
:10261000F081654E08AF0025E9B2724809F0EAF88A
:1026200058F8043BC3F5967300FB03F086FB0023C8
:102630000135C017C0EB63100C2D47F8040BEBD12C
:102640005B4B0C9D1F885F4B02935F4B00930B9B72
:102650000A98099ADFF8A0C1089EDFF8A0910F99A7
:10266000BB429E46ACBF4FF0000E4FF0010EAF4292
:10267000D4BF002501258742109B8CF80050D4BFA1
:1026800000200120504D89F800009742D4BF00225D
:102690000122B742D4BF4FF000084FF001082A7062
:1026A0009F42474A4448474E80F80080D4BF0023E9
:1026B00001231370129A414886F800E08F42D4BF7C
:1026C00000210121974201701ADC00224648DFF800
:1026D00024A102708BE7039C46B12678002E40F0BF
:1026E0006081441EABE50C3C012285E594F800E0D6
:1026F0000138CEEB0004BEF1000F7FF4A0AD9DE5E4
:10270000119A9742D4BF00220122DFE70C9A374B7F
:102710009142CCBF012200221A7040F34581052569
:102720008AF80050234B52E7002E3FF487AD012674
:1027300085E51C78009B029893F80080019B9CF82B
:1027400000601B7890F800C099F800700398A4EB23
:102750004604E71B90F800E0C3EB8374A8EB880005
:102760003844C3EB8403034403EB4C0303EB8103C2
:10277000BEF1000F40F0488101269AF8001007488A
:1027800033440C2414FB0131016088E5329FFF1FA4
:10279000D49CFF1F2E8AFF1F4B9FFF1FEC9EFF1F25
:1027A0002C9DFF1F64A0FF1FB5814E1BF09CFF1FD7
:1027B0005E9FFF1FAE9EFF1FE49EFF1FE69EFF1F52
:1027C000E59EFF1F749DFF1F369FFF1F989FFF1FF1
:1027D000459DFF1FEB9EFF1F449DFF1F499FFF1F4D
:1027E0004A9FFF1F249DFF1F0A9DFF1F639FFF1F1E
:1027F000608AFF1FA19EFF1F919FFF1F5C9FFF1F0D
:10280000308AFF1FA34CDFF89CE2207805909EF8E9
:10281000004001980494059C007801900134A4EBD9
:1028200040040498002840F0AF80039890F800E03E
:102830000498261ACEEB06000390BEF1000F40F07C
:102840009E8074460298944E0078029003983678E1
:102850000496041BA4EB460402983C44CBEB04040E
:10286000002800F08780B7FA87F040099CF80060E4
:102870002044871B1EB10498061C18BF0126009C2B
:1028800099F800002478BE1B301AA0EB4400804465
:102890000198C3EB0803A3EB4103002867D1BEF105
:1028A000000F40F0BB807344002C5ED100290CBFA8
:1028B00000206FF009009AF80010784C03440C20B7
:1028C00010FB01312160EAE4039E019C36780396F7
:1028D000009E2478019434786F4E714899F800E096
:1028E000009496F800906F4C9DF80C6086709DF8EF
:1028F0000460067080F806E09DF8006080F80390A0
:102900009CF800C02478DFF8B491DDF804E080F88A
:102910000880077180F805C0C671417244704FF09D
:1029200000080120009500215D4C0D465FFA88FCEF
:102930004F46764607E0022809D00A290BD014F842
:10294000016F17F8010F864201F10101F3D1013542
:102950000A29EDB2F3D1092D72D808F10108B8F1B6
:10296000100F36D019F80A0FDDE70020A3E74FF06B
:10297000000E98E7029879E7CEEB040003900198E7
:10298000041C18BF01245DE7019800284ED003986D
:1029900090F800E0BEF1000FEED1601E0390744687
:1029A00050E7841B01264AE40B9A3F4B9142CCBF6F
:1029B000012200221A703EDC0A9A3C4B9142CCBFA5
:1029C000012200221A7052DD03258AF80050384B8C
:1029D000FDE5304837490478C86B0299009D0978B5
:1029E00001342044CBEB0000084400219AF8004059
:1029F0002A4B401A0C2111FB040119604FE41BF112
:102A0000000618BF01269BE52349097800293FF4F9
:102A1000B3AE1BF1000618BF0126AEE604980028ED
:102A20000CBF4FF0000E4FF0090E3CE7039890F8F2
:102A300000E03046FDE604258AF800501C4BC6E550
:102A400014481C49047851F828000299009D09781F
:102A500001342044CBEB000066460844002BC4D070
:102A6000002EC2D1BBF1000FBFD00121BEE7099AF1
:102A7000114B9142CCBF012200221A7004DD0225C5
:102A80008AF800500A4BA2E5089B994218DD0125FF
:102A90009AE500BF2E8AFF1F4B9FFF1FEC9EFF1F72
:102AA000689DFF1F809FFF1F629FFF1F619FFF1F89
:102AB000AE9EFF1FDC89FF1F609FFF1FC43B01000C
:102AC000154B1D78012D25D9144A8AF8005012881B
:102AD000D2B1134A1288013A92B2062A14D8114A86
:102AE00012788AB1104A1268012A7FF470AD0F4A39
:102AF0000F4E10680C2290FBF2F102FB11023280A3
:102B00000C4A0321117062E5074A1268012A7FF41A
:102B10005EADF5E735465AE5AE9EFF1F149FFF1FD9
:102B2000B69EFF1F9E9DFF1F2C9FFF1F849FFF1FB0
:102B3000F09EFF1FD089FF1F2DE9F04F3A4B1B7805
:102B40008BB0002B6BD10E200BF08CF90FF0C8FA74
:102B500001463648364E374DFDF7ECFC3348FDF75D
:102B6000BFFC0FF0D7FC80F30C003060FFF7F2FAE7
:102B70002C68012C7AD0022C00F0B182032C00F0DA
:102B8000C3832D4E2D4C33682D4A2E4E0993099B3D
:102B9000316812882360591A013A9142274F00F296
:102BA0009982294E32689A1A0D2A00F28282274EA3
:102BB00032689A1A132A00F27782254E32689A1ADE
:102BC000252A1AD9234B1B88002B40F05B81224B0E
:102BD0001B78002B40F05681FEF756FB1F4B1B88DD
:102BE0001B3B9BB2022B04D81D4B1B78002B40F0E3
:102BF0004C8104F02FF8236833601A4D2A689B1A21
:102C0000502B00F20D82184B1B88012B00F02582FF
:102C100006F050FE06F034FD0BB0BDE8F08F08F072
:102C200059F80BB0BDE8F08FF69CFF1FC49EFF1F44
:102C3000009FFF1F2C9FFF1F64A0FF1FC09EFF1F50
:102C4000D889FF1F989DFF1F809DFF1F549DFF1F68
:102C5000589DFF1FAA9EFF1FEC9CFF1F329FFF1F66
:102C6000D49CFF1FA49EFF1F049FFF1FDFF820932B
:102C70009F4AB9F800001378834204D0C3B21846C3
:102C8000137006F009FEDFF804839A4AB8F80030A2
:102C90001178994204D0984F3978002940F0F08695
:102CA000964A33681288964E9A42C0F2F880954A46
:102CB0001278002A40F0F380DFF8D8A2BAF800308A
:102CC00023B9914B1B88002B00F005858F4A904B50
:102CD00011881B888F4A0B4412685B1093428E4AFE
:102CE000126880F2A78400219342B4BF01230B46EF
:102CF00004910093ACBF4FF0010B8B4605910E2061
:102D00000BF0B0F8854B864A1B68176803930133B4
:102D1000A7F25232002B8446029240F3C286802BE7
:102D2000A8BF80237F4A804912780191002A00F0D1
:102D3000C0800978914200F0BC80B8F80010DFF83C
:102D40004CE2994201F0AB806B49AEF80030774B12
:102D50004FF0010E81F800E01978DFF83CE2019BAA
:102D60008EF800101A70009B002B00F01781BAF843
:102D70000030002B00F012816D4B1B685A1C002A9A
:102D800040F39386802A00F38F866A4C6A496B4829
:102D90002488098800682144B0EB610FC1F2F382F6
:102DA000A3F148020F2A02D8473BA9F800300E20B1
:102DB0000BF058F86FF454731F44874202DC604BE9
:102DC00000221A705F4B1B88002B00F02B845E4B97
:102DD0005E4A1B781178994243D0002B41D05C4960
:102DE0000C78002C00F025875A4991F800C0BCF1FE
:102DF000000F40F01C87584F0097584F58480297D3
:102E0000554F007887F800C0544F4FF0010E87F8F7
:102E100000C081F800E0002841F091805149097814
:102E2000002900F0E587504903910C4609780029F4
:102E300040F0DB874D48494F0078397001210297F7
:102E4000217070B1444843490090494803270770F6
:102E5000002008700099029F0870039901243C70BB
:102E600008701370434B1B88A3F11B02012A40F228
:102E7000CB851D2B7FF486AE3C4A3F4B12781A70EF
:102E80003E4C80E6FEF7A2F9A6E63D4B1B78002BF0
:102E90003FF4AFAE2B68012B7FF4ABAEABE63168ED
:102EA000384A069106983849106002220B602A6061
:102EB00002E71E49DFF8E0E0097800293FF44FAF50
:102EC0009EF8000081423FF44AAF03984B2840F33C
:102ED000AD871833802BB8F80000A8BF8023984234
:102EE0003FF43DAF2948038003480123037036E7D0
:102EF000979EFF1F5C9DFF1FDC9CFF1F9C9DFF1F7B
:102F000064A0FF1FEC9CFF1F869DFF1F049DFF1FF9
:102F1000FC9EFF1F209DFF1FE49CFF1F789FFF1F4B
:102F2000C49CFF1F6E9FFF1F389DFF1F6F9FFF1FD9
:102F3000EC9EFF1FB09EFF1FAC9EFF1F149DFF1F46
:102F4000FC9CFF1FB69EFF1F0A9DFF1FB49CFF1F26
:102F5000959FFF1FF49EFF1F489FFF1F9E9DFF1F11
:102F6000969FFF1F929FFF1FB59CFF1FD49CFF1FC2
:102F7000D089FF1F329FFF1FD09CFF1FC09EFF1FE5
:102F8000379FFF1F4C9DFF1FBC9EFF1F349FFF1FDD
:102F9000B49EFF1F409DFF1F399DFF1F029B9C4554
:102FA000BFF605AF8B4B1B88002B3FF400AFBBF186
:102FB000000F7FF4E1AE884B1B881BB1059B002BF3
:102FC0007FF4DAAE049B002B3FF4F1AE834B1A780A
:102FD000002A7FF4ECAEDFF8809299F800400122DD
:102FE0001A70002C40F044837D4B1B78002B02F0BC
:102FF00060807C4B1B78002B02F03E837A4B1B7861
:10300000002B7FF4D4AE794B1B78002B3FF4CFAE6E
:10301000B8F8003076490A3BA8F800300A70C6E6D6
:1030200005F012FA734B1B7873B9734B1B785BB9BD
:10303000724B1B7843B9724B1B782BB9714B1B78C1
:1030400013B903F0DDFD01E003F0E6FD23682B601A
:103050006D4B1B88012B7FF4DBAD6C4A6C4B116808
:103060006C481A78A1F118032A2101FB03F10160D1
:10307000002A00F0C182684C2368994200F36A83F9
:1030800010DA66480278002A40F04687644A1068E1
:10309000D0F17F0048BF0330801001301B1A9942E5
:1030A00042F34E862160A9E2FEF7E2FB236833601B
:1030B00083E5FDF77BFCFEF713F95A4B1B88032BC6
:1030C00000F01385584B1B88032B00F00A852368FA
:1030D00033606CE5FDF7B6FB3B68336061E5534A4E
:1030E00034681188A14204DB464B1B78002B00F0AA
:1030F00061834F4E4F48336807934F4B079A0068E0
:103100001B88121A9A4200F2AD80002B00F0AA80B0
:103110004A4B1A88002A3FF435AD494B49481B6891
:103120000088A342B8BF2346994241F32281464B0F
:103130001960DFF8288188F80020344FFDF782FB02
:1031400038687F2840F36F85404B7F3883FB00321F
:10315000C317C3EB620303EB4303A0EB830073309D
:103160003B4B01931B883860002B40F09186234B2A
:1031700000931B78002B00F0C883364C2378002B7B
:1031800000F0C383DFF8D890DFF8C0A04FF0000B49
:103190000CE003F17300C0B298F8001006F014FCC4
:1031A00023780BF1010B5B4540F3AF833B6859F883
:1031B000040F1844A0F17F038AFB0321DA17C2EB46
:1031C000610202EB42027F28A3EB8203E1DCFDF700
:1031D00059FAE0E7869DFF1FBA9EFF1FFC9CFF1F68
:1031E000929FFF1F939FFF1F949FFF1F959FFF1F9D
:1031F000DC9CFF1F9E9DFF1FF49EFF1F489FFF1F2B
:10320000B59CFF1FEC9CFF1F049FFF1F849FFF1FA7
:10321000469DFF1F789DFF1F889DFF1F509FFF1F2A
:103220004C9FFF1F069FFF1F989EFF1F9C9DFF1F27
:1032300064A0FF1F4C9DFF1F849DFF1FD29CFF1F9A
:10324000BC9EFF1F649FFF1FB89CFF1FABAAAA2A4A
:103250001A9DFF1F9889FF1FA19EFF1F759DFF1FCD
:103260007089FF1F554B564A1B681088554AA34268
:10327000B8BF2346994200F38482534C128883429C
:10328000A8BF03462360002A7FF453AF9942C8BF0A
:10329000134640F37D82401AB0F5804FAABF9B03CE
:1032A000C3EB8333013093FBF0F0FDF7B1FAC0F3C9
:1032B000C6100EF015FF454B044618880EF010FF9F
:1032C0004349074620460EF05FFF014638460EF0A0
:1032D0005BFF21460EF050FE4FF07E5104460FF08A
:1032E000F1F8002841F03A803A4920460FF008F9F9
:1032F000002840F01E8620460FF032F9C0B2DFF8F9
:10330000F48088F8000018E7334B34681988A1422C
:1033100074DD324B1B78002B70D1DFF8DC9099F80C
:1033200000007F2840F3F485A3F155337F3803F183
:10333000004383FB0032C317C3EB620303EB430379
:10334000A0EB83007330264B01931B88C0B289F831
:103350000000002B40F0E387224B00931B78002BEA
:1033600000F09484204C2378002B00F08F841F4FB2
:10337000DFF87C804FF0000A0AE003F17300C0B26E
:1033800006F046FB23780AF1010A534540F37E8498
:1033900057F8043F99F800001844A0F17F0388FB18
:1033A0000321DA17C2EB610202EB42027F28A3EB92
:1033B0008203E2DCFDF766F9E1E700BFBC9EFF1F78
:1033C000649FFF1FD29CFF1FB89CFF1F709FFF1FB1
:1033D000CDCCCC3D0000FE429C9DFF1FEC9CFF1F0E
:1033E0001A9DFF1F489FFF1F9889FF1F7089FF1FAD
:1033F000ABAAAA2A759DFF1FEA9EFF1FB84F386827
:103400007F2840F3CC81B74B7F3883FB0032C31752
:10341000C3EB620303EB4303A0EB83007330DFF8DD
:10342000249399F800A0824500F01582AE4B1B88CA
:10343000002B43D1AD4AAE4812680088914205DCAA
:103440008242D4BFC1EB0203C1EB0003411AB1F5C4
:10345000804FA6BF9B030131C3EB833393FBF1F095
:10346000FDF7D6F9C0F3C6100EF03AFEA14B0446A4
:1034700018880EF035FEA049804620460EF084FEE6
:10348000014640460EF080FE21460EF075FD4FF0DD
:103490007E5104460FF016F8002840F0BA8697498E
:1034A00020460FF02DF8002840F0408520460FF010
:1034B00057F8C0B2DFF8908288F80000BAF17F0FA9
:1034C00040F3A3838748AAF17F0A80FB0A304FEAC2
:1034D000EA73C3EB600000EB4000AAEB800073309E
:1034E000874B00931B78C0B289F80000002B40F096
:1034F0000383844B03931B78002B40F0EC84824BB6
:1035000002931B78002B40F02C87804B0193029B89
:103510001B78FBB17E4B1B88012B00F0F885022B3A
:1035200000F08087032B01F02181042B01F021831F
:10353000052B01F0C183062B01F08785072B01F0D5
:103540004387082B02F04980092B02F010810A2BD7
:1035500002F01083009B1B78002B00F05984019B24
:103560006A4C1988002900F0AF8438687F2840F33E
:10357000C0825C4B7F3883FB0032C317C3EB62030E
:1035800003EB4303A0EB830073303860002940F065
:103590005E84009B1B78002B00F069815D4C2378D2
:1035A000002B00F06481DFF8A4A1DFF89C814FF0CC
:1035B000000B0CE003F17300C0B298F8001006F0A5
:1035C00003FA23780BF1010B5B4540F350813B6814
:1035D0005AF8040F434A1844A0F17F0382FB0321E9
:1035E000DA17C2EB610202EB42027F28A3EB8203EF
:1035F000E0DCFDF747F8DFE7474B1960474B1B68F6
:10360000A92202FB03F3002BBCBF03F57F533F331A
:103610009B13543B194481F30C0128200AF0E0FE6F
:10362000FFF7F6BA384C3E483549364A23700370E6
:103630000B7016E493424FF0000B80F2B38001232D
:10364000CDF800B0CDF814B00493FFF758BB354B5C
:103650001B78002B7FF4ABAB039B334A243B83F3F3
:103660004703D9B25B20136006F07EF999F8004059
:10367000032C30D1DFF8D88098F80030002B42F0CE
:10368000E4812A4F3B78002B42F0D281254C2378ED
:10369000002B42F0C081264B1B78002B42F0AE81FC
:1036A000244A1380244B1B78002B42F000810E4BE0
:1036B0007F221A8098F800306BB93B785BB9237889
:1036C0004BB91E4A7F210720138006F04DF97F2158
:1036D0000B2006F049F91A4B1F68FFF768BB00BFC3
:1036E000849FFF1FABAAAA2AD29CFF1FB89CFF1F72
:1036F000649FFF1F709FFF1FCDCCCC3D0000FE429A
:10370000489FFF1FB59CFF1F9E9DFF1F1A9DFF1F17
:10371000B69EFF1F9889FF1F889DFF1FD489FF1F3A
:10372000F49EFF1F959FFF1F009DFF1F949FFF1F8B
:10373000939FFF1F8E9DFF1F969FFF1FE89EFF1FF9
:10374000C49CFF1FEA9EFF1F759DFF1F7089FF1F0E
:10375000929FFF1FB54A1078002840F03D83B44A7D
:103760001268D2F17F0248BF033203EBA202531C5E
:10377000B04A23609942B8BF1160FFF63FAF1946C7
:103780003CE7AD4B12881960002A7FF4D2AC0B469F
:103790009842D4BFC1EB0003C1EB03037BE5FCF708
:1037A00071FF3CE60123CDF810B0CDF800B00593D1
:1037B000FFF7A5BA01232B60FFF7E3B9029B1B7843
:1037C000FBB19E4B1B88012B00F01A84022B00F0EA
:1037D000A786032B01F04080042B01F0EF81052B1D
:1037E00001F0E082062B01F03984072B01F03985C6
:1037F000082B01F0A386092B02F022800A2B02F08D
:103800007F81019B1B88002B00F02A83009B1B7883
:103810003BB9039B1B7823B9029B1B78002B00F05C
:103820009B87874B1B78002B00F0FE8085490B7827
:10383000082B00F2F98084483A680068834C013311
:10384000DBB25F1E101A44F827000B70804B3468FF
:10385000198889F800208C427E4E7FF793A9326840
:103860007D4B0892089A7D4C1A60FFF78CB9039B38
:103870001B78002BA2D03B68A3F10C007F2840F3FB
:10388000338377488B3B80FB0320DA17C2EB600061
:1038900000EB4000A3EB800303F17300DFF8D48159
:1038A000C0B298F8001006F08FF8009B1B78002B30
:1038B00084D0644C2378002B80D0DFF8BCA14FF07B
:1038C000000B0CE003F17300C0B298F8001006F092
:1038D0007BF823780BF1010B5B457FF76FAF3B68FB
:1038E0005AF8040F5E4A1844A0F18B0382FB0321AF
:1038F000DA17C2EB61020C3802EB42027F28A3EB1D
:103900008203DFDCFCF7BEFEDEE74D4B1B78002BAD
:1039100040F0AC823B68534A1278002A45D0A3F1AC
:103920000C007F2840F3F1824D4A8B3B82FB032140
:10393000DA17C2EB610202EB4202A3EB820303F14E
:103940007300C0B298F8001006F03EF8009B1B7898
:1039500053B33C4C23783BB3DFF81C91DFF800A154
:103960004FF0000B0BE003F17300C0B298F80010A9
:1039700006F02AF823780BF1010B5B4514DD3B6858
:1039800059F8040F1844A0F18B038AFB0321DA17BE
:10399000C2EB61020C3802EB42027F28A3EB8203E8
:1039A000E1DCFCF76FFEE0E73B682F4A1278FAB1E2
:1039B000224A1288012A00F02F84022A00F0318660
:1039C000032A00F0C687042A01F01F81052A01F0AE
:1039D0005C82062A01F06683072A01F09D83082A8B
:1039E00001F05D86092A01F0F9860A2A02F0548066
:1039F000019A1288002A00F044821C4A174C137066
:103A000003232B60FFF7BFB8DFF8708098F8003011
:103A1000002B40F0FE80164F3B78002B40F0C68410
:103A20000E4C3B70FFF7AFB83A680FE7509FFF1F8F
:103A30004C9FFF1F889DFF1FB89CFF1FB69EFF1F56
:103A4000F49EFF1F9889FF1FE09CFF1F7489FF1FD2
:103A50009C9DFF1F64A0FF1F30A0FF1FC09EFF1F83
:103A6000ABAAAA2AB59CFF1F9E9DFF1FEA9EFF1FBF
:103A7000D09CFF1F759DFF1F7089FF1FD49CFF1FE7
:103A8000DBB21846137006F02DF8A54BA5491A466F
:103A9000A54B184600230B703B7013700370FFF7A3
:103AA000FFB80123FFF73EB98024A049A04BA14AEB
:103AB00009881B8812680B44B2EB630FBFF677A925
:103AC0009D4B1B78002B40F0F081B8F800309B4AEA
:103AD000A3423FF46CA99A4B148001221A70FFF79D
:103AE00066B9FCF737FEFFF7F2BAFCF7DDFDFFF72A
:103AF000E9BAFCF7C7FD48E5924B01931B8863BB0D
:103B0000894B0393904B0293904C23787BB3DFF85F
:103B10005882DFF83CA24FF0000B09E003F173007C
:103B2000C0B205F075FF23780BF1010B5B451EDD7C
:103B300058F8043F99F800001844A0F17F038AFB6D
:103B40000321DA17C2EB610202EB42027F28A3EBEA
:103B50008203E3DCFCF796FDE2E7734B03937A4BB9
:103B6000029305F055FF009B1B78002BCCD1039BE3
:103B70001B78002B3FF4CBAC99F80030A3F10C007C
:103B80007F2840F3BF8172488B3B80FB0320DA170C
:103B9000C2EB600000EB4000A3EB800303F1730075
:103BA000C0B205F035FF009B1B78002B00F09F8111
:103BB000664C2378002B01F05D82DFF8AC81DFF8E2
:103BC00090A14FF0000B0AE003F17300C0B205F0C2
:103BD0001FFF23780BF1010B5B457FF798AC58F87A
:103BE000043F99F800001844A0F18B038AFB0321DD
:103BF000DA17C2EB61020C3802EB42027F28A3EB1A
:103C00008203E1DCFCF73EFDE0E75046FCF73AFDBD
:103C100066E4504A1278002A40F09E814E4F4F4C85
:103C20003B70FEF7B0BFFCF72DFDFFF799BA0020FF
:103C300008704B49087840B139490091097800294A
:103C400000F07A81009F00213970464909780029E7
:103C50007FF4E9A8002C40F0CB80002840F0C88019
:103C6000354C2F4F94F800E02F4C0394364C0294BF
:103C70002D4C2C492070344C0097087038702070FF
:103C8000BEF1000F7FF4E1A8FFF7EBB8264B1B78DD
:103C9000002B6BD099F80030A3F10C007F2840F383
:103CA00090832B4A8B3B82FB0321DA17C2EB610224
:103CB00002EB4202A3EB820303F17300C0B205F0F2
:103CC000A7FE009B1B78002B50D0204C2378002BA4
:103CD0004CD0254FDFF878804FF0000A09E003F15F
:103CE0007300C0B205F094FE23780AF1010A53452F
:103CF0003CDD57F8043F99F800001844A0F18B030D
:103D000088FB0321DA17C2EB61020C3802EB420296
:103D10007F28A3EB8203E2DCFCF7B4FCE1E700BF01
:103D2000489FFF1FF49EFF1FB59CFF1FB09EFF1F03
:103D3000AC9EFF1F149DFF1FD49CFF1F349FFF1FCD
:103D4000DC9CFF1F1A9DFF1F9E9DFF1F9889FF1F70
:103D5000ABAAAA2A379FFF1FD09CFF1FC09EFF1F40
:103D6000969FFF1F929FFF1F7089FF1F904B1B782C
:103D7000FBB1904B1B88012B00F07486022B00F0E6
:103D80006E87032B01F0E480042B01F07E81052B6C
:103D900001F0B983062B01F05484072B01F09485C0
:103DA000082B01F01087092B01F07E870A2B01F008
:103DB0005C87019B1B88002B00F0BA827E4B1B782E
:103DC000002B40F0B0827D4B7D4A1988346800207A
:103DD000012310602B603EE50130C0B2022886BF8F
:103DE000002111701070194608E403980021017039
:103DF0007449097800293FF434A86D490291097883
:103E0000002900F05287029800210170FFF729B8BD
:103E1000039B1B78002B7FF4A2AB029B1B78002B2B
:103E20007FF49DAB019B1988FFF79FBB243B002BC0
:103E3000B8F8000040F3748498423EF490AF9BB20F
:103E40006148A8F8003001230370FEF788BFDFF84F
:103E50007C81C0B298F8001005F0B6FDFFF799BB61
:103E60005A4B3878197805F0AFFDCFE47F21402018
:103E700005F07AFD5649574A3B680B6000211170E6
:103E800049E5D8B298F8001005F09EFD3B68B4E50E
:103E9000C0B298F8001005F097FDFFF768B94E4BD7
:103EA000DFF854E11978FEF75ABF4B2C40F34582F6
:103EB0001834802CB8F80030484AA8BF8024A342A8
:103EC0007FF409AEFEF773BF99F8000005F0A0FD7E
:103ED0002188FFF74ABB424B01931B88002B41F01E
:103EE0003387334B029347E6FCF7CCFBD6E4029BC7
:103EF0001B78002B7FF40EAB039B1B78002B7FF409
:103F00002EAB8FE7FCF7BEFB4AE6FCF7BBFB18E5E0
:103F1000FCF7B8FBFFF717BA0132D2B2022A40F21F
:103F20005682002202701946FFF768BB7F20FFF718
:103F3000C1BA7F20FFF7E3B91D4F1F4902974FF029
:103F4000000C81F800C0009F02994FF0010E87F825
:103F500000E081F800C078E6224F387802F0E4FEF5
:103F6000214B1B78002B00F040823B887E2B00F217
:103F70003C821E4CDFF884902268D9F80010521A57
:103F80000F2A40F229821A4A0133108899B23980E7
:103F9000002800F04382C9B2C0B205F0E5FC154F1D
:103FA000226898F80030C9F800203B70FEF7EBBD9E
:103FB0009E9DFF1FB69EFF1FF49EFF1F9C9DFF1F2F
:103FC000B89CFF1FD49CFF1FDC9CFF1F759DFF1F2B
:103FD000E09CFF1F9889FF1F6F9FFF1F349FFF1FEB
:103FE0001A9DFF1F109DFF1F979FFF1FC09EFF1F61
:103FF000649DFF1FD09CFF1F399DFF1F7C9FFF1FEB
:10400000DFF89CA33868BAF80030E04AE04CC31AE5
:1040100082FB031ED917C1EB6E0101EB4101A3EB3B
:10402000810303EB430354F8233018447F2840F303
:1040300007857F3882FB0032C317C3EB620303EBB3
:104040004303A0EB83007330DFF85883DFF858B3E5
:1040500098F80010C0B205F0B7FCBBF80030022B96
:104060007FF6CFAB3968BAF80030C84ACB1A82FB6A
:10407000030ED817C0EB6E0000EB4000A3EB8003EB
:1040800003EB430304EB8303586808447F2840F3A1
:10409000EE867F3882FB0032C317C3EB620202EB6D
:1040A0004202A0EB82007330C0B298F8001005F015
:1040B0008BFCBBF80030032B7FF6A3AB3968BAF852
:1040C0000030B24ACB1A82FB030ED817C0EB6E0049
:1040D00000EB4000A3EB800303EB430304EB8304FA
:1040E000A06808447F2840F37D817F3882FB00323E
:1040F000C317C3EB620202EB4202A0EB82007330F3
:1041000098F80010C0B205F05FFCFFF77ABBDFF84B
:1041100090A299F80000BAF800309C4A9C4CC31A4F
:1041200082FB031ED917C1EB6E0101EB4101A3EB2A
:10413000810303EB430354F8233018447F2840F3F2
:1041400005847F3882FB0032C317C3EB620303EBA5
:104150004303A0EB83007330DFF84CB2C0B205F02C
:1041600057FCBBF80030022B7FF6F4A999F8001039
:10417000BAF80030854ACB1A82FB030ED817C0EB81
:104180006E0000EB4000A3EB800303EB430304EB62
:104190008303586808447F2840F36D867F3882FB8C
:1041A0000032C317C3EB620202EB4202A0EB8200B3
:1041B0007330C0B205F02CFCBBF80030032B7FF647
:1041C000C9A999F80010BAF80030704ACB1A82FBDE
:1041D000030ED817C0EB6E0000EB4000A3EB80038A
:1041E00003EB430304EB8304A06808447F2840F3F7
:1041F000C7807F3882FB0032C317C3EB620202EB39
:104200004202A0EB82007330C0B205F001FCFFF760
:10421000A1B90120FFF74EB9DFF884A15B49BAF8D4
:1042200000205B4C9A1A81FB020ED017C0EB6E0087
:1042300000EB4000A2EB800202EB420254F82200A5
:1042400018447F2840F30084A0F17F0381FB032101
:10425000DA17C2EB610000EB4000A3EB8000733083
:10426000DFF844B198F80010C0B205F0ADFBBBF820
:104270000030022B50D93968BAF80030434ACB1AC3
:1042800082FB030ED817C0EB6E0000EB4000A3EBDF
:10429000800303EB430304EB8303586808447F283F
:1042A00040F3B9867F3882FB0032C317C3EB62024A
:1042B00002EB4202A0EB82007330C0B298F800100B
:1042C00005F082FBBBF80030032B25D93868BAF81B
:1042D00000302E4AC31A82FB031ED917C1EB6E01B0
:1042E00001EB4101A3EB810303EB430304EB8304E4
:1042F000A36818447F2867DD7F3882FB0032C3172C
:10430000C3EB620202EB4202A0EB82007330C0B248
:1043100098F8001005F058FB3B68FFF769BB05F003
:1043200077FBFFF719B80021402005F01DFB4AE597
:1043300099F8000005F06CFB40E5243C002CB8F82F
:10434000003040F39C85A3423EF431ADA4B2114B42
:10435000A8F8004001221A70FEF729BD0120FEF7DF
:10436000CEBF0D4B01931B88002B3FF4D0A8FFF765
:10437000F8BB0A498342A8BF03460B60FEF7D9BECB
:10438000FCF780F940E71446FFF79ABBABAAAA2ACC
:10439000C83A0100DC9CFF1F1A9DFF1FB89CFF1F3D
:1043A000F09EFF1F759DFF1FF49CFF1FDF4BE04C2D
:1043B00019886A2005F05AFC98F800303B70FEF727
:1043C000E2BBFCF75FF979E4FCF75CF99FE7027068
:1043D0001946FFF713B9D64CD64F98F800303B700A
:1043E000FEF7D1BBFCF74EF98AE6D34B1B78002BC6
:1043F000F1D03B88CD4F002BEDD0CD4CDFF848936A
:104400002268D9F80010521A0F2AE5D9CB4A013B8D
:10441000108899B2398000287FF4BDADC8B205F08C
:1044200043FBBCE5DFF824A399F80000BAF800309C
:10443000C34AC44CC31A82FB031ED917C1EB6E01D9
:1044400001EB4101A3EB810303EB430354F8233059
:1044500018447F2840F3FD837F3882FB0032C31766
:10446000C3EB620303EB4303A0EB83007330DFF87D
:10447000E0B2C0B205F0CCFABBF80030022B7FF6F8
:1044800069A899F80010BAF80030AD4ACB1A82FB3F
:10449000030ED817C0EB6E0000EB4000A3EB8003C7
:1044A00003EB430304EB8303586808447F2840F37D
:1044B000DD857F3882FB0032C317C3EB620303EB59
:1044C0004303A0EB83007330C0B205F0A1FABBF840
:1044D0000030032B7FF63EA899F80010BAF80030A0
:1044E000974ACB1A82FB030ED817C0EB6E0000EB85
:1044F0004000A3EB800303EB430304EB8304A068B9
:1045000008447F287FF73CAF7F3882FB0032C31717
:10451000C3EB620303EB4303A0EB8300733073E64A
:10452000DFF828A23868BAF80030854A854CC31AEB
:1045300082FB031ED917C1EB6E0101EB4101A3EB16
:10454000810303EB430354F8233018447F2840F3DE
:1045500059837F3882FB0032C317C3EB620303EB3E
:104560004303A0EB83007330DFF8E881DFF8E0B1AC
:1045700098F80010C0B205F027FABBF80030022B03
:104580007FF63FA93968BAF800306D4ACB1A82FB32
:10459000030ED817C0EB6E0000EB4000A3EB8003C6
:1045A00003EB430304EB8303586808447F2840F37C
:1045B00068857F3882FB0032C317C3EB620303EBCD
:1045C0004303A0EB83007330C0B298F8001005F0ED
:1045D000FBF9BBF80030032B7FF613A93868BAF853
:1045E0000030574AC31A82FB031ED917C1EB6E0174
:1045F00001EB4101A3EB810303EB430304EB8304D1
:10460000A36818447F287FF7EDAE7F3882FB003225
:10461000C317C3EB620303EB4303A0EB83007330C8
:104620006EE5DFF828A14649BAF80020454C9A1AF1
:1046300081FB020ED017C0EB6E0000EB4000A2EB36
:10464000800202EB420254F8220018447F2840F313
:104650000383A0F17F0381FB0321DA17C2EB610022
:1046600000EB4000A3EB80007330DFF8E4B098F873
:104670000010C0B205F0A8F9BBF80030022B7FF69D
:104680004BAE3968BAF800302D4ACB1A82FB030EC4
:10469000D817C0EB6E0000EB4000A3EB800303EBE8
:1046A000430304EB8303586808447F2840F3F684EF
:1046B0007F3882FB0032C317C3EB620303EB430373
:1046C000A0EB83007330C0B298F8001005F07CF9BD
:1046D000BBF80030032B7FF61FAE3868BAF8003005
:1046E000174AC31A82FB031ED917C1EB6E0101EBF7
:1046F0004101A3EB810303EB430304EB8304A368B1
:1047000018447F287FF760AE7F3882FB0032C317E2
:10471000C3EB620303EB4303A0EB83007330F6E5C6
:1047200001283EF41CAB0123FFF78ABB109DFF1F3D
:10473000C09EFF1FD09CFF1F969FFF1F649DFF1F01
:10474000ABAAAA2A9C3D01007C9FFF1FF09EFF1F81
:10475000F49CFF1F759DFF1F4FF47A43013BFDD171
:1047600099F8000005F054F9FFF75BB8DFF8E8A20C
:1047700099F80000BAF80030B54AB64CC31A82FB6B
:10478000031ED917C1EB6E0101EB4101A3EB8103BD
:1047900003EB430354F8233018447F2840F3DD81B2
:1047A0007F3882FB0032C317C3EB620202EB420286
:1047B000A0EB82007330DFF8A4B2C0B205F028F994
:1047C000BBF80030022B7EF6C5AE99F80000BAF8AF
:1047D00000309F4AC31A82FB0321DA17C2EB610241
:1047E00002EB4202A3EB820303EB430304EB8303DC
:1047F0005B6818447F2840F312847F380C2290FBBA
:10480000F2F302FB13007330C0B205F001F9BBF8FC
:104810000030032B7EF69EAE99F80000BAF8003007
:104820008B4AC31A82FB0321DA17C2EB610202EB47
:104830004202A3EB820303EB430304EB8304A3686C
:1048400018447F287FF79CAD7F380C2290FBF2F351
:1048500002FB13007330D7E4DFF8FCA13868BAF824
:1048600000307B4A7B4CC31A82FB031ED917C1EB75
:104870006E0101EB4101A3EB810303EB430354F809
:10488000233018447F2840F365817F3882FB003253
:10489000C317C3EB620202EB4202A0EB820073304B
:1048A000DFF8BC81DFF8B4B198F80010C0B205F0B1
:1048B0008BF8BBF80030022B7EF6A3AF3868BAF84D
:1048C0000030634AC31A82FB0321DA17C2EB61028C
:1048D00002EB4202A3EB820303EB430304EB8303EB
:1048E0005B6818447F2840F3A7837F380C2290FB35
:1048F000F2F302FB13007330C0B298F8001005F019
:1049000063F8BBF80030032B7EF67BAF3868BAF84B
:1049100000304F4AC31A82FB0321DA17C2EB61024F
:1049200002EB4202A3EB820303EB430304EB830499
:10493000A36818447F287FF755AD7F380C2290FB81
:10494000F2F302FB13007330FFF7DABBFBF79AFEBA
:1049500002E4DFF804A13E49BAF800203D4C9A1A5F
:1049600081FB020ED017C0EB6E0000EB4000A2EB03
:10497000800202EB420254F8220018447F2840F3E0
:10498000EF80A0F17F0381FB0321DA17C2EB610105
:1049900001EB4101A3EB81007330DFF8C0B098F860
:1049A0000010C0B205F010F8BBF80030022B7FF603
:1049B000B3AC3868BAF80030254AC31A82FB032129
:1049C000DA17C2EB610202EB4202A3EB820303EBB4
:1049D000430304EB83035B6818447F2840F32F8371
:1049E0007F380C2290FBF2F302FB13007330C0B24D
:1049F00098F8001004F0E8FFBBF80030032B7FF6B6
:104A00008BAC3868BAF80030114AC31A82FB032114
:104A1000DA17C2EB610202EB4202A3EB820303EB63
:104A2000430304EB8304A36818447F287FF7CCACCE
:104A30007F380C2290FBF2F302FB1300733066E424
:104A4000FBF720FEFFF700BBFBF71CFE08E400BFEE
:104A5000ABAAAA2A2C3E0100F09EFF1FF49CFF1F68
:104A6000759DFF1FDFF834A399F80000BAF80030F5
:104A7000C24AC34CC31A82FB0317D917C1EB6701A3
:104A800001EB4101A3EB810303EB430354F8233013
:104A900018447F286ADD7F3882FB0032C317C3EBDE
:104AA000620202EB4202A0EB82007330DFF8F0B248
:104AB000C0B204F0ADFFBBF80030022B7FF679A93D
:104AC00099F80000BAF80030AC4AC31A82FB0321FF
:104AD000DA17C2EB610202EB4202A3EB820303EBA3
:104AE000430304EB83035B6818447F2840F3AA82E6
:104AF0007F380C2290FBF2F302FB13007330C0B23C
:104B000004F086FFBBF80030032B7FF652A999F81A
:104B10000000BAF80030994AC31A82FB0321DA1761
:104B2000C2EB610202EB4202A3EB820303EB4303FD
:104B300004EB8304A36818447F2814DD7F380C221B
:104B400090FBF2F302FB13007330C0B204F060FF7D
:104B5000FFF72FB9FBF796FDA2E6FBF793FD2AE6D8
:104B6000FBF790FD19E7FBF78DFDEEE7FBF78AFDFC
:104B70009CE7DFF828A299F80000BAF800307F4AD5
:104B8000804CC31A82FB031ED917C1EB6E0101EBE7
:104B90004101A3EB810303EB430354F82330184492
:104BA0007F28DADD7F3882FB0032C317C3EB620354
:104BB00003EB4303A0EB83007330FCE5DFF8DCA1DB
:104BC0003868BAF800306D4A6E4CC31A82FB031E77
:104BD000D917C1EB6E0101EB4101A3EB810303EB9C
:104BE000430354F8233018447F28B3DD7F3882FB19
:104BF0000032C317C3EB620303EB4303A0EB830054
:104C000073304DE6FBF73EFDAEE4DFF890A15B4963
:104C1000BAF800205B4C9A1A81FB020ED017C0EB49
:104C20006E0000EB4000A2EB800202EB420254F85F
:104C3000220018447F2893DDA0F17F0381FB03212C
:104C4000DA17C2EB610000EB4000A3EB8000733089
:104C5000A3E6FBF717FD0AE4FBF714FD05E5DFF813
:104C60003CA199F80000BAF80030444A464CC31AF7
:104C700082FB0317D917C1EB670101EB4101A3EBDD
:104C8000810303EB430354F8233018447F287FF754
:104C90006DAF7F3882FB0032C317C3EB620303EBB7
:104CA0004303A0EB8300733000E738480090384896
:104CB00038490390FEF7C9B8DFF8E0A099F8000082
:104CC000BAF800302D4A344CC31A82FB0321DA179C
:104CD000C2EB610202EB4202A3EB820303EB43034C
:104CE00054F8233018447F2840F3A0817F380C22E9
:104CF00090FBF2F302FB13007330DFF8A4B0C0B2F4
:104D000004F086FEBBF80030022B19D999F8000098
:104D1000BAF800300C22C11A91FBF2F302FB131314
:104D200002FB03435B6818447F2840F352847F38BA
:104D300090FBF2F302FB13007330C0B204F068FE84
:104D4000BBF80030032B7EF605ACBAF8003099F8BA
:104D500000000C22C11A91FBF2F302FB131302FBB9
:104D60000344A36818447F287FF70AAB7F3890FB81
:104D7000F2F302FB13007330FFF746BAABAAAA2A7C
:104D8000C83A0100343701009C3D0100489FFF1FD5
:104D9000B59CFF1FF49EFF1F643C0100F09EFF1FA7
:104DA000F49CFF1FDFF864A33868BAF80030CE4ADD
:104DB000CE4CC31A82FB0321DA17C2EB610202EB6D
:104DC0004202A3EB820303EB430354F8233018445D
:104DD0007F2840F328817F380C2290FBF2F302FBFE
:104DE00013007330DFF82883DFF828B398F8001039
:104DF000C0B204F0E9FDBBF80030022B1AD93868C4
:104E0000BAF800300C22C11A91FBF2F302FB131323
:104E100002FB03435B6818447F2840F3D4837F3848
:104E200090FBF2F302FB13007330C0B298F800104D
:104E300004F0CAFDBBF80030032B7EF6E2ACBAF8F2
:104E4000003038680C22C11A91FBF2F302FB1313F5
:104E500002FB0344A36818447F287FF7C3AA7F3866
:104E600090FBF2F302FB13007330FFF749B9FBF735
:104E700009FCFFF719B9FBF705FCFFF79AB9012BFD
:104E80003DF495AF0124FFF762BADFF880A296499E
:104E9000BAF80020954C9A1A81FB0210D117C1EB89
:104EA000600101EB4101A2EB810202EB420254F8E6
:104EB000220018447F2840F3BC80A0F17F030C201F
:104EC00093FBF0F200FB12307330DFF848B298F831
:104ED0000010C0B204F078FDBBF80030022B1AD9E4
:104EE0003868BAF800300C22C11A91FBF2F302FBC9
:104EF000131302FB03435B6818447F2840F3668367
:104F00007F3890FBF2F302FB13007330C0B298F8C5
:104F1000001004F059FDBBF80030032B7FF6FCA90C
:104F2000BAF8003038680C22C11A91FBF2F302FB88
:104F3000131302FB0344A36818447F287FF744AA95
:104F40007F3890FBF2F302FB13007330FFF7DFB9F9
:104F5000DFF8B8A199F80000BAF80030624A644C52
:104F6000C31A82FB0321DA17C2EB610202EB420291
:104F7000A3EB820303EB430354F8233018447F2848
:104F800046DD7F380C2290FBF2F302FB13007330F6
:104F9000DFF880B1C0B204F03BFDBBF80030022B5B
:104FA00019D999F80000BAF800300C22C11A91FB07
:104FB000F2F302FB131302FB03435B6818447F28E0
:104FC00040F38F807F3890FBF2F302FB13007330C5
:104FD000C0B204F01DFDBBF80030032B7EF6E9AE35
:104FE000BAF8003099F800000C22C11A91FBF2F3D4
:104FF00002FB131302FB0344A36818447F287FF7C6
:10500000B2AD7F3890FBF2F302FB130073309CE5E6
:10501000FBF738FBBCE7FBF735FBFFF74EB9FBF7B7
:1050200031FBFFF7F1BBFBF72DFBDBE6FBF72AFBC0
:1050300063E6FBF727FB48E7FBF724FB5CE4FBF7A1
:1050400021FBD4E4FBF71EFB59E5DFF8C0A099F87B
:105050000000BAF80030244A264C35E6DFF8ACA050
:105060003868BAF80030204A224CA2E6FBF70AFB67
:10507000FFF72ABA029B1B78002B7EF44BAAFEF79F
:105080006EBAFBF7FFFAFFF79FBADFF880A099F836
:105090000000BAF80030144A174C61E7FBF7F2FA47
:1050A000FFF711BBDFF864A00F49BAF80020114CDC
:1050B000F1E6124B1B78002B00F0CB82104B1B78D3
:1050C000002B7DF474AE0F4B1B78002B3DF46FAEBC
:1050D000B8F800300C490A33A8F800300A70FDF720
:1050E00066BEFBF7CFFA73E7ABAAAA2A643C0100BD
:1050F0002C3E0100203F010034370100939FFF1F29
:10510000949FFF1F959FFF1FDC9CFF1FF09EFF1FBA
:10511000759DFF1FF49CFF1FA44C2288002A00F0FD
:105120002383A349DFF89CB20988BBF80000033150
:10513000884227DD9F48A0490088B1F800E0DFF8E9
:105140007CC2181A0C2190FBF1F901FB19004FF0F9
:10515000900909FB0EFE01FB00E06FF00B0E5CF8FE
:10516000000003440EFB02307F2840F328857F387F
:1051700090FBF1F301FB13007330C0B298F80010FC
:1051800004F022FCBBF8002023881344022B23DD0B
:10519000884B894A38681B88B2F800C0DFF81CE2E7
:1051A000C31A0C2193FBF1F201FB1232902303FB93
:1051B0000CF301FB023373445B6818447F2840F30F
:1051C000A3857F3890FBF1F301FB13007330C0B26D
:1051D00098F8001004F0F8FBBBF800202388134473
:1051E000032B23DD734B744A38681B88B2F800C068
:1051F000DFF8C8E1C31A0C2193FBF1F201FB123274
:10520000902303FB0CF301FB023373449B681844A7
:105210007F2840F326857F3890FBF1F301FB1300D4
:105220007330C0B298F8001004F0CEFBBBF8002039
:1052300023881344042B7FF76FA85D4B1B88012B39
:105240007FF46AA83A68A2F10C007F287FF7BCA817
:105250008B3A0C2092FBF0F300FB13207330FFF726
:1052600056B8524C2388002B40F0A282DFF854B18C
:105270005049514A0988D7F80080B2F800E04F48F9
:10528000C1EB080C0C229CFBF2F102FB11C14FF0A8
:10529000900C0CFB0EFE02FB01E16FF00B0E405870
:1052A00080440EFB03807F2840F38584A0F17F03B8
:1052B00093FBF2F002FB10307330414BC0B219780F
:1052C00004F082FBBBF8002023881344022B23DD6B
:1052D000384A394B11883868B3F800C0DFF8DCE091
:1052E000411A0C2291FBF2F302FB1311902303FBF2
:1052F0000CF302FB013373445B6818447F2840F3CE
:10530000A3847F3890FBF2F302FB130073302C4B25
:10531000C0B2197804F058FBBBF80020238813446E
:10532000032B23DD234A244B11883868B3F800C0CF
:10533000DFF888E0411A0C2291FBF2F302FB131113
:10534000902303FB0CF302FB013373449B68184466
:105350007F2840F36C847F3890FBF2F302FB13004C
:105360007330174BC0B2197804F02EFBBBF8002045
:1053700023881344042B7EF744AA0D4B1B88012B72
:105380007EF43FAA3A68A2F10C007F2840F35681D0
:105390008B3A0C2092FBF0F300FB13207330084B88
:1053A000C0B2197804F010FBFEF72BBA7C9DFF1FEA
:1053B0000E9DFF1FF09EFF1FA29EFF1FC43701001E
:1053C000759DFF1FF49CFF1FCF4C2388002B40F0DE
:1053D000FA81DFF868B3CD49CD4A098899F8000011
:1053E000B2F800E0DFF85883C1EB000C0C229CFB04
:1053F000F2F102FB11C14FF0900C0CFB0EFE02FB10
:1054000001E16FF00B0E58F8011008440EFB030089
:105410007F2840F3AC83A0F17F0393FBF2F002FB03
:1054200010307330C0B204F0F3FABBF800202388C8
:105430001344022B22DDB54AB54B118899F80000C0
:10544000B3F800C0DFF8F8E2411A0C2291FBF2F346
:1054500002FB1311902303FB0CF302FB0133734493
:105460005B6818447F2840F3F3837F3890FBF2F3A6
:1054700002FB13007330C0B204F0CAFABBF800207C
:1054800023881344032B22DDA04AA14B118899F8ED
:105490000000B3F800C0DFF8A8E2411A0C2291FB2B
:1054A000F2F302FB1311902303FB0CF302FB013315
:1054B00073449B6818447F2840F3BD837F3890FB7A
:1054C000F2F302FB13007330C0B204F0A1FABBF890
:1054D000002023881344042B7EF73CA88D4B1B88A7
:1054E000012B7EF437A899F80020A2F10C007F2848
:1054F0007EF746AF8B3A0C2092FBF0F300FB1320B3
:105500007330FEF781BEDFF804A299F80000BAF804
:105510000030814CC11A0C2291FBF2F302FB1313F1
:1055200002FB03F3E35818447F287FF771AD7F38FF
:1055300090FBF2F302FB1300733029E5774B1A88D6
:10554000182A13D03B681344A3F118007F2840F3B6
:1055500085830C20973B93FBF0F200FB123303F1A1
:1055600073006F4BC0B2197804F02EFA6D4B6E4980
:105570001A78022A94BF013200221A701A7831F880
:105580001200182810D10424022A02F10100C2B22C
:1055900088BF002231F81200182804D1013CF3D151
:1055A0001A70FEF72EB91A703B680344A3F1180075
:1055B0007F2843DD0C20973B93FBF0F200FB123376
:1055C00003F17300EBE6FBF75DF82EE4FBF75AF806
:1055D0009CE4FBF757F8FFF7B0BB504B1B88182B28
:1055E00012D099F800201344A3F118007F2840F34B
:1055F0001B830C20973B93FBF0F200FB123303F16B
:105600007300C0B204F004FA464A474B127833F8EC
:105610001230182B3DF49EAF99F800201344A3F1EB
:1056200018007F287EF7ACAE0C20973B93FBF0F27E
:1056300000FB123303F17300FEF7E6BDFBF722F81F
:10564000ADE6DFF8C8A099F80000BAF80030374C92
:1056500060E7374B1B78002B7DF4F9AF354B1B7897
:10566000002B3DF4A4ABB8F8003033490133A8F85F
:1056700000300A70FDF79BBB2D4B1B78002B7DF48F
:1056800096AB2C4B1B78002B3DF491ABB8F8003057
:105690002949013BA8F800300A70FDF788BB1F4A72
:1056A0001288182A12D01344A3F118007F2840F35F
:1056B000D2820C20973B93FBF0F200FB123303F1F4
:1056C0007300C0B298F8001004F07EF9154B16492B
:1056D0001A78022A94BF013200221A701A7831F81F
:1056E000120018282FD10424022A02F10100C2B2AC
:1056F00088BF002231F81200182823D1013CF3D1D1
:105700001A703B68FEF774B97C9DFF1FF09EFF1F67
:10571000A29EFF1F0E9DFF1F643C0100469FFF1FBE
:10572000759DFF1FD089FF1F0C9FFF1F203F0100A9
:10573000949FFF1F959FFF1FDC9CFF1FF49CFF1F82
:10574000C43701001A703B680344A3F118007F2896
:105750007EF73AAE0C20973B93FBF0F200FB12333E
:1057600003F17300FEF7D3BDDFF828B3E2E4BD4BCD
:105770001B88182B12D099F800201344A3F11800AD
:105780007F2840F35B820C20973B93FBF0F200FBF9
:10579000123303F17300C0B204F03AF9B24AB34BCA
:1057A000127833F81230182B7FF436AFFDF7D2BEE3
:1057B000AF4ADFF8E0B21288BBF800100332914222
:1057C0007FF780AD54E5AA4ADFF8C8B21288BBF86B
:1057D0000010033291427FF728AEFCE5A14A1288FF
:1057E000182A12D01344A3F118007F2840F37B82BB
:1057F0000C20973B93FBF0F200FB123303F1730094
:10580000C0B298F8001004F0DFF8974B97491A7867
:10581000022A94BF013200221A701A7831F812005D
:10582000182890D10424022A02F1010294BFD2B2B6
:10583000002231F81200182884D1013CF3D15FE72F
:10584000884B1A88182A13D03B681344A3F1180018
:105850007F2840F3F6810C20973B93FBF0F200FB8E
:10586000123303F17300834BC0B2197804F0ACF823
:105870007D4B7E491A78022A94BF013200221A70A9
:105880001A7831F8120018287FF48EAE0424022A08
:1058900002F1010294BFD2B2002231F8120018289E
:1058A0007FF481AE013CF2D11A70FDF7AABF724BB2
:1058B00000227F2107201A8004F056F87F210B2058
:1058C00004F052F8FDF7F6BE6C4C2388002B40F034
:1058D0001082DFF8C0B16A4999F80000694A098866
:1058E0001788DFF8A4E1411A0C2291FBF2FC02FBBD
:1058F0001C114FF0900C0CFB07F702FB01716FF0CD
:105900000B075EF80110014407FB03107F2840F3EA
:10591000ED817F3890FBF2F302FB13007330C0B2CD
:1059200004F076F8BBF8002023881344022B21DD15
:10593000534B544A99F800001B88B2F800E0524FCC
:10594000C31A0C2193FBF1F201FB1232902303FBEB
:105950000EF301FB02333B445B6818447F2840F39D
:10596000DA817F3890FBF1F301FB13007330C0B292
:1059700004F04EF8BBF8002023881344032B21DDEC
:105980003F4B404A99F800001B88B2F800E03E4FB8
:10599000C31A0C2193FBF1F201FB1232902303FB9B
:1059A0000EF301FB02333B449B6818447F2840F30D
:1059B000AF817F3890FBF1F301FB13007330C0B26D
:1059C00004F026F8BBF8002023881344042B7EF74C
:1059D000F0A9274B1B88012B7EF4EBA999F8002036
:1059E000A2F10C007F287FF7BEA88B3A0C2092FB17
:1059F000F0F300FB13207330FFF7A7B8234B01220D
:105A00007F2107201A8003F0AFFF7F210B2003F0D6
:105A1000ABFFFDF747BE1E4B04227F2107201A80F3
:105A200003F0A2FF00210B2003F09EFFFDF733BE21
:105A3000174B02227F2107201A8003F095FF7F2158
:105A40000B2003F091FFFDF721BE114B0021072031
:105A50001C8003F089FF7F210B2003F085FFFDF7F9
:105A600010BE00BF069DFF1FD089FF1F849EFF1F31
:105A70000E9DFF1F759DFF1FD29CFF1F7C9DFF1F6A
:105A8000F09EFF1FA29EFF1FC43701008E9DFF1FC7
:105A9000E89EFF1FF49CFF1FAD4A1288182A12D0FF
:105AA0001344A3F118007F2840F347810C20973B53
:105AB00093FBF0F200FB123303F17300C0B298F8CD
:105AC000001003F081FFA34BA3491A78022A94BF68
:105AD000013200221A701A7831F8120018287FF467
:105AE00032AE0424022A02F1010294BFD2B2002293
:105AF00031F8120018287FF425AE013CF2D1FFE501
:105B0000934B1A88182A13D03B681344A3F118004A
:105B10007F2840F309810C20973B93FBF0F200FBB8
:105B2000123303F173008D4BC0B2197803F04CFFB0
:105B3000884B89491A78022A94BF013200221A70D0
:105B40001A7831F8120018287FF42EAD0424022AA6
:105B500002F1010294BFD2B2002231F812001828DB
:105B60007FF421AD013CF2D11A70FDF74ABEFAF77D
:105B700089FD57E4764B1B88182B12D099F800202A
:105B80001344A3F118007F2840F3CB800C20973BEF
:105B900093FBF0F200FB123303F17300C0B203F089
:105BA00037FF6C4A6C4B127833F81230182B7FF4A5
:105BB00033ADFDF7CFBCFAF765FDFFF77EBBFAF713
:105BC00061FDFFF7DABA664B1B88182B12D099F8E3
:105BD00000201344A3F118007F2840F39F800C207D
:105BE000973B93FBF0F200FB123303F17300C0B25A
:105BF00003F00EFF574A5B4B127833F81230182B24
:105C00003EF4D7A899F800201344A3F118007F2888
:105C10007EF7A9AF0C20973B93FBF0F200FB123309
:105C200003F17300FEF791BFFAF72CFDE9E4FAF7F0
:105C300029FDFFF796BBFAF725FD45E4FAF722FDAB
:105C4000A9E5FAF71FFD0EE6FAF71CFDFFF75FBBAB
:105C5000FAF718FD0FE4FAF715FD32E5FAF712FD31
:105C60007FE4FAF70FFDFFF7DCBA394B1B88182BDE
:105C700011D099F800201344A3F118007F2856DDB5
:105C80000C20973B93FBF0F200FB123303F17300FF
:105C9000C0B203F0BDFE2F4A2F4B127833F81230FA
:105CA000182BAFD1FEF785B82F4B1B88182B11D0BE
:105CB00099F800201344A3F118007F283ADD0C2046
:105CC000973B93FBF0F200FB123303F17300C0B279
:105CD00003F09EFE1F4A254B127833F81230182B22
:105CE00090D1FEF766B8FAF7CDFC89E5FAF7CAFC61
:105CF00015E61F4ADFF880B01288BBF800100332A7
:105D000091427FF70FAEE6E5FAF7BCFCFFF75FBA0A
:105D1000FAF7B8FC53E6FAF7B5FC28E6FAF7B2FC56
:105D200065E7FAF7AFFC39E7FAF7ACFCFBE6FAF700
:105D3000A9FCADE7FAF7A6FCC9E7FAF7A3FCBDE6B4
:105D400023601946FDF75ABC0A4B0293FDF709BFC1
:105D5000089DFF1FD089FF1F8C9EFF1F759DFF1F91
:105D6000469FFF1F0C9FFF1F069DFF1F849EFF1F66
:105D70000E9DFF1F9E9DFF1FF49CFF1F38B508F06E
:105D80000DF90E4805F00CFD0D4805F009FD0D4814
:105D900005F006FD00234FF07E5201210A48FAF774
:105DA00065FB0A4B0A4A0B49802400251C711846E2
:105DB0001D60BDE838400BF009BC00BFF09CFF1F20
:105DC000249DFF1F949DFF1FC49EFF1F549FFF1F14
:105DD0001C89FF1F2906000010B50446A420636833
:105DE000198803F043FFE368A6201988BDE8104036
:105DF00003F03CBF43682A20198803F037BF00BF77
:105E000010B5044622206368198803F02FFFE36869
:105E100024201988BDE8104003F028BF10B50446BF
:105E20000A206368198803F021FFE3680C201988B1
:105E3000BDE8104003F01ABF10B5044606206368A1
:105E4000198803F013FFE36808201988BDE81040A3
:105E500003F00CBF10B5044602206368198803F0F4
:105E600005FFE36804201988BDE8104003F0FEBE7A
:105E700070B50E4C84B0122504220123064603900F
:105E8000029320468DE824001423102107F032FBF2
:105E900006220923029303960195204600921423BB
:105EA000102107F027FB04B070BD00BFC49FFF1F87
:105EB000F8B5B04CB4F90030032B00F01281002B80
:105EC0006AD0022B00F08A80052B00F0B580012BF0
:105ED00000F0DD80042B00D0F8BDA74FA74E0025B1
:105EE0004FF4AF74E9B2A64805F084FC57F8043BC0
:105EF000C3F5967300FB03F086FB0023C017C0EBCD
:105F00006310844205F10105A8BF0446062DE9D1BE
:105F10009C4F9A4E0025E9B29B4805F06BFC57F860
:105F2000043BC3F5967300FB03F086FB0023C01708
:105F3000C0EB6310844205F10105A8BF04460C2D97
:105F4000E9D1924F8D4E0025E9B2914805F052FCFF
:105F500057F8043B894AC3F5967300FB03F086FBB0
:105F60000013C017C0EB6310844205F10105A8BF00
:105F700004460C2DE8D1A4F11401312900F3A380CB
:105F800040F26C7232218348834B01801A602A20D0
:105F9000BDE8F84003F06ABE0E2007F063FF40F64C
:105FA000FF71C8308842A8BF084620EAE07000F2BE
:105FB000DC5283B28A42794D794EA8BF0A4602204C
:105FC000194633802A8003F051FE2988042003F00B
:105FD0004DFEB4F90030022B7FF476AF012009F0BA
:105FE000DDFA0546002009F0D9FAA842B8BF2846D4
:105FF00000F1C801B1F5FA7FC0F2B480B1F57A6F53
:10600000A8BF4FF47A6101F54873B3F57A6FA8BF62
:106010004FF47A639BB289B2624A634D11800A20C1
:106020002B8003F023FE29880C2003F01FFEB4F917
:106030000030052B7FF44BAF0F2009F0AFFAC0F50D
:106040003F630433B3F5AF6FC0F28980B3F5FA6FE5
:10605000A8BF4FF4FA6399B2544BC0F54360B0F552
:10606000AF6F198061DBB0F5FA6FA8BF4FF4FA602B
:1060700083B24F4DA4202B8003F0F8FD2988A62081
:1060800003F0F4FDB4F90030012B7FF423AF1520A9
:1060900007F0E8FE00F59671B1F52F7F4DDB41F278
:1060A0005C23994263DC434A00F5617089B2B0F524
:1060B0002F7F1180B8BF4FF42F7344DB8342A8BFFA
:1060C00003469BB23FE040F23A73A4F5B97403FB78
:1060D00004F482FB0432E417A4EB621289B2323278
:1060E00051E7102009F05AFAC830B0F5FA7F1FDBEB
:1060F000B0F57A6F0146A8BF4FF47A6101F51673C7
:10610000B3F57A6FA8BF4FF47A639BB289B22A4A7B
:106110002A4D118022202B8003F0A8FD29882420FD
:1061200003F0A4FDB4F90030C9E64FF4AF63A0E773
:1061300040F24C434FF4FA71E9E740F214534FF444
:106140002F711C4A11801E4D06202B8003F08EFDFE
:106150002988082003F08AFDB4F90030BAE64FF42C
:10616000AF6179E740F214534FF4FA7154E71946DE
:10617000E7E700BFA29FFF1F608AFF1FB5814E1B8C
:10618000F09CFF1F308AFF1F249DFF1F4089FF1FC7
:10619000949DFF1F5E9FFF1F1C8AFF1F649FFF1FB0
:1061A0009C9DFF1FFC9EFF1F049DFF1FA09DFF1FC6
:1061B0001C9FFF1F429DFF1FB09EFF1FAC9EFF1F35
:1061C000309FFF1F2DE9F041224D82B0012602B21F
:1061D00084B20092284601967823192107F0D0F85E
:1061E00004F10C0212B28DE844002846A719782366
:1061F000192104F1020807F0C3F83FB20FFA88F83A
:1062000019233A46284619460196CDF8008007F032
:10621000B7F878233A4628461946CDF8008001960B
:1062200004F10A070B3407F0ABF83FB224B278232D
:106230003A46284619468DE8500007F0A1F8192380
:1062400000943A4601962846194607F099F802B09C
:10625000BDE8F081C49FFF1F30B583B000230C461A
:1062600005B2009326225B231C210C4806F0D8FDC2
:10627000294601232622094806F0EEF8002C24B214
:1062800005DB214601232622044806F0E5F8044AEE
:10629000044B15801C8003B030BD00BFC49FFF1F9E
:1062A0007A8AFF1F7C8AFF1F2DE9F041BB4C2378BF
:1062B00082B01BB1BA4B4FF6FF721A80B94BB3F9DB
:1062C0000030CBB9B84AB64B1068B3F9002080F360
:1062D0000C005B2303FB00F000131C3082424BD008
:1062E0004FF0FF31FFF7B8FFB04806F0FDFD002387
:1062F000237002B0BDE8F081012B1BD0022B5AD0D5
:10630000032B3FD0042B00F09980052BEFD10F20F9
:1063100009F044F9C0F53B600830B0F5AF6F48DBD9
:10632000B0F5FA6FA8BF4FF4FA60A0F5AF625B2337
:106330009F4835E09F4B1B78002B75D0152007F048
:1063400091FD9D4B1860B0F52F7F32DB41F25C234D
:106350009842A8BF1846A0F52F735B22974802FB0E
:1063600003F380FB0320DB17C3EBA0201C308C4B16
:10637000B3F900308342B3D1914BB3F9003001330C
:10638000AED1B4E78F4B1B68B3F5FA7F11DBB3F5E1
:106390007A6FA8BF4FF47A638B48A3F5FA725B2338
:1063A00003FB02F380FB0320DB17C3EB20201C3030
:1063B000DDE71C20DBE7854B1B68B3F5FA7F3BDB91
:1063C000B3F57A6FA8BF4FF47A63A3F5FA727E48EB
:1063D0005B2303FB02F380FB0320DB17C3EB2020CE
:1063E0001C307B4B1B68B3F5FA7F23DBB3F57A6F68
:1063F000A8BF4FF47A63A3F5FA7273495B2303FBDA
:1064000002F381FB0321DB17C3EB21211C31644B19
:10641000B3F9003083427FF465AF694BB3F90030C4
:106420008B427FF45FAF62E7112009F0B7F8624B4F
:10643000186088E71C21EAE71C20D2E72522002506
:106440008DE8240076231C215848624E624FDFF805
:10645000A08106F095FF16E0B0F5AF7FA8BF4FF41E
:10646000AF70323802FB00F088FB0031C017C0EB80
:1064700061111C3109B201231D4425224B4805F04E
:10648000EBFF0C2D14D0E9B2544805F0B3F956F8DF
:10649000043BC3F5967300FB03F087FB0013C017A2
:1064A000C0EB631031284FF05B02D5DC1C21E2E722
:1064B000262200258DE8240076231C213B48484EE7
:1064C000454FDFF82C8106F05BFF16E0B0F5AF7F9B
:1064D000A8BF4FF4AF70323802FB00F088FB0031E8
:1064E000C017C0EB61111C3109B201231D442622E3
:1064F0002E4805F0B1FF0C2D14D0E9B2394805F053
:1065000079F956F8043BC3F5967300FB03F087FB5B
:106510000013C017C0EB631031284FF05B02D5DCCD
:106520001C21E2E7272200258DE8240076231C2188
:106530001E482D4E284FDFF8B88006F021FF17E0E7
:10654000B0F5AF7FA8BF4FF4AF70323802FB00F058
:1065500088FB0031C017C0EB61111C3109B2012367
:106560001D442722114805F077FF062D3FF4BCAEED
:10657000E9B21E4805F03EF956F8043BC3F59673A0
:1065800000FB03F087FB0013C017C0EB631031283A
:106590004FF05B02D4DC1C21E1E700BF9C9FFF1F92
:1065A0007A8AFF1FA29FFF1F009FFF1FC49FFF1F2C
:1065B00037800B6DB89EFF1FC09CFF1FD305854120
:1065C0007C8AFF1F149DFF1F011FB812209DFF1F13
:1065D000E49CFF1F308AFF1FB5814E1B249DFF1FC7
:1065E0004089FF1F949DFF1F608AFF1FF09CFF1FC3
:1065F0004B48371B2DE9F043754C054683B02046C8
:10660000D5F80080EE6806F063FB1120FFF7DAFD95
:10661000012719234FF02809194620460197242203
:10662000CDF8009006F0ACFE78231946242201979D
:106630002046CDF8009006F0A3FE3946204607F02C
:1066400029FA0223192240462382E2810CF078FDC8
:106650004146024620460AF04BFC20460AF05EFC0A
:106660000027142303225B4923822046E7810AF096
:106670003FFC20460AF052FC2323204603225649C1
:10668000E78123820AF034FC20460AF047FC6EB111
:106690002F20FFF797FD322303225049E781204640
:1066A00023820AF025FC20460AF038FC01234C4ADC
:1066B00018461370FFF7DCFB29896A896B68521A48
:1066C0001B885C2AA3EB010357DD03EB4303013274
:1066D000C3EB431393FBF2F303F11B023C4FDFF8D0
:1066E0000CE113B21A214FF001088DE8020138467F
:1066F000AEF800201946142206F042FE002E4ED0BD
:10670000298A6B8AEA685B1A5C2B12883DDC511A75
:106710005C2202FB01F292FBF3F31B33314A2C485B
:10672000138001261BB2382219468DE8440032221C
:1067300006F026FE0022402309218DE806002448A9
:10674000194606F0EBFD3146214807F0A3F96B68C6
:106750001F48022244212282E18119880AF02EFC7E
:10676000324621491A480AF0C3FBEB6818481988D9
:1067700003B0BDE8F0430AF021BC5C2101FB03F348
:1067800093FBF2F303F11B02A8E7521A02EB420259
:10679000C2EB4212434492FBF3F31B33BEE74023A8
:1067A00009213246009138461946019606F0B6FD99
:1067B0004146384607F06EF96B6868210222F9817C
:1067C0003A821988384603B0BDE8F0430AF0F6BBB8
:1067D000C49FFF1F884001008C40010090400100D1
:1067E00045A0FF1FA09FFF1F944001009E9FFF1F19
:1067F0002DE9F04F1F4685B01446002A4ED0052AD9
:106800000646D0F80C8000F0AB800F9B8C4A00EB62
:10681000C305012CB5F80AE029896868C1EB0E03AD
:1068200082FB03C21A444FEAE373C3EBA21302884C
:1068300051D0042C00F08D80824D0022092140238C
:1068400028468DE80600194606F068FD2846012115
:1068500007F020F9B8F1000F00F0E8807368022219
:1068600044212A82E981198828460AF0A7FB764943
:10687000012228460AF03CFBF368284619880AF0F2
:106880009DFB724B022CB3F9001000F0AD80082C78
:1068900000F0C980012005B0BDE8F08F6C4E6D4A54
:1068A00033681268CB1A93420D4655D96A4A3B8821
:1068B00011786448012918BF012414700E9A063219
:1068C0001BB212B28DE814001946BDF9382006F04B
:1068D00057FD3560DEE79BB2D31A994203DC9E4533
:1068E0007146A8BF19460E9A0180B7F90030BDF96C
:1068F00038A0544802F106094FF0000E0FFA89F94A
:1069000019465246CDF80090CDF804E006F038FD67
:1069100029896A896868521A03885C2AA3EB0103F3
:106920007ADD03EB43030132C3EB431393FBF2F332
:1069300003F11B0213B201203A801946524601901E
:10694000CDF800903F4806F01BFD434B00221A7023
:1069500072E712FA83F3C0E7204605B0BDE8F08F76
:10696000384D4FF0070A4FF0000B28465A232322D8
:106970008DE8000C1A2106F0D1FC2846012107F011
:1069800089F84FF001094FF0350E2323A5F80EE0EA
:1069900052462B823149A5F814902846A5F812904A
:1069A00003930AF0A5FA28460AF0B8FA284606F03A
:1069B0009BFA4FF4FA6007F0DFFEFFF779FA039BCA
:1069C0001A211A4628465A238DE8000C06F0A6FC28
:1069D000284606F089FA3046FFF70CFE204B83F874
:1069E0000090FFF761FC27E74A1C12B21A8091421F
:1069F0003FF450AF0E9AB7F9003012480632012426
:106A000012B2009219460194BDF9382006F0B8FC84
:106A1000204605B0BDE8F08F5C2101FB03F393FB3A
:106A2000F2F21B3286E700221A80E0E773686821E1
:106A30000222E9812A82198828460AF0BFFA20E753
:106A4000C94216B2C49FFF1F94400100A69FFF1FBA
:106A500030A0FF1F4450010045A0FF1F98400100D7
:106A60009C9FFF1F2DE9F04F5A4E5B4DB6F9007009
:106A70004C7855F8277085B08146984604B10C785B
:106A8000DFF874A11AB99AF80030002B39D0534DB1
:106A9000002338462B808AF80030FFF7ABFD504AC0
:106AA000504BB5F90000012111704FF6FF721A80AA
:106AB00060B301285ED0012032232246019000936A
:106AC0004946494B3846FFF793FE00240346B5F983
:106AD0000020022A39DD00222A80B6F900203D4933
:106AE000002A3BDB052AC4BF00220A80B8F1000F50
:106AF00039D1002C0CBF18464FF0FF3005B0BDE86F
:106B0000F08F364DB5F900000028D2D1DFF8ECB097
:106B1000364ADBF800301268C3EB0903934227D9E9
:106B2000334B1A78012A18BF01201870FFF7A0F91B
:106B30000123CBF80090012C2AD0042C35D0022C54
:106B40003AD0082C3ED00024C1E7C6D1FA68002A0A
:106B5000C1D0B6F900201F49002AC3DA05220A80F5
:106B6000B8F1000FC5D00393FFF79EFB039BC0E76E
:106B70000346E0E74FF0000E142322468DE808405C
:106B800049461C4B38467446FFF732FE03469EE7E3
:106B900032888AF80040013232807A6982B100245A
:106BA000384603939047039B91E732880121013ACD
:106BB00032808AF80010F0E701222A8000248CE756
:106BC000144684E77A69002129804FF0FF34002AB7
:106BD000E6D182E7A29FFF1F808AFF1FA69FFF1FAB
:106BE0009C9FFF1F7A8AFF1FA09FFF1F4450010038
:106BF00045A0FF1F9E9FFF1FA49FFF1F30A0FF1FE8
:106C000001210D2007F07CBD00210D2007F078BD8B
:106C100001460D2007F074BD08B50D2007F076FD84
:106C2000B0FA80F149090D20BDE8084007F068BDC1
:106C300010B5002144080D2007F062FD204607F042
:106C40009BFD0D20012107F05BFD2046BDE81040B3
:106C500007F092BD2D4A2E4B10881B68984210B544
:106C600049DA2C4A1288141A9A42A8BF1A46B4F577
:106C7000157F36DA121A40F2532303FB02F393FB1B
:106C8000F4F105310A2007F0ABFB234B1978C9B3A7
:106C9000224B23491B6840F2271283F3070302FBB0
:106CA00003F381FB03211944DB17C3EBA111053169
:106CB000092007F095FB1B4B1968F1B181F307011F
:106CC00040F22712164802FB01F380FB032119440E
:106CD000DB17C3EBA11105311620BDE8104007F00A
:106CE0007FBB131A4FF41572611C02FB03F393FB75
:106CF000F1F10531C6E70021C4E71620BDE81040D8
:106D000007F06EBB092007F06BFBD4E79C9DFF1FCB
:106D1000B89CFF1F649FFF1F469DFF1F4C9FFF1FD6
:106D200009040281189FFF1F7F2838B5A8BF7F2064
:106D30000F4C4FF4167202FB00F284FB0231114437
:106D4000D2170546C2EBA1110A2007F049FB7F3D8F
:106D50004FF4967303FB05F384FB03211944DB17FF
:106D6000A3EBA1110920BDE8384007F039BB00BFF3
:106D700009040281C368B3F9003030B583EAE374D3
:106D8000A4EBE374002BA0B218DB012300E0134650
:106D900003EB830252009442F9DA0A4D90FBF3F2BE
:106DA00085FB03E403FB1200DB173032D3EBA403B3
:106DB00080B201F8012BF1D10B7030BD2D230B7087
:106DC0000131E2E76766666638B5094D82242046E0
:106DD00002F066FF35F8021B00B28842204601D05F
:106DE00002F044FF0234A4B28A2CF0D138BD00BFB7
:106DF0008C9EFF1F024B8020198802F037BF00BF16
:106E0000089DFF1F38B5094D7824204602F048FF41
:106E100035F8021B00B28842204601D002F026FF5E
:106E20000234A4B2802CF0D138BD00BF849EFF1F75
:106E3000024B7620198802F019BF00BF069DFF1F84
:106E400038B5094D4624204602F02AFF35F8021BCA
:106E500000B28842204601D002F008FF0234A4B2FA
:106E60004E2CF0D138BD00BF0C9FFF1F024B4420B9
:106E7000198802F0FBBE00BF469FFF1F024B4E2049
:106E8000198802F0F3BE00BF1A9DFF1F024B9A2023
:106E9000198802F0EBBE00BF7C9DFF1F024B9820BB
:106EA000198802F0E3BE00BF0E9DFF1F024B8C202D
:106EB000198802F0DBBE00BFA29EFF1F024B9C2080
:106EC000198802F0D3BE00BFF49CFF1F024BA02024
:106ED000198802F0CBBE00BF149FFF1F024B962003
:106EE000198802F0C3BE00BFF09EFF1F024B8A202C
:106EF000198802F0BBBE00BFB69EFF1F024B1020D8
:106F0000198802F0B3BE00BFB49EFF1F024B2C20B5
:106F1000198802F0ABBE00BFEE9CFF1F024B1E2083
:106F2000198802F0A3BE00BF0C9DFF1FC3680E208E
:106F3000198802F09BBE00BF024B2820198802F07E
:106F400095BE00BF0A9FFF1F024B6420198802F004
:106F50008DBE00BF049FFF1F024B5A20198802F00C
:106F600085BE00BFC89CFF1F024B1620198802F087
:106F70007DBE00BFD29CFF1F024B2E20198802F05D
:106F800075BE00BF849DFF1F024B3020198802F0A0
:106F90006DBE00BF709FFF1F024B9E20198802F03C
:106FA00065BE00BFD889FF1F024BAC20198802F0D4
:106FB0005DBE00BF069FFF1F024BAE20198802F086
:106FC00055BE00BF189DFF1F024BB020198802F06C
:106FD0004DBE00BF989EFF1F024BB220198802F0E1
:106FE00045BE00BF3A9DFF1F024B1820198802F0D2
:106FF0003DBE00BFA29DFF1F024BA220198802F0D8
:1070000035BE00BF3A9FFF1F024B1A20198802F0BD
:107010002DBE00BF289DFF1F024B1C20198802F0C7
:1070200025BE00BF1C9DFF1F024B6620198802F081
:107030001DBE00BF449FFF1F024B7220198802F043
:1070400015BE00BF6C9FFF1F024B2020198802F065
:107050000DBE00BF429FFF1F024B3220198802F075
:1070600005BE00BF329FFF1F024B6820198802F047
:10707000FDBD00BF649DFF1F024B6C20198802F00C
:10708000F5BD00BFBC9CFF1F024B6E20198802F0AB
:10709000EDBD00BF9A9FFF1F024B5220198802F0DE
:1070A000E5BD00BF7289FF1F024B5020198802F016
:1070B000DDBD00BF3689FF1F024B5420198802F046
:1070C000D5BD00BF2C8AFF1F024B5C20198802F03F
:1070D000CDBD00BF788AFF1F024B5E20198802F0E9
:1070E000C5BD00BF7089FF1F024B5620198802F0F2
:1070F000BDBD00BF729DFF1F244B1B880B2B43D8C7
:10710000DFE803F00B10151A1F24292E33383D0633
:10711000084604221E490CF0D1B8084604221D4935
:107120000CF0CCB8084604221B490CF0C7B808463E
:1071300004221A490CF0C2B80846042218490CF07F
:10714000BDB80846042217490CF0B8B80846042216
:1071500015490CF0B3B80846042214490CF0AEB837
:107160000846042212490CF0A9B808460422114925
:107170000CF0A4B8084604220F490CF09FB808464A
:1071800004220E490CF09AB8704700BFF09EFF1F12
:10719000F84C01004C4A0100B4480100E8490100E4
:1071A000B8480100044E0100BC480100C04801007D
:1071B000904B0100C4480100044D0100C848010083
:1071C000064B074A10B41C88064B0846002C14BF17
:1071D00011461946042210BC0CF070B8409DFF1FE8
:1071E000CC480100D0480100064B074A10B41C8867
:1071F000064B0846002C14BF11461946042210BC49
:107200000CF05CB8869DFF1FCC480100D0480100FF
:10721000064B074A10B41C88064B0846002C14BFC6
:1072200011461946042210BC0CF048B8AA9EFF1F54
:10723000CC480100D0480100064B074A10B41C8816
:10724000064B0846002C14BF11461946042210BCF8
:107250000CF034B8F29EFF1FCC480100D04801006A
:10726000064B074A10B41C88064B0846002C14BF76
:1072700011461946042210BC0CF020B88E9DFF1F49
:10728000CC480100D04801001B4B1B880A2B0AD8B0
:10729000DFE803F00A0E12161A1E22262A2E060016
:1072A000164B186808607047154B186808607047DF
:1072B000144B186808607047134B186808607047D3
:1072C000124B186808607047114B186808607047C7
:1072D000104B1868086070470F4B186808607047BB
:1072E0000E4B1868086070470D4B186808607047AF
:1072F0000C4B186808607047B69EFF1FF8480100E5
:10730000D0480100D4480100D8480100DC48010001
:10731000E0480100E4480100E8480100EC480100B1
:10732000F0480100F4480100F0B52B4E2B4FDFF878
:10733000C4E005460FCE87B06C460FC496E8030044
:107340003B68274A274F44F8040B40F6CC30834271
:10735000C8BF3A46BEF800602180012E118892789D
:10736000ADF80D108DF80F202AD032D340F6CA02A6
:10737000022E18BF00229A4226DAA3F698031A4971
:107380001A4AC3EB031381FB03011944DB17C3EB58
:107390006123243382FB0321DA17C2EBA10202EB43
:1073A0008201A3EB4103303330328DF813308DF876
:1073B00011206946284616220BF080FF07B0F0BD69
:1073C00040F698029A42D8DB094B1868CDF81100B4
:1073D000EFE740F6FC02CEE70C490100F89EFF1FE4
:1073E00000490100FC4801003B773B9867666666F0
:1073F00004490100949EFF1FF8B5174C174E2278E0
:10740000174D33782F888E46003218BF012201466F
:107410007046FFF727FB002398423370237015DB7B
:1074200014BF012000202B889F420ED040F23A72F8
:10743000A3F5AF730B490C4C02FB03F381FB031262
:10744000DB17A3EB621332332360F8BD0749012237
:1074500018460A702270E6E7288BFF1FB59FFF1FB2
:107460005E9FFF1FB5814E1B1C8AFF1F44A0FF1F9C
:10747000014B187802F06ABB2CA0FF1F014B187853
:1074800002F07EBB3C91FF1F134BB3F9003030B5C7
:1074900083EAE374A4EBE374002BA0B218DB0123AE
:1074A00000E0134603EB830252009442F9DA0B4DDD
:1074B00090FBF3F285FB03E403FB1200DB17303291
:1074C000D3EBA40380B201F8012BF1D10B7030BDD6
:1074D0002D230B700131E2E73C91FF1F6766666662
:1074E000144BB3F9003070B583EAE375A5EBE3758F
:1074F000002BACB21ADB012300E0034603EB830050
:1075000040008542F9DA0C4E94FBF3F086FB03E56C
:1075100003FB1044DB173030D3EBA503A4B201F812
:10752000010BF1D105480B70106070BD2D230B705D
:107530000131E0E7C89CFF1F6766666624490100C9
:10754000134BB3F9003030B583EAE374A4EBE37472
:10755000002BA0B218DB012300E0134603EB8302EB
:1075600052009442F9DA0B4D90FBF3F285FB03E4F1
:1075700003FB1200DB173032D3EBA40380B201F817
:10758000012BF1D10B7030BD2D230B700131E2E7DF
:10759000D889FF1F67666666134BB3F9003030B5B4
:1075A00083EAE374A4EBE374002BA0B218DB01239D
:1075B00000E0134603EB830252009442F9DA0B4DCC
:1075C00090FBF3F285FB03E403FB1200DB17303280
:1075D000D3EBA40380B201F8012BF1D10B7030BDC5
:1075E0002D230B700131E2E7189DFF1F6766666669
:1075F000134BB3F9003030B583EAE374A4EBE374C2
:10760000002BA0B218DB012300E0134603EB83023A
:1076100052009442F9DA0B4D90FBF3F285FB03E440
:1076200003FB1200DB173032D3EBA40380B201F866
:10763000012BF1D10B7030BD2D230B700131E2E72E
:107640003A9DFF1F67666666134BB3F9003030B58D
:1076500083EAE374A4EBE374002BA0B218DB0123EC
:1076600000E0134603EB830252009442F9DA0B4D1B
:1076700090FBF3F285FB03E403FB1200DB173032CF
:10768000D3EBA40380B201F8012BF1D10B7030BD14
:107690002D230B700131E2E73A9FFF1F6766666694
:1076A000134BB3F9003030B583EAE374A4EBE37411
:1076B000002BA0B218DB012300E0134603EB83028A
:1076C00052009442F9DA0B4D90FBF3F285FB03E490
:1076D00003FB1200DB173032D3EBA40380B201F8B6
:1076E000012BF1D10B7030BD2D230B700131E2E77E
:1076F0007289FF1F67666666134BB3F9003030B5B9
:1077000083EAE374A4EBE374002BA0B218DB01233B
:1077100000E0134603EB830252009442F9DA0B4D6A
:1077200090FBF3F285FB03E403FB1200DB1730321E
:10773000D3EBA40380B201F8012BF1D10B7030BD63
:107740002D230B700131E2E73689FF1F67666666FD
:10775000134BB3F9003030B583EAE374A4EBE37460
:10776000002BA0B218DB012300E0134603EB8302D9
:1077700052009442F9DA0B4D90FBF3F285FB03E4DF
:1077800003FB1200DB173032D3EBA40380B201F805
:10779000012BF1D10B7030BD2D230B700131E2E7CD
:1077A0002C8AFF1F67666666134BB3F9003030B54D
:1077B00083EAE374A4EBE374002BA0B218DB01238B
:1077C00000E0134603EB830252009442F9DA0B4DBA
:1077D00090FBF3F285FB03E403FB1200DB1730326E
:1077E000D3EBA40380B201F8012BF1D10B7030BDB3
:1077F0002D230B700131E2E7788AFF1F676666660A
:10780000134BB3F9003030B583EAE374A4EBE374AF
:10781000002BA0B218DB012300E0134603EB830228
:1078200052009442F9DA0B4D90FBF3F285FB03E42E
:1078300003FB1200DB173032D3EBA40380B201F854
:10784000012BF1D10B7030BD2D230B700131E2E71C
:107850007089FF1F6766666608B5702002F020FA1F
:10786000044B1988884204D07020BDE8084002F01B
:10787000FDB908BD949EFF1F08B5742002F010FAF0
:10788000044B1988884204D07420BDE8084002F0F7
:10789000EDB908BD289FFF1F054B1B880846042231
:1078A00013B904490BF00ABD03490BF007BD00BF33
:1078B0001A9DFF1F2C490100284901000E4B1B880F
:1078C000032B17D8DFE803F0110C07020846042247
:1078D0000A490BF0F3BC0846042209490BF0EEBC40
:1078E0000846042207490BF0E9BC08460422064971
:1078F0000BF0E4BC704700BFA29EFF1F3849010097
:107900003449010030490100D049010010B40A4B4C
:107910000A4C0A4693E8030083B0238802AC04E9CA
:10792000030004EB8303104653F8081C052203B040
:1079300010BC0BF0C3BC00BF18410100049FFF1F27
:1079400030B40A4B0A4D0C4693E8070084B02B88EC
:1079500004AD05E9070005EB8303204653F80C1C32
:10796000042204B030BC0BF0A9BC00BF20410100D0
:10797000949EFF1FF0B40C4D0C4F0E460FCD8CB0F3
:1079800001AC0FC40FCD0FC495E807003B8884E815
:1079900007000CAA02EB8303304653F82C1C042288
:1079A0000CB0F0BC0BF08ABC2C410100E89EFF1F1C
:1079B00030B50A4B0A4D0C460FCB85B00DF1100EB9
:1079C0000EE90F002B880EEB8303204653F8101CA2
:1079D000042205B0BDE830400BF070BC68410100E6
:1079E000069FFF1F30B50A4B0A4D0C460FCB85B0E2
:1079F0000DF1100E0EE90F002B880EEB83032046CD
:107A000053F8101C042205B0BDE830400BF056BC02
:107A100068410100989EFF1FF0B40B4D0B4F0E46BE
:107A20000FCD86B06C460FC495E803003B8884E810
:107A3000030006AA02EB8303304653F8181C042205
:107A400006B0F0BC0BF03ABC78410100A29DFF1FCC
:107A5000F0B40A4D0A4F0E460FCD86B001AC0FC4EC
:107A60002A683B88226006AA02EB8303304653F85B
:107A7000141C0C2206B0F0BC0BF020BC904101009D
:107A80001C9DFF1FF0B40B4D0B4F0E460FCD86B063
:107A90006C460FC495E803003B8884E8030006AAFF
:107AA00002EB8303304653F8181C042206B0F0BCE6
:107AB0000BF004BCA4410100289FFF1F164B1B883C
:107AC0000BB31BB283EAE370A0EBE370002B30B57D
:107AD00084B21DDB012300E0134603EB8302520056
:107AE0009042F9DA0D4894FBF3F280FB03E503FBC7
:107AF0001244DB173032D3EBA503A4B201F8012BFB
:107B0000F1D10B7030BD0846042205490BF0D6BBFD
:107B10002D230B700131DDE7649DFF1F67666666EC
:107B20003C490100F0B40A4D0A4F0E460FCD86B015
:107B300001AC0FC42A683B88226006AA02EB8303CB
:107B4000304653F8141C042206B0F0BC0BF0B6BB50
:107B5000BC410100BC9CFF1F054B1B881BB9054B9A
:107B60001868086070470846042203490BF0A6BB5A
:107B7000149FFF1FD0480100CC480100164B1B8802
:107B80000BB31BB230B583EAE374A4EBE374002BB0
:107B9000A0B21CDB012300E0134603EB830252007A
:107BA0009442F9DA0D4D90FBF3F285FB03E403FBFD
:107BB0001200DB173032D3EBA40380B201F8012BA3
:107BC000F1D10B7030BD064B1868086070472D234B
:107BD0000B700131DEE700BF0C9DFF1F6766666614
:107BE000D0480100164B1B880BB31BB230B583EA9B
:107BF000E374A4EBE374002BA0B21CDB012300E0D0
:107C0000134603EB830252009442F9DA0D4D90FBC8
:107C1000F3F285FB03E403FB1200DB173032D3EBF6
:107C2000A40380B201F8012BF1D10B7030BD064BDB
:107C30001868086070472D230B700131DEE700BF24
:107C4000F69EFF1F67666666D0480100164B1B88CC
:107C50000BB31BB230B583EAE374A4EBE374002BDF
:107C6000A0B21CDB012300E0134603EB83025200A9
:107C70009442F9DA0D4D90FBF3F285FB03E403FB2C
:107C80001200DB173032D3EBA40380B201F8012BD2
:107C9000F1D10B7030BD064B1868086070472D237A
:107CA0000B700131DEE700BFD29CFF1F676666667E
:107CB00040490100174B1B881BB31BB270B583EA08
:107CC000E375A5EBE375002BACB21EDB012300E0EE
:107CD000034603EB830040008542F9DA0E4E94FB25
:107CE000F3F086FB03E503FB1044DB173030D3EBE6
:107CF000A503A4B201F8010BF1D108480B70106084
:107D000070BD074B1868086070472D230B70013158
:107D1000DCE700BF849DFF1F67666666444901007B
:107D2000D0480100164B1B880BB31BB230B583EA59
:107D3000E374A4EBE374002BA0B21CDB012300E08E
:107D4000134603EB830252009442F9DA0D4D90FB87
:107D5000F3F285FB03E403FB1200DB173032D3EBB5
:107D6000A40380B201F8012BF1D10B7030BD064B9A
:107D70001868086070472D230B700131DEE700BFE3
:107D8000709FFF1F67666666D0480100164B1B8810
:107D90000BB31BB230B583EAE374A4EBE374002B9E
:107DA000A0B21CDB012300E0134603EB8302520068
:107DB0009442F9DA0D4D90FBF3F285FB03E403FBEB
:107DC0001200DB173032D3EBA40380B201F8012B91
:107DD000F1D10B7030BD064B1868086070472D2339
:107DE0000B700131DEE700BF449FFF1F67666666C8
:107DF000D0480100164B1B880BB31BB230B583EA89
:107E0000E374A4EBE374002BA0B21CDB012300E0BD
:107E1000134603EB830252009442F9DA0D4D90FBB6
:107E2000F3F285FB03E403FB1200DB173032D3EBE4
:107E3000A40380B201F8012BF1D10B7030BD064BC9
:107E40001868086070472D230B700131DEE700BF12
:107E50006C9FFF1F67666666D0480100174B1B8842
:107E60001BB31BB270B583EAE375A5EBE375002B7A
:107E7000ACB21EDB012300E0034603EB83004000AD
:107E80008542F9DA0E4E94FBF3F086FB03E503FB23
:107E90001044DB173030D3EBA503A4B201F8010B7B
:107EA000F1D108480B70106070BD074B186808606E
:107EB00070472D230B700131DCE700BF429FFF1F8D
:107EC0006766666644490100D0480100054B1B887F
:107ED0001BB1054B186808607047044B18680860B0
:107EE000704700BF729DFF1F5849010054490100AF
:107EF00070B5FAF72FF9164B1B7813B1154C237890
:107F000033B9154B1020198801F0B0FE012070BD67
:107F1000124D134E2B783288B3FA83F382F00802A5
:107F20005B09114642202B70328001F09FFE2378BE
:107F30000BB12B782BB90021212006F0E1FB0020AA
:107F400070BD0121212006F0DBFB002070BD00BFC9
:107F5000D49CFF1F9A9EFF1FB49EFF1FB29EFF1F5F
:107F6000669FFF1F184B1A8852B3184A128830B503
:107F70000A80B3F90030002B83EAE374A4EBE374C6
:107F8000BCBF2D238B70A0B2ACBF023103310123E3
:107F900000E0134603EB830252009442F9DA0C4DE1
:107FA00090FBF3F285FB03E403FB1200DB17303296
:107FB000D3EBA40380B201F8012BF1D10B7030BDDB
:107FC000044B186808607047289DFF1F5C4901003A
:107FD00067666666D048010070B53C4D2B78064652
:107FE000002B35D11C4673780BB9204670BDFAF7CB
:107FF000B1F8374A374B3848127831781B78007817
:1080000002EB43034A1E03EB80030E2AEDD801A0C6
:1080100050F822F07D8000009F800000EB7F000080
:108020007D800000EB7F0000EB7F0000EB7F000015
:108030006B800000EB7F0000EB7F0000EB7F000017
:10804000EB7F0000EB7F0000EB7F0000678000000B
:10805000AE21224804F0F0FB204804F039FE002352
:108060002B700124BFE707F0B9FBAF211B4804F0D8
:10807000E3FB1B4A012313702B70B6E783B9194841
:10808000038804294FF6FF7103F1FF320CBF01236F
:108090000B46134403F07F03013303800FE073B1F9
:1080A000013B114A32F813304BB10E4E0F481049C4
:1080B000104A33800123002606700B701370084AA3
:1080C0000221012311702B70204670BD288BFF1FE9
:1080D000499FFF1F4A9FFF1F4B9FFF1FC49FFF1F0A
:1080E00044A0FF1F349FFF1F749EFF1F5C9DFF1F56
:1080F000DC9CFF1F47A0FF1F10B5064B064C1A88DB
:108100002046012101F0A0FD21884220BDE8104059
:1081100001F0ACBD409DFF1F669FFF1F10B5064BD1
:10812000064C1A882046022101F08EFD218842204B
:10813000BDE8104001F09ABD869DFF1F669FFF1F9E
:1081400010B5064B064C1A882046042101F07CFD30
:1081500021884220BDE8104001F088BDAA9EFF1F83
:10816000669FFF1F10B5064B064C1A88204600215B
:1081700001F06AFD21884220BDE8104001F076BD83
:10818000F29EFF1F669FFF1F08B5122001F088FDB9
:10819000054B1988884206D0122001F067FDBDE822
:1081A000084001F005BC08BDE89EFF1F08B5582037
:1081B00001F076FD054B1988884206D0582001F061
:1081C00055FDBDE8084001F0F3BB08BDF69EFF1F5A
:1081D00008B5142001F064FD054B1988884206D0CB
:1081E000142001F043FDBDE8084001F0E1BB08BDEB
:1081F0008E9DFF1FF0B480EAE075A5EBE0750028C6
:10820000ACB21FDB1DBF2B230B704E1C0E4601238F
:1082100000E0134603EB830252009542F9DA0B4F5C
:1082200094FBF3F287FB030503FB1244DB173032A8
:10823000D3EBA503A4B206F8012BF1D133700846A5
:10824000F0BC70472D230B704E1CE0E76766666636
:10825000084B188828B10D2807D00D3800B2FFF759
:10826000C9BF054A106808607047044A1068086072
:10827000704700BF9A9FFF1FD0480100604901006E
:10828000174B18880C2813D0192815D01A2817D086
:108290001B2819D01C281BD01D281DD01E2803D038
:1082A0000C3800B2FFF7A6BF0E4A1068086070478E
:1082B0000D4A1068086070470C4A106808607047E3
:1082C0000B4A1068086070470A4A106808607047D7
:1082D000094A106808607047084A106808607047CB
:1082E000329FFF1F7C490100644901006849010079
:1082F0006C4901007049010074490100784901008E
:10830000034B1888A0EB8000400000B2FFF772BF5B
:108310002CA0FF1F024B1888033800B2FFF76ABF7A
:108320000A9FFF1F024B18880C3800B2FFF762BF8C
:10833000CE9CFF1F024B1888183800B2FFF75ABFB7
:10834000089DFF1F024B1888183800B2FFF752BF74
:10835000069DFF1F024B1888183800B2FFF74ABF6E
:10836000469FFF1FC3681888183800B2FFF742BF46
:10837000054B1B881BB9054B1868086070470846F9
:10838000042203490AF09ABF0E9DFF1FD048010046
:10839000CC480100054B1B881BB9054B18680860C9
:1083A00070470846042203490AF088BF7C9DFF1FDE
:1083B000D0480100CC48010030B5134C85B00125F0
:1083C0002B463C2202212046009504F0ABFA2046C1
:1083D00004F07EFC0022402180232046019100937E
:1083E00011460A4B029505F021F9204604F07CFD68
:1083F00007480849084A0023036083800B608B808C
:108400001360938005B030BDC49FFF1F3844010046
:10841000A89FFF1FBC9FFF1F34A0FF1F10B500EBDC
:10842000C00000F10F02D2B293B284B09C1E981C1F
:108430003D2303918DE819003921024805F05AF8CF
:1084400004B010BDC49FFF1F014B01221A7070477A
:10845000B59FFF1FF0B5704B704C714F714E724D50
:1084600085B004228DE80C00029320466F4B402219
:10847000802104F05FF820466D4C6E4A6E4909F089
:10848000A5F8A7616D486E4FE7616E4F87616E4931
:108490006E4FC7616E4F8F616E4A6F4FCF616F4FE6
:1084A00097616F4B6F4FD7616F4F9F616F4FDF6168
:1084B0006F4FB7616F4FF7616F4FAF616F4C704F88
:1084C000EF61704FA7617048704FE761704F87612F
:1084D0007049714FC761714F714A8F61714FCF61A0
:1084E000714F724B9761724FD761724F724E9F619D
:1084F000724FDF61724F734DB761734FF761734F06
:10850000734CAF61734FEF61734F7448A761744F41
:10851000E761744F74498761744FC761744F8F610D
:10852000744A754FCF61754F9761754B754FD76121
:10853000754F9F61754E764FDF61764FB761764D0F
:10854000764FF761764FAF61764C774FEF61774F9B
:10855000A7617748774FE761774F87617749784F11
:10856000C761784F8F61784A784FCF61784F9761B4
:10857000784B794FD761794F9F61794E794FDF61A1
:10858000794F7A4DB7617A4FF7617A4F7A4CAF6184
:108590007A4FEF617A4F7B48A7617B4FE7617B4F52
:1085A0007B4987617B4FC7617B4F7C4A8F617C4FE2
:1085B000CF617C4F7C4B97617C4FD7617C4F7D4E68
:1085C0009F617D4FDF617D4F7D4DB7617D4FF761CD
:1085D0007D4F7E4CAF617E4F7E487F49EF617F4F7C
:1085E0007F4DA761E5617F4F7F4D804CDFF820E232
:1085F0007F4A804B8761C5618C617F4E7F4F804D84
:10860000804CC1F81CE0804880499761D5619C612D
:10861000D861B16005B0F0BD40420F00C49FFF1F9C
:1086200025830000D08DFF1F408DFF1F7091FF1F1D
:10863000F48DFF1F1C89FF1F8DC50000908FFF1F49
:108640002D6F000015830000DC8EFF1F396F0000C6
:10865000C1710000D48CFF1FF9800000E971000097
:10866000B48FFF1F1D8100001172000041810000C6
:108670000D790000496F000039720000AC8DFF1FBA
:108680006581000001830000888DFF1F7174000068
:10869000897400006C8FFF1F7D7400004179000019
:1086A000688CFF1F59780000757900002090FF1F2B
:1086B00089810000E57B00001C8DFF1FAD8100005B
:1086C000E1740000288CFF1F596F000061720000E8
:1086D000B090FF1FD18100004D7C0000F88CFF1F7F
:1086E000696F0000B57C0000188EFF1F796F0000D5
:1086F000257D0000B08CFF1F896F000041750000D0
:10870000E08BFF1F996F0000B17900006890FF1F98
:10871000A96F000099750000248FFF1FB96F00003A
:10872000E5790000988BFF1FC96F0000F17500000C
:10873000508BFF1FD96F0000197A0000E08AFF1FDD
:10874000E96F000049760000648DFF1FF96F00009B
:10875000657F0000488FFF1F09700000517A0000FC
:108760004C91FF1F197000008D7D0000B88EFF1F17
:1087700029700000F57D0000748BFF1F3970000028
:10878000857A00004490FF1F797800005D7E00002C
:10879000008FFF1F4970000081820000BC8BFF1F0B
:1087A00059700000BD7A00002C8BFF1F697000001B
:1087B000257B0000988AFF1F79700000518200001D
:1087C0001891FF1F89700000A17600008C8CFF1F9C
:1087D00099700000048BFF1F048CFF1FF9760000C6
:1087E000A970000051770000B9700000A97700005F
:1087F000D88FFF1FBC8AFF1F4091FF1F0178000028
:10880000D9700000CD7E0000E9700000CD8D000021
:10881000C9700000F0B5461C83B00D460127032344
:1088200036B22AB2044631468DE888002348ADB2FC
:1088300004F0F6FD0C23AA1C12B200930197052345
:1088400021B21E4804F0ECFD1D4A1E4B12881B6825
:10885000BA422AD023D3022A10D11B4CA3F6CA0352
:1088600084FB03241C44DB17C3EB24140A2CA8BF8D
:108870000A2424EAE474A2B223B202E000231A46D6
:108880001C460D35AA1A01200093019012B2314600
:1088900003230A4804F042FD204603B0F0BD0B4C10
:1088A000A3F6FC0384FB0324DDE7094CA3F698033D
:1088B00084FB0324DB17C3EBA404D7E7C49FFF1F8B
:1088C000949EFF1FF89EFF1F898888881F85EB51A3
:1088D000398EE3382DE9F0438FB283B0DFF84C8056
:1088E000BD1D461D2DB204B236B24FF001090AB2C9
:1088F0002346314640460095CDF8049004F040FDF3
:108900002A463346214640468DE8200204F038FDD1
:1089100007F10C020095334612B22146CDF80490BF
:10892000404604F02DFD03B0BDE8F083C49FFF1F57
:108930002DE9F04F804685B0002959D101213148F9
:1089400005F0A8F8304998F8062098F8083011F892
:108950000290994525DADFF8ACB04FEA89064D461A
:108960000C244FF0000AD8F80C309B595F68ABF824
:1089700010403846ABF80EA00AF0E2FB394602463A
:10898000204808F0B5FA1F4808F0C8FA98F80830EF
:1089900001350934AB42A4B206F1040601DD422CD4
:1089A000E1D1B9F1000F13D109F1060999450CDAAB
:1089B0003C2301213B22039102930093019239232E
:1089C0003F223A210F4804F095FD05B0BDE8F08F35
:1089D0000F2301213B22039102930093019239233B
:1089E0000C223A21074804F085FD98F80830DBE7AF
:1089F00000213423009301913F230C22014804F00D
:108A00008DFC9BE7C49FFF1FBC9FFF1F38B50F4C19
:108A1000012320461946A3826382552505F03AF8C2
:108A20003423204602220A492382E58108F060FAB5
:108A300020460522074908F05BFA204608F06EFA46
:108A40002046BDE8384004F04FBA00BFC49FFF1F66
:108A5000C8490100CC490100F8B50F4606460AF0A6
:108A60006FFB00EB40008400AFB338460AF068FBB0
:108A700000EB4000400023185B10194D03F1600229
:108A8000121A4FF0280E01212846C3F16004EA8132
:108A9000A5F810E004F0FEFF38460AF051FB394615
:108AA0000246284608F024FA284608F037FA022140
:108AB0000B4804F0EFFF212330462B82EC810AF0B3
:108AC0003FFB31460246064808F012FA0448BDE86A
:108AD000F84008F023BA6410C4F16004004DE6E7E2
:108AE000C49FFF1F10B50D4B1B5C51F8234023782A
:108AF00084B013B1012004B010BD04AA01A942F84A
:108B0000103D2046A3699847A38A9B07F2D401A889
:108B10000099FFF7A1FF012004B010BDA89FFF1F1F
:108B20002DE9F04F304DDFF8D0B0DFF8C8A00FCD01
:108B300091B003AC0FC40FCD0FC40FCD0FC42B6881
:108B400023600025A8462F462E4600E09846BAF836
:108B5000003026495BF82320DFF8A0901123284637
:108B6000F7F740FE00EBC00300EB8300204B83FBD4
:108B700000340444C017C0EB6434C4F13C00C6F1B7
:108B80003C0207F14101012600B208F141030090C7
:108B90001BB2019612B209B2484604F0F1FB08EB91
:108BA000060305F211153C2B2646ADB24746CDD142
:108BB0006B22342300214846A9F80E20A9F8103072
:108BC00004F068FF0B4B1B8810AA02EB830353F8D9
:108BD000344C20460AF0B4FA21460246484611B009
:108BE000BDE8F04F08F084B9D0410100A03B01007E
:108BF00009000280EE9CFF1F043A0100C49FFF1F82
:108C0000234B70B5B3F9003083EAE374A4EBE3744B
:108C1000002B82B0A1B234DB68466D46012300E030
:108C2000134603EB830252009442F9DA194E91FB8A
:108C3000F3F286FB03E403FB1211DB173032D3EBB4
:108C4000A40389B205F8012BF1D119462B70FFF767
:108C500003FF114B1B7813B1104B1B780BB902B0FB
:108C600070BD0F4C0121204604F014FF642533230E
:108C7000204604220B49E581238208F039F902B02D
:108C800070BD2D238DF800300DF101056846C5E754
:108C9000B49EFF1F676666669A9EFF1FB29EFF1F07
:108CA000C49FFF1FD449010070B5404E404D82B0B3
:108CB000304604F00DF82B78D3B93C4C0621204601
:108CC00004F0E8FE2B78012B38D9022B4FF0030279
:108CD0004FF00A030CBF37493749E381204623820E
:108CE00008F006F9204602B0BDE8704008F016B959
:108CF000324B1A7801210523002A33D101910093C8
:108D00001146304604F08CFB2D4B1A78002A34D0E3
:108D1000052301220192009300220A21234804F036
:108D2000FDFA284B1A78002A33D10121052301913D
:108D3000009314211D4804F073FBBEE7224B1988F1
:108D4000092930D963298CBF0A221F220A23174818
:108D5000F281338208F032F9144802B0BDE8704065
:108D600008F0DCB80022019100931146304604F06F
:108D7000D5FA134B1A78002ACAD105230121019193
:108D800000930A21094804F04BFB0E4B1A78002A85
:108D9000CBD0012205230192009300221421034825
:108DA00004F0BCFA89E73022D0E700BFC49FFF1F60
:108DB00047A0FF1FDC490100E0490100499FFF1F58
:108DC0004A9FFF1F4B9FFF1F349FFF1F2DE9F04756
:108DD000714E307848B9714B1B6899425FD3704A25
:108DE000012313703370BDE8F0876E4D6B4F0C4656
:108DF000284603F06DFF04F6AC5331240022EC81C9
:108E00000124114628462A82AC826C823B60327073
:108E100004F040FE05226449644E284608F068F8D4
:108E2000102728464FF00C0808F078F80B2260490C
:108E3000EF812846A5F8108008F05AF85D49052210
:108E4000284608F055F8284608F068F85A4BEF8194
:108E50001A68A2F69803C3EB031386FB03161E449D
:108E6000DB17C3EB662640F6CC3320219A422982D9
:108E700006F124064FF022014FF0040011DCFFF749
:108E8000C9FC4E4BB3F800908246B9F1000F30D0C8
:108E9000B9F1010F4DD0B9F1020F47D02046BDE81E
:108EA000F087FFF717FD46490922284608F020F809
:108EB0004449EF8181FB0637F317C3EBA7072A2349
:108EC000394628462B8208F079F822463E49284642
:108ED00008F00EF807EB8701A6EB4101284608F0E1
:108EE0006DF822462846394908F002F82046BDE8C8
:108EF000F08737493A46284607F0FAFF284608F037
:108F00000DF82A232B825146EF8128462D4F08F079
:108F100055F807222F49284607F0EAFFF31787FB89
:108F20000627C3EBA70739462846CCE742462A491D
:108F3000E1E742462949234C284607F0D9FF284655
:108F400007F0ECFF2A232B8251462846EF8108F0D8
:108F500035F807221F49284607F0CAFFF31784FB9C
:108F60000624C3EBA4042146284608F027F84A4605
:108F70001549284607F0BCFF04EB8401A6EB41012C
:108F8000284608F01BF84A462846104907F0B0FF6B
:108F90004846BDE8F08700BF288BFF1F28A0FF1FB1
:108FA00044A0FF1FC49FFF1FE44901003B773B988B
:108FB000EC490100CC490100F89EFF1F949EFF1F61
:108FC000F849010067666666E051010050510100F2
:108FD000044A0100184A0100304A0100204A0100F9
:108FE0002DE9F041744C2278002A05460F4614BF43
:108FF0004FF001084FF000084ED1704E3368CB1A85
:10900000B3F5FA6F04D86B78A3B94046BDE8F08198
:109010006B4B6C486C49DFF8CCE11A70012303708C
:109020000988237026208EF8002000F01FFE6B7840
:10903000002BEAD03760F9F78DF8644A644B654934
:10904000127828781B78097802EB4303421E03EB61
:1090500081030E2AD9D801A151F822F049910000CC
:10906000159100000B900000499100000B9000004A
:109070000B9000000B900000FD9000000B90000092
:10908000B39000000B9000000B9000000B900000CC
:109090000B900000AF900000AF214F48474E03F007
:1090A000CBFBFFF701FE002337602370ABE706F030
:1090B00095FB494C204603F00BFE2046022104F0AC
:1090C000E9FC23250F23238205224449E58120461C
:1090D00007F00EFF204607F021FF1E23052240491E
:1090E00023822046E58107F003FF204607F016FFA4
:1090F000204603F0F9FE00F0ABFC86E7394D2B78F3
:10910000012B50D9304B2620198800F0AFFD0023E9
:109110002B707AE7002B3FF478AF013B324A32F8EC
:109120001330002B3FF471AF274C304825492D4AAE
:1091300023804FF001080023037081F8008082F83B
:109140000080FFF7B1FD60E793B1013B264A32F89A
:10915000131019B31C4B254D1A4C224A19800026B6
:10916000012326202E702370137000F07FFD15E080
:10917000154C1E4922880B7004284FF6FF7002F12F
:10918000FF310CBF012202460A440E4E154D02F07B
:109190007F0201320121228031702B70FFF784FDA4
:1091A0004FF0010831E70649064A01230020087004
:1091B00013702370A6E700BF288BFF1F40A0FF1F7E
:1091C00044A0FF1FDC9CFF1F349FFF1F499FFF1F10
:1091D0004A9FFF1F4B9FFF1FC49FFF1F404A010074
:1091E000484A010047A0FF1F749EFF1F5C9DFF1FA0
:1091F0002DE9F04FAE4E4FF00109A6F81490A6F8F5
:109200001290838813EA09048BB005460F469346F3
:1092100040F0AB80DFF8C48298F80030002B7BD19F
:10922000AA79A44CA35CA3B9DFF8B4A279781AF8A0
:10923000029039B33B78013B072B00F2B280DFE8A4
:1092400013F0EF005101B0006B01B000B000B000AE
:10925000E7007E78002E00F0C580013BE868397891
:1092600050F82360F0684B1E0788072B00F2A3809C
:10927000DFE813F070015901A1006A01A100A1000B
:10928000A1009B008C4E3368C3EB0B03B3F5967FB4
:1092900072D98A4B187801281ABF012018701970EA
:1092A000874B18BF0146985CC0EB0900C0B2FFF7BE
:1092B000B5F80124C6F800B0AB889B076DD57B7864
:1092C000002B6AD0F8F746FF7E4B7F4A7F481B7819
:1092D000127839780078022515FB02330A2903EB4E
:1092E000800300F049810C2957D1002B55D003F1A0
:1092F0001900774E774A013B0021400080B226F8E2
:1093000013100123157088F8003000F0AFFC724B89
:10931000032220461A702CE0304603F0D9FC304678
:10932000494604F0B7FBF4813482AB88580725D452
:109330002C68204609F004FF21460246304607F01B
:10934000D7FD304607F0EAFD092201238DE80C0025
:1093500000217F23564804F013F800212846FFF728
:10936000E7FA002388F800305AE783681146384648
:1093700098470BB0BDE8F08F0846FAE72B6804A8C1
:10938000984704A809F0DCFE04A90246304607F01D
:10939000AFFD304607F0C2FDD6E720460BB0BDE872
:1093A000F08F00240AF8029086E70023A354304689
:1093B000F3699847F0680780002425223C238DE854
:1093C0001400412118223A4803F0A8FFE968A8795F
:1093D000FFF788FB394A384B1470C3F800B00BB064
:1093E000BDE8F08F34490B68C3EB0B03B3F5967FF0
:1093F00040F2E080314FC1F800B03C78012C00F021
:10940000AF800123E9683B701046FFF76BFBB0E7C4
:10941000304BE9791970012388F800300024C1E746
:109420002B7A013B4B45BCDD09F10104E4B2A145B7
:10943000B7D0234E16F802B0CBEB0900C0B2002122
:10944000FEF7ECFF2B7A052BD9461BD9CBEB040298
:10945000042A40F3A980A4F1040BBBF1000FC0F271
:10946000AD80063B5B45A8BF5B465FFA83F9AA79EE
:109470001348B15C994205D000F8029001212846BA
:10948000FFF756FAC9EB0400C0B201210B4EFEF7FC
:10949000C5FF00213423019100930B223170044851
:1094A00040233F21A14603F039FF0124AA7979E73F
:1094B000C49FFF1F34A0FF1F30A0FF1F45A0FF1F48
:1094C000BC9FFF1F499FFF1F4A9FFF1F4B9FFF1F0E
:1094D000749EFF1F44A0FF1F47A0FF1F288BFF1F84
:1094E000A89FFF1F0FFA89F3E9685D4851F823B080
:1094F000036804935B499BF8003004980860002BD4
:109500006CD0012B7FF44DAF57499BF8080088F8C9
:1095100000300870002445E7B9F1000F4CD009F184
:10952000FF34E4B283E7B38A03F004039BB2002B59
:109530003FF43CAF336A984700283FF43BAFAB7928
:10954000F0680022E25436E7738ABB4240D9013703
:10955000BFB230E7338ABB4234D2013FBFB22AE701
:1095600025238DE8480041483E703C2318224121C4
:1095700003F0D4FE2046FCE6002B3FF40EAF3C4A3D
:109580003C4E1188384A03F11900013B400080B27B
:1095900026F81310012388F80030157000F066FBE0
:1095A000354B20461D70E4E6002A3FF75AAF04F120
:1095B000FF3B52E73046DCE64C46F3E64FF000094D
:1095C0004B4654E7B38AD9077FF5F5AE778AF2E6C2
:1095D000B38ADA077FF5EFAE378AECE627490393C3
:1095E000885CC0EB090009F1010EC0B2012104F84A
:1095F00002E0FEF713FF039BDBF808B0019334236E
:109600001A4800930B2240233F2103F087FE0124D8
:1096100034230B228DE818003F214023134803F028
:10962000FFFE2146114804F035FA584609F088FD3E
:10963000A0EB800000F15F030F22F38132825846D5
:1096400009F07EFD59460246084807F051FC0748DC
:1096500007F064FCE968A879FFF744FAAA79A1E663
:1096600064A0FF1F30A0FF1F44A0FF1FC49FFF1F67
:10967000349FFF1F749EFF1F47A0FF1FBC9FFF1F4B
:109680002DE9F047DFF808926D4B99F800601B68F0
:10969000DFF800A282B0003601934FF0030018BF3C
:1096A0000126019F9AF8008005F030F80546042055
:1096B00005F02CF80446052005F028F8800040EA63
:1096C0004404062005F022F82C4364B25D4944EAC4
:1096D000C0000A7880F00F03DBB29A425A4A3CD0AD
:1096E0001760002259480B7003788DF800808DF8C0
:1096F000012053B3564A12684EF66021BA1A8A42C4
:1097000019D8022B59D0012B5FD0062B48D0032B40
:1097100063D0042B69D0052B77D0072B7DD0082B85
:1097200000F08380092B68D016B14A4803F0DCFBB7
:1097300002B0BDE8F087484A484C0023012123705D
:1097400003701360938089F800103A4669464448D4
:10975000FFF74EFD3043C6B2E6E71268BA1A1E2A7A
:109760006BD99AF80020934222D0394C3D488AF8B0
:109770000030012B276082EA030207609846B1D0CF
:10978000042BAFD137480068381AB0F5C87FA9D983
:10979000354C2068381A3228A4D927601A46A1E728
:1097A0003A4669463148FFF723FD3043C6B2BBE76E
:1097B000012B4FF00002E3D1E4E73A4669462C481A
:1097C000FFF716FD3043C6B2AEE73A466946294870
:1097D000FFF70EFD3043C6B2A6E73A466946264873
:1097E000FFF706FD3043C6B29EE73A466946234876
:1097F000FFF7FEFC3043C6B296E73A46694620487A
:10980000FFF7F6FC3043C6B28EE73A4669461D487C
:10981000FFF7EEFC3043C6B286E73A4669461A487F
:10982000FFF7E6FC3043C6B27EE73A466946174882
:10983000FFF7DEFC3043C6B276E7002252E700BFF6
:1098400064A0FF1F48A0FF1FB09FFF1F44A0FF1F81
:109850003CA0FF1FC49FFF1F34A0FF1F46A0FF1F97
:10986000084401004CA0FF1FB89FFF1F38480100AB
:1098700084430100984201003442010090500100ED
:1098800088420100F0420100D05001004091FF1FCA
:10989000288BFF1FB49FFF1F28B11028044BA8BFBF
:1098A000102018607047024B01201860704700BFFD
:1098B00050A0FF1F08B5002006F088FE0028FAD14E
:1098C00008BD00BF70B50D461446064605F04EFDB6
:1098D000284605F04BFD204605F048FD084B1B7857
:1098E00013B1084B1B7803B970BD304605F0CCF9B5
:1098F000284605F0C9F92046BDE8704005F0C4B916
:109900009A9EFF1FB29EFF1F38B5164D2B78044656
:1099100041F6FF72A0F50050824203F1FF33A8BF69
:1099200002461B0202F5005203F47063100443F474
:10993000604343F00E0300F4FE005204184302F0AB
:10994000FE42104306F078FD2868013860F01F00E1
:10995000C4F3C61204F07F01C0B2BDE83840FFF77F
:10996000B1BF00BF50A0FF1F70B5104E3378013B50
:109970001B0203F47063044643F4304308062204D8
:1099800000F0FE4043F00B03034302F4FE001843D3
:109990000D4606F051FD3068013860F04F002A4650
:1099A0002146C0B2BDE87040FFF78CBF50A0FF1F3A
:1099B00008B564210720FFF7D7FF7F210B20BDE802
:1099C0000840FFF7D1BF00BF70B5104E3378013BA0
:1099D0001B0203F47063044643F410430806220498
:1099E00000F0FE4043F00903034302F4FE00184375
:1099F0000D4606F021FD3068013860F06F002A4600
:109A00002146C0B2BDE87040FFF75CBF50A0FF1F09
:109A100038B50E4D2B78013B1B0203F470630446EE
:109A200043F41043000443F0090300F4FE0018431C
:109A300006F002FD2868013860F06F002146C0B2D0
:109A40000022BDE83840FFF73DBF00BF50A0FF1F18
:109A500010B500217B20FFF787FF0024E0B2FFF75D
:109A6000D7FF0134022004F087FE802CF6D110BD10
:109A700038B50C46054605F079FC204605F076FC25
:109A8000074B1B7813B1074B1B7803B938BD284629
:109A900005F0FAF82046BDE8384005F0F5B800BFFB
:109AA0009A9EFF1FB29EFF1F38B50D4D2B78013BCC
:109AB0001B0203F47063044643F45043000443F074
:109AC0000D0300F4FE00184306F0B6FC28680138C8
:109AD00060F02F002146C0B2BDE83840FFF7C8BF94
:109AE00050A0FF1F38B50E4D2B78013B01381B02EB
:109AF000C4B203F47063200443F4404343F00C0306
:109B000000F4FE00184306F097FC2868013860F066
:109B10003F002146C0B2BDE83840FFF7A9BF00BFF3
:109B200050A0FF1F38B504460D46F02005F01EFC7E
:109B300035B1254414F8010B05F018FCAC42F9D1FD
:109B4000F720BDE8384005F011BC00BF00B50B4B55
:109B500083B00246998818680090032AADF8041073
:109B600002D903B05DF804FB684606218DF8052094
:109B7000FFF7D8FF03B05DF804FB00BF10510100F0
:109B800000B50B4B024683B0186899880090131FEC
:109B90004C2BADF8041002D903B05DF804FB684605
:109BA00006218DF80520FFF7BDFF03B05DF804FB2B
:109BB00018510100030203F4FE43C0F3C61018431A
:109BC000704700BF03784078DB0103F47E5300F058
:109BD0007F001843704700BF82B002AA114642F8C6
:109BE000040D002012F8013B03F07F03914243EA89
:109BF0000020F7D102B0704710B547F61221044695
:109C00000D4807F02FF805F0D1FB0C4B1B7833B94A
:109C100074B1102C0A4BA8BF10241C6010BD47F66D
:109C20001221084806F06EFF05F0EAF8002CF0D18A
:109C3000034B01241C6010BD4C93FF1F9A9EFF1F15
:109C400050A0FF1F3893FF1F003210B403884FF05D
:109C5000010404FA01F418BF012202FA01F123EA17
:109C600004020A43028010BC704700BF70B5CEB238
:109C70000C46054604F0DAF9864203D03146284600
:109C800004F0EEF90135284604F0D0F9240A8442A4
:109C900005D021462846BDE8704004F0E1B970BD0A
:109CA00038B5054604F0C2F94FF0000460F307042C
:109CB000681C04F0BBF960F30F24A0B238BD00BFEC
:109CC000F8B504460020FFF7EBFF002C00F09C8560
:109CD0004FF4AF610220FFF7C9FF4FF47A6104200F
:109CE000FFF7C4FF4FF496610620FFF7BFFF4FF464
:109CF000FA610820FFF7BAFF4FF4FA610A20FFF774
:109D0000B5FF40F6B8310C20FFF7B0FF4FF42F61DC
:109D10002220FFF7ABFF40F6AC512420FFF7A6FF4F
:109D20007D212A20FFF7A2FF0C210E20FFF79EFFC6
:109D300001211020FFF79AFF02211220FFF796FF62
:109D400000211420FFF792FF00211620FFF78EFF5D
:109D500002211820FFF78AFF01211A20FFF786FF52
:109D600001211C20FFF782FF04211E20FFF77EFF48
:109D700014212020FFF77AFF01212620FFF776FF2C
:109D800003212820FFF772FF04212C20FFF76EFF2C
:109D900014212E20FFF76AFF00213020FFF766FF15
:109DA0000C213220FFF762FF00213420FFF75EFF15
:109DB00000213620FFF75AFF00213820FFF756FF19
:109DC00000213A20FFF752FF00213C20FFF74EFF11
:109DD00000213E20FFF74AFF00214020FFF746FF09
:109DE00000214220FFF742FF1F214420FFF73EFFE2
:109DF00013214620FFF73AFF0E214820FFF736FFD8
:109E000011214A20FFF732FF0A214C20FFF72EFFD5
:109E100000214E20FFF72AFF06215020FFF726FFE2
:109E200002215220FFF722FF0C215420FFF71EFFD2
:109E300000215620FFF71AFF00215820FFF716FFD8
:109E400001215A20FFF712FF08215C20FFF70EFFC7
:109E50000A215E20FFF70AFF00216020FFF706FFBE
:109E600004216220FFF702FF01216420FFF7FEFEBC
:109E700000216620FFF7FAFE0B216820FFF7F6FEAF
:109E80007F216A20FFF7F2FE00216C20FFF7EEFE33
:109E900000216E20FFF7EAFE00217020FFF7E6FEAA
:109EA00000217220FFF7E2FE00217420FFF7DEFEA2
:109EB0001F217620FFF7DAFE13217820FFF7D6FE68
:109EC0000E217A20FFF7D2FE11217C20FFF7CEFE73
:109ED0000A217E20FFF7CAFE1F218020FFF7C6FE61
:109EE00013218220FFF7C2FE0E218420FFF7BEFE61
:109EF00011218620FFF7BAFE0A218820FFF7B6FE5F
:109F000000218A20FFF7B2FE00218C20FFF7AEFE71
:109F100000219620FFF7AAFE00219820FFF7A6FE59
:109F200000219A20FFF7A2FE05219C20FFF79EFE4C
:109F300006219E20FFF79AFE0021A020FFF796FE43
:109F40007F21A220FFF792FE40F2A461A420FFF738
:109F50008DFE4FF4E161A620FFF788FE0021A820C6
:109F6000FFF784FE0021AA20FFF780FE0221AC202B
:109F7000FFF77CFE0121AE20FFF778FE0121B02023
:109F8000FFF774FE0B21B220FFF770FE2A2100209C
:109F9000FFF76CFE0220FFF783FEB0F5805F0346FB
:109FA00080F0F585D24A04201380FFF779FEB0F5E2
:109FB000805F034680F0E285CE4A06201380FFF7DB
:109FC0006FFEA0F52F739BB2B3F57A6F024606D9E8
:109FD00040F628210620FFF749FE40F62822C64B0E
:109FE00008201A80FFF75CFEA0F52F739BB2B3F533
:109FF0007A6F024606D940F6E4410820FFF736FEA4
:10A0000040F6E442BD4B0A201A80FFF749FEA0F556
:10A01000FA739BB240F6AC518B42024606D94FF41C
:10A02000FA610A20FFF722FE4FF4FA62B44B0C20CB
:10A030001A80FFF735FEA0F5FA739BB240F6AC51DB
:10A040008B42024606D940F6B8310C20FFF70EFECF
:10A0500040F6B832AB4B0E201A80FFF721FE1828CD
:10A06000034600F28485A84A10201380FFF718FEEB
:10A07000431E9BB20F2B024604D901211020FFF78B
:10A08000F5FD0122A14B12201A80FFF709FE0A28D4
:10A09000034600F265859E4A14201380FFF700FEF8
:10A0A0000128034604D900211420FFF7DFFD002317
:10A0B000984A16201380FFF7F3FD7F28034600F22D
:10A0C0004885954A18201380FFF7EAFD05280346C6
:10A0D00000F23885914A1A201380FFF7E1FD0C2821
:10A0E000034600F228858E4A1C201380FFF7D8FD16
:10A0F0000428034600F218858A4A1E201380FFF7C1
:10A10000CFFD0928034600F20885874A20201380E6
:10A11000FFF7C6FD4628034600F2F884834A222052
:10A120001380FFF7BDFDA0F5FA739BB240F6AC516A
:10A130008B42024606D94FF42F612220FFF796FD8D
:10A140004FF42F627A4B24201A80FFF7A9FDA0F567
:10A15000FA739BB240F6AC54A342024604D921469E
:10A160002420FFF783FD2246724B26201A80FFF73A
:10A1700097FD7F28034600F2C2846F4A282013808F
:10A18000FFF78EFD0628034600F2B2846B4A2A20B0
:10A190001380FFF785FDA0F132039BB2B3F5967FE4
:10A1A000024604D97D212A20FFF760FD7D22644B01
:10A1B0002C201A80FFF774FD0C28034600F29184CE
:10A1C000604A2E201380FFF76BFD1E28034600F225
:10A1D00081845D4A30201380FFF762FD0928034621
:10A1E00000F25384594A32201380FFF759FD1E288C
:10A1F000034600F24384564A34201380FFF750FD93
:10A200007F28034600F23384524C36202380FFF728
:10A2100047FD7F28034600F2238438206380FFF740
:10A220003FFD7F28034600F214843A20A380FFF705
:10A2300037FD7F28034600F205843C20E380FFF7CA
:10A240002FFD7F28034600F2F7833E202381FFF78E
:10A2500027FD7F28034600F2E98340206381FFF752
:10A260001FFD7F28034600F2DB834220A381FFF716
:10A2700017FD394D28804420FFF712FD3028034692
:10A2800000F2C883354A46201380FFF709FD3028C5
:10A29000034600F2B983324C48202380FFF700FDCB
:10A2A0003028034600F2AA834A206380FFF7F8FCB7
:10A2B0003028034600F29C834C20A380FFF7F0FC7B
:10A2C0003028034600F28E834E20E380FFF7E8FC3F
:10A2D0000128034604D900214E20FFF7C7FC0023C4
:10A2E000204A50201380FFF7DBFC431E3CE000BFF8
:10A2F0009C9DFF1F649FFF1F429DFF1F309FFF1FFC
:10A30000FC9EFF1F049DFF1FCE9CFF1FB49EFF1FDE
:10A31000E89EFF1F8E9DFF1FD29CFF1FA29DFF1F67
:10A32000289DFF1F1C9DFF1F0C9DFF1F429FFF1FAD
:10A33000B09EFF1FAC9EFF1F349FFF1F0A9FFF1F91
:10A340005E9FFF1FEE9CFF1F849DFF1F709FFF1FDE
:10A35000329FFF1F749EFF1F669FFF1F469FFF1FB8
:10A360000C9FFF1F1A9DFF1F9BB20B2B024604D9A7
:10A3700006215020FFF77AFC0622CF4B52201A808C
:10A38000FFF78EFC0428034600F22683CB4A5420B4
:10A390001380FFF785FC431E9BB21D2B024604D998
:10A3A0000C215420FFF762FC0C22C54B56201A806A
:10A3B000FFF776FC0128034604D900215620FFF759
:10A3C00055FC0023BF4A58201380FFF769FC7F2803
:10A3D000034600F2FB82BC4A5A201380FFF760FC60
:10A3E000431E9BB2092B024604D901215A20FFF7D4
:10A3F0003DFC0122B54B5C201A80FFF751FC431E47
:10A400009BB2102B024604D908215C20FFF72EFCDA
:10A410000822AF4B5E201A80FFF742FC431E9BB21E
:10A420001D2B024604D90A215E20FFF71FFC0A22D9
:10A43000A84B60201A80FFF733FC0228034600F285
:10A44000BF82A54A64201380FFF72AFC0128034637
:10A4500004D901216420FFF709FC01239F4A6220EF
:10A460001380FFF71DFCC31E9BB2012B024604D9CB
:10A4700004216220FFF7FAFB0422994B66201A8020
:10A48000FFF70EFC7F28034600F29482954A68206D
:10A490001380FFF705FC7F28034600F28582924A6D
:10A4A0006A201380FFF7FCFB7F28034600F27682C8
:10A4B0008E4A6C201380FFF7F3FB0428034600F25A
:10A4C00067828B4A6E201380FFF7EAFB1928034648
:10A4D00000F25882874A70201380FFF7E1FB0228C0
:10A4E000034600F24982844A72201380FFF7D8FBAA
:10A4F0000628034600F23A82804A74201380FFF750
:10A50000CFFB0528034600F22B827D4A8A20138068
:10A51000FFF7C6FB0A28034600F21C82794A8C200A
:10A520001380FFF7BDFB0428034600F20D82764A34
:10A5300098201380FFF7B4FB0128034604D90021BB
:10A540009820FFF793FB0023704A9A201380FFF7AF
:10A55000A7FB0128034604D900219A20FFF786FBB8
:10A5600000236B4A96201380FFF79AFB0B280346C3
:10A5700000F2E481674A9C201380FFF791FB831E61
:10A580009BB2032B024604D905219C20FFF76EFBEA
:10A590000522614B76201A80FFF782FB30280346A4
:10A5A00000F2C6815D4A78201380FFF779FB3028DE
:10A5B000034600F2B7815A4C7A202380FFF770FBE4
:10A5C0003028034600F2A8817C206380FFF768FBF7
:10A5D0003028034600F29A817E20A380FFF760FBBB
:10A5E0003028034600F28C818020E380FFF758FB7F
:10A5F0003028034600F27E814A4A82201380FFF70A
:10A600004FFB3028034600F26F81474C84202380A3
:10A61000FFF746FB3028034600F260818620638006
:10A62000FFF73EFB3028034600F252818820A380CA
:10A63000FFF736FB3028034600F24481A020E38078
:10A64000FFF72EFB0128034604D90021A020FFF7C5
:10A650000DFB0023354A9E201380FFF721FBC31E0C
:10A660009BB20C2B024604D906219E20FFF7FEFA6E
:10A6700006222F4BA2201A80FFF712FB431E9BB22B
:10A680007E2B024604D97F21A220FFF7EFFA7F221A
:10A69000284BA4201A80FFF703FBA0F5AF639BB201
:10A6A000B3F5167F024647D940F2A461A420FFF714
:10A6B000DDFA40F2A4623FE03689FF1F7289FF1F76
:10A6C0002C8AFF1F729DFF1FF69EFF1FC89CFF1F55
:10A6D000788AFF1F7089FF1FA89EFF1F049FFF1F1E
:10A6E000309DFF1F449FFF1F649DFF1F109DFF1F94
:10A6F000BC9CFF1F9A9FFF1F949EFF1F6C9FFF1F14
:10A70000289FFF1FB69EFF1FA29EFF1F0E9DFF1FCB
:10A710007C9DFF1FF09EFF1FF49CFF1F069DFF1FE7
:10A72000849EFF1F089DFF1F8C9EFF1F149FFF1F0D
:10A73000D889FF1F3A9FFF1FD74BA6201A80FFF72B
:10A74000AFFAA0F5AF639BB2B3F5167F024606D908
:10A750004FF4E161A620FFF789FA4FF4E162CF4B95
:10A76000A8201A80FFF79CFA0628034600F2A4806E
:10A77000CB4AAA201380FFF793FA0328034600F27E
:10A780009580C84AAC201380FFF78AFA0328034655
:10A7900000F28680C44AB0201380FFF781FA0328B4
:10A7A000034677D8C14AAE201380FFF779FA7F2895
:10A7B000034669D8BE4AB2201380FFF771FA7F289A
:10A7C0005CD82B88DFF808E3BA4FBB4ABB4DBC4EC0
:10A7D000BC4CBD4903F0010CAEF800C0C3F3400E01
:10A7E000A7F800E0C3F380071780C3F3C007B74A98
:10A7F0002F70C3F30017C3F34015C3F380133780E2
:10A8000025800B801080F8BD4FF6FF7398423FF40F
:10A810005FAA2A283FF4BEAB17287FF659AA192849
:10A820007FF6C2AA1B287FF6DFAA1C283FF4F4AAF1
:10A830001E287FF6F9AA1F283FF4FEAA20283FF41D
:10A8400017AB21283FF420AB22283FF425AB232867
:10A850003FF42EAB24283FF45FAB25283FF464ABD4
:10A8600026283FF465AB27283FF46AAB28283FF43D
:10A8700075AB29287FF48AABFFF778BBB2200B2198
:10A88000FFF7F4F90B209CE70121AE20FFF7EEF96A
:10A8900001238FE70121B020FFF7E8F9012381E7C9
:10A8A0000221AC20FFF7E2F9022373E70021AA207E
:10A8B000FFF7DCF9002364E70021A820FFF7D6F9B1
:10A8C000002355E70A218820FFF7D0F90A23B5E6CF
:10A8D00011218620FFF7CAF91123A7E60E21842053
:10A8E000FFF7C4F90E2399E613218220FFF7BEF982
:10A8F00013238AE61F218020FFF7B8F91F237BE688
:10A900000A217E20FFF7B2F90A236DE611217C208F
:10A91000FFF7ACF911235FE60E217A20FFF7A6F9C5
:10A920000E2351E613217820FFF7A0F9132342E606
:10A930001F217620FFF79AF91F2333E60021962086
:10A94000FFF794F9002315E600218C20FFF78EF91C
:10A950000023ECE500218A20FFF788F90023DDE5DC
:10A9600000217420FFF782F90023CEE50021722038
:10A97000FFF77CF90023BFE500217020FFF776F98F
:10A980000023B0E500216E20FFF770F90023A1E558
:10A9900000216C20FFF76AF9002392E57F216A20ED
:10A9A000FFF764F97F2383E50B216820FFF75EF949
:10A9B0000B2374E500216620FFF758F9002365E5B5
:10A9C00000216020FFF752F900233AE500215820CA
:10A9D000FFF74CF90023FEE402215220FFF746F96D
:10A9E0000223D3E40A214C20FFF740F90A236BE449
:10A9F00011214A20FFF73AF911235DE40E21482086
:10AA0000FFF734F90E234FE413214620FFF72EF908
:10AA1000132340E41F214420FFF728F91F2331E4CA
:10AA200000214020FFF722F900231EE400213E20F0
:10AA3000FFF71CF9002310E400213C20FFF716F972
:10AA4000002302E400213A20FFF710F90023FFF76A
:10AA5000F4BB00213820FFF709F90023FFF7E5BB1D
:10AA600000213620FFF702F90023FFF7D6BB0021B3
:10AA70003420FFF7FBF80023FFF7C6BB0C21322080
:10AA8000FFF7F4F80C23FFF7B6BB00213020FFF7E7
:10AA9000EDF80023FFF7A6BBA09DFF1F1C9FFF1F23
:10AAA000CA9CFF1F489DFF1F069FFF1F989EFF1F08
:10AAB000189DFF1F409DFF1F869DFF1FB29EFF1F19
:10AAC000AA9EFF1F089FFF1FBA9EFF1F3A9DFF1FF0
:10AAD000F29EFF1F14212E20FFF7C8F81423FFF762
:10AAE00078BB04212C20FFF7C1F80423FFF768BBD3
:10AAF00003212820FFF7BAF80323FFF747BB012102
:10AB00002620FFF7B3F80123FFF737BB14212020DD
:10AB1000FFF7ACF81423FFF701BB04211E20FFF759
:10AB2000A5F80423FFF7F1BA01211C20FFF79EF8D6
:10AB30000123FFF7E1BA01211A20FFF797F801235B
:10AB4000FFF7D1BA02211820FFF790F80223FFF790
:10AB5000C1BA00211620FFF789F80023FFF7B1BA28
:10AB600002211220FFF782F80223FFF794BA0C218A
:10AB70000E20FFF77BF80C23FFF775BA4FF47A61CC
:10AB80000420FFF773F84FF47A63FFF715BA4FF418
:10AB9000AF610220FFF76AF84FF4AF63FFF702BA24
:10ABA000F8B5C52007F030FD204B214A054603CB00
:10ABB0001368C5F803001A0CB420C5F807102B80E1
:10ABC000AA70FEF7F7FF2E46002426F80B0FA0B25E
:10ABD000FFF766F8FEF7EEFF0234B42C26F8020FFA
:10ABE000F5D16C1E05F1C0064FF0FF3014F8013F9F
:10ABF000082758400F4B40F300017A1E0B4012F01B
:10AC0000FF0783EA5000F5D1B442EFD1C043FEF70D
:10AC1000E3FF3A46C5F8C100C521284605F05AFCB5
:10AC20002846BDE8F84007F0F7BC00BF24510100FA
:10AC3000205101002083B8EDF0B50E4B0E4C0546B7
:10AC400093E8070085B024682E88AD7801AB83E8CF
:10AC50000700270C184600220B21ADF804408DF8A0
:10AC60000670ADF80C608DF80E5005F033FC05B0A1
:10AC7000F0BD00BF3051010020510100F0B5124B72
:10AC8000124D1E68124F0FCD87B06C460FC495E869
:10AC9000030044F8040B38683B79CDF80D00320C02
:10ACA0002A2021808DF802208DF81130ADF8006047
:10ACB000FEF780FF0022ADF80B001221684605F078
:10ACC00009FC07B0F0BD00BF205101003C5101005C
:10ACD000CC490100002005F079BC00BF03F05EB94B
:10ACE00070B5104C82B00025402306462946204608
:10ACF000009301958023202202F010FB01232022E3
:10AD000030462282A3826382E58108F019FA314637
:10AD10000246204606F0ECF8204602B0BDE870403E
:10AD200002F0E2B8C49FFF1FF0B5C42983B075D903
:10AD30000546441E00F1C0064FF0FF3014F8012F05
:10AD400008275040404A40F300017B1E0A4013F0A0
:10AD5000FF0782EA5000F5D1B442EFD1C043FEF7BD
:10AD60003BFF0146D5F8C1000190019A914202D003
:10AD7000B2F17F2F0BD105F10B00FEF723FFB428B2
:10AD80000BD03248FFF7ACFF002003B0F0BD3048D5
:10AD9000FFF7A6FF384603B0F0BD05F10D00FEF742
:10ADA00011FF2A2840D1002440F6AC5613E00428B5
:10ADB0001AD0062821D008281FD00A2828D00C280D
:10ADC00022D1A1F5FA7292B2B24201D8FEF74EFF3B
:10ADD0000234B42C0ED004F10D002844FEF7F2FE2C
:10ADE000022C0146A0B2E2D1B1F5805FEED302346D
:10ADF000B42CF0D1012003B0F0BDA1F52F7292B2B6
:10AE0000B2F57A6FE4D8E1E7222801D0242811D1E5
:10AE1000A1F5FA7292B2B242DAD8D7E70D48FFF73D
:10AE20005FFF002003B0F0BD0B48FFF759FF002083
:10AE300003B0F0BD2A28C9D1A1F1320292B2B2F515
:10AE4000967FC5D8C2E700BF2083B8ED80510100CE
:10AE50006C510100545101009451010003290CD997
:10AE600070B5461C82B005460C46304603222A497E
:10AE700008F0D4F910B102B070BD70470B2C05D9A1
:10AE800005222649281D08F0C9F940B12448FFF7DA
:10AE900027FF244802B0BDE87040FFF7CDBE05F1A2
:10AEA0000901032201A808F009FA01A803221E499A
:10AEB00008F0B4F9D8B103221C4901A808F0AEF992
:10AEC00008B301A803221A4908F0A8F9B0B9194833
:10AED000FFF706FFA11E89B23046FFF725FF0028C5
:10AEE000C9D0154802B0BDE87040FFF7F9BE13485D
:10AEF000FFF7F6FEFFF754FE1148F3E71148FFF79E
:10AF0000EFFE1148C6E71148FFF7EAFE02B0BDE8C0
:10AF10007040FFF7B3BE00BF20510100AC510100EB
:10AF2000B4510100C8510100CC510100F45101009D
:10AF30000C5201001052010024520100D0510100B6
:10AF4000E4510100385201004C520100F851010057
:10AF50002DE9F043174D2B6883B081460F4690468C
:10AF6000F3B1154E34880A1992B218461146328050
:10AF700007F0C8FE28603A464946204402F092FD98
:10AF8000B8F1000F09D031882868FFF767FF2868FB
:10AF900007F042FB00232B60338003B0BDE8F08351
:10AFA000054E01930846318007F02EFB019B286077
:10AFB0001C46E0E758A0FF1F54A0FF1F10B51D4C12
:10AFC0004FF4FA70FBF734FE204601F081FE0023B7
:10AFD000194601222046E3812382A282628202F086
:10AFE00059FD0B221449204605F082FF204605F04A
:10AFF00095FF0F221149204605F07AFF204605F003
:10B000008DFF0F490722204605F072FF204605F00C
:10B0100085FF204601F068FF0A4B0B4A1A604FF487
:10B02000FA70FBF705FEFFF729FE0848BDE810405F
:10B03000FFF756BEC49FFF1F505201005C52010033
:10B040006C5201006CA2FF1F51AF0000745201004E
:10B050000020704790F8392090F83800101A704797
:10B0600090F8383090F839209A4205D95A1C034498
:10B0700080F83820187E70474FF0FF30704700BFCF
:10B0800090F8383090F839209A4286BF1B18187E05
:10B090004FF0FF30704700BF704700BF38B505461E
:10B0A000B0F85E0090B195F85D301446C3F121020E
:10B0B00094420CD805F13B001844224602F0F2FC01
:10B0C00095F85D30234485F85D30204638BD012079
:10B0D00014462871EEE700BFB0F85E306BB190F80F
:10B0E0005D30202B07D8C218013380F85D30012075
:10B0F00082F83B107047012303710020704700BFA6
:10B100000023426980F8383080F8393080F85C30AC
:10B1100080F85D3080F85E3080F85F3006CA30B469
:10B120000D68046943662A4383660A60A370426916
:10B1300090F861301649146813441D7A5B7B01EB6B
:10B14000C5051B026D6803F4E06343F064032B60E4
:10B1500090F8623013449D7CDB7D01EBC5011B023E
:10B16000496803F4E06343F064030B6021685368AB
:10B17000194205D0036927225A70036904229A7183
:10B18000036920225A71036980229A7030BC70478B
:10B19000985D010043690CCB12681A420CD0094B30
:10B1A00099420AD9084B9942036994BF1A220D2289
:10B1B0005A70036904229A717047036927225A70F2
:10B1C000F7E700BF7F1A06003F420F0010B5026983
:10B1D000D378DBB2D90604463DD510215806D1708C
:10B1E00038D503F0040303F0FF02002B51D03D4992
:10B1F000626E00230B7084F85D30002A5BD09047AC
:10B2000094F85D30002B56D02369D0229A702369C0
:10B2100094F83B201A712369012284F85C200222F1
:10B22000DA7010BD304B84F860009C424AD02F4B3E
:10B230009C4252D094F8391013791F29DBB207D8F9
:10B240002848007820B16018013184F8391003765D
:10B250000223D37010BD5906C3D4917801F01001B8
:10B2600001F0FF000029DDD013F001031ED194F896
:10B270005C1094F85D00884281BF4B1C091984F86A
:10B280005C3091F83B3013712369D0229A702269A7
:10B29000DEE7236984F83920C0229A702369114AB5
:10B2A0001979012111700222DA7010BDC023937048
:10B2B00022691379CCE70122002384F85D2084F809
:10B2C0003B30A1E7626994F86130094913440322D5
:10B2D000187A02F0B3FF2269ACE7626994F8613032
:10B2E0000449F3E75CA0FF1F7091FF1FDC91FF1F73
:10B2F00055B3000061B300000369DB7803F020035D
:10B3000073B190F860300133DBB2012B80F860300C
:10B310001AD9426990F861301344187A03F00AB8D8
:10B3200070B5426903F0FF0590F86130134404469C
:10B33000187A02F0FFFFA36E5BB184F8385094F8DE
:10B340003900BDE87040184790F85F30002BE0D01E
:10B35000704770BD0148FFF7CFBF00BF7091FF1F5E
:10B360000148FFF7C9BF00BFDC91FF1F2DE9F0477F
:10B37000374FDFF8E0903B68026982B006460093E1
:10B38000DDF800800021A025D3789B065BD53B68C3
:10B390000193019BC8EB03030F2BF5D949B1102B87
:10B3A000F2D000209070336980229A7002B0BDE81C
:10B3B000F087726996F8613013440521187A03F01A
:10B3C000B3F9726996F861301344012193F812A021
:10B3D000504603F0A9F909240021504603F090F9E2
:10B3E0002B46013BFDD10121504603F089F92B4644
:10B3F000013BFDD1013CEFD1706996F86110014429
:10B400004FF4A0720C7A4B7B09EBC4011B02496814
:10B4100003F4E06343F064030B6096F86230034486
:10B42000997CDB7D09EBC1011B02496803F4E063F1
:10B4300043F064030B60013AFDD13269D3789B0677
:10B440004FF00101A3D4012002B0BDE8F08700BF96
:10B4500064A0FF1F985D0100F0B503691222DA7045
:10B460000269937803F0200385B004460D46002B53
:10B470005ED0B42393703C4922690B680093009E10
:10B4800005E00B680193019B9B1B042B42D8D378EA
:10B4900003F0200303F0FF00002BF2D094F85D309E
:10B4A000002B31D04FF0000E4FF0020C04EB0E03D6
:10B4B00093F83B3013710B680393039F206907E0F7
:10B4C0009B060DD50B680293029BDB1B052B28D82E
:10B4D000C378DBB203F0020202F0FF06002AEFD0CD
:10B4E00080F803C02669F378DBB2DF0632462DD43C
:10B4F0009F062BD5DB0731D40EF1010E94F85D3099
:10B500005FFA8EFE7345D1D800201DBB002384F85E
:10B510005E3004E09070236980229A70042005B0A8
:10B52000F0BD86702369802204209A7005B0F0BDBA
:10B5300003F0FF06FFF71AFF10B9042005B0F0BDB5
:10B54000236984F85F60B0229A7094E78023B37017
:10B550000420DAE726698023B370D7E7BEF1000F35
:10B560000CBF02200320F6E764A0FF1F2DE9F04185
:10B5700006690025122780F8385080F83950F77096
:10B58000D0F810C09CF802E00EF0200E88B00446FF
:10B59000884615461E46BEF1000F49D0B4238CF8EC
:10B5A0000230784B21691A680092DDF800E006E06D
:10B5B0001A6801920198CEEB0000042830D8C878B0
:10B5C00000F0200000F0FF070028F1D04FEA480209
:10B5D00042F00102D2B20A711A680292DDF808E064
:10B5E000206906E01A6803920399CEEB0101052950
:10B5F0002AD8C17801F0020101F0FF070029F1D03B
:10B600004FF0020C80F803C02269D17811F01107C5
:10B6100022D12DBB002E0CBFA0238023937003E00A
:10B620008F70236980229A70384608B0BDE8F08197
:10B630000EF0FF07FFF79AFE0028F5D0236984F883
:10B640005F70B0229A70ACE7877023698022384619
:10B650009A7008B0BDE8F081802393700027E3E77B
:10B66000012D75D0A021917021690A79BE466746E7
:10B670004FF0A80C1A680492049805E01A68059225
:10B68000059A121A052A4AD8CA7802F0020202F074
:10B69000FF08002AF2D0CF702169CA78D2B212F026
:10B6A000100F08465AD1920658D5013DEDB2012D32
:10B6B00049D0BEF11F0F3BD90A79012DDAD11A68A2
:10B6C0000692069D05E01A680792079A521B052A02
:10B6D00046D8C27802F0020202F0FF01002AF2D03E
:10B6E0000223C3702269D378DBB2D9063AD49B0611
:10B6F00034D5B023BEF11F0F93703FD8226904EBFD
:10B700000E0312791A760EF1010E5FFA8EFE16B153
:10B71000236980229A7084F839E0774684E781F8BB
:10B720000280236980229A70774684F839E07BE7AB
:10B7300004EB0E0291F8048082F818800EF1010EDD
:10B740005FFA8EFEB9E781F802C021690846B0E7CA
:10B75000A82191702069BE460279B0E7774663E779
:10B760008170DEE71021A023D170013BFDD1226959
:10B77000937803F0F7037746937055E723691B79B5
:10B78000C5E700BF64A0FF1F0148FFF71FBD00BF52
:10B790007091FF1F0148FFF719BD00BFDC91FF1F2B
:10B7A00000220260704700BF30B5056889B00123F0
:10B7B00000240A460193294602A8009400F006F9E5
:10B7C00002A800F0ADF9C0B209B030BD30B50568CF
:10B7D00089B0012400230A468DE818002946022377
:10B7E00002A800F0F3F802A800F09AF980B209B0BC
:10B7F00030BD00BF0C2901D900207047023149003B
:10B8000001F0FE01FFF7E2BF2DE9F04303688FB0BE
:10B81000012600240D4607461946904633465E220F
:10B8200002A80196009400F0D1F802A800F078F97F
:10B830005E2D03D0A5F17303072B10D8012300243C
:10B84000396801932A4608A8009400F0BFF8224600
:10B85000414608A800F006F90FB0BDE8F083814624
:10B860002246214602A800F0FDF8396833462A46F0
:10B870008DE8500008A800F0A9F82246414608A823
:10B8800000F0F0F822465FFA89F102A800F0EAF829
:10B890000FB0BDE8F08300BFF8B505460F46164669
:10B8A000412421463A462846FFF7AEFF611C023488
:10B8B000C9B232462846E4B2FFF7A6FF592CF0D1B0
:10B8C000F8BD00BF2DE9F843044600689DF82090BC
:10B8D0000E461746984610B1102105F081FB102046
:10B8E00005F07CFB3A460546314600F057F92560E5
:10B8F0002846012100F078F9054618B900252846A8
:10B90000BDE8F883632280212046FFF77DFF0120F8
:10B9100002F032FF00225E212046FFF775FF5D2115
:10B920002046FFF741FF2428E8D14A4641462046F9
:10B93000FFF7B2FF204601222B21FFF765FF2046CB
:10B9400001222C21FFF760FF20460E222D21FFF758
:10B950005BFF204600222E21FFF756FF20460122E2
:10B960002F21FFF751FF204605223021FFF74CFF22
:10B97000204601223121FFF747FF204600223221D5
:10B98000FFF742FF204600223321FFF73DFF20460C
:10B9900000223421FFF738FF204600223521FFF72F
:10B9A00033FF204600225B21FFF72EFF20461022A6
:10B9B0005C21FFF729FF204620225D21FFF724FFAD
:10B9C00020468C225E21FFF71FFF98E770B49DF898
:10B9D00010609DF80C500160002146738573428110
:10B9E00003734161416070BC704700BFF0B543898B
:10B9F000056885B0DCB21B128DF80C408DF80D3057
:10BA00004DB1437B019303AB00932846012300F023
:10BA1000FBF805B0F0BD43680BB31746027A0E463B
:10BA20006AB904F07F048DF80C40427B00923146E5
:10BA30003A46184603AB00F055FA05B0F0BD022AAD
:10BA400004D164F07F048DF80C40EEE7012AECD1BC
:10BA500004F07F0444F040048DF80C40E5E71846FC
:10BA6000D7E700BF02B9027B042A1AD8F0B44161BB
:10BA700000F10F077AB102F10E03867B3C460344C6
:10BA800000F10E055EB92170013BAB424FEA112176
:10BA900004F10104F6D13946F0BCFFF7A7BF1970D5
:10BAA000F2E70020704700BF70B54489066884B093
:10BAB000E5B224128DF80C508DF80D405EB1437B39
:10BAC000009200241A4630460B46019403A900F068
:10BAD0000BF904B070BD4468FCB1037A7BB965F022
:10BAE0007F058DF80C50437B0092FF251A462046B7
:10BAF0000B46019503A900F08BFA04B070BD022B30
:10BB000004D105F07F058DF80C50ECE7012B04BF44
:10BB100065F03F058DF80C50E5E72046D9E700BFFA
:10BB200038B500F10F042146027B0546FFF7BCFF44
:10BB300010B94FF0FF3038BD287B0028FBD00E3005
:10BB40002B18AA7B21460E35002007E01C78013B0C
:10BB5000AB4240EA040001F101010AD00002002AD0
:10BB6000F4D00C78013BAB4240EA040001F1010142
:10BB7000F4D138BD70B5044640681E4603685B6862
:10BB800015469847854201D0002070BD3146606857
:10BB9000FFF762FCB0FA80F0400970BD30B40025B8
:10BBA00020240572C4600170426030BC704700BF41
:10BBB000037A10B5044683B12278636801215200EC
:10BBC00083F83B2083F85E1083F85D106068FFF710
:10BBD00043FCB0FA80F0400910BD012100F004F8E8
:10BBE0000028E9D110BD00BF38B5044640680D46B5
:10BBF000FFF786FA0120207205B938BD2046BDE85E
:10BC00003840FFF7D5BF00BF2DE9F041079EC4685B
:10BC1000DDF818E09519A54219D81546027898461E
:10BC200043680F4652000121044683F83B2083F805
:10BC30005E1083F85D106EB1BEF1000F0AD040684F
:10BC4000036871465B6832469847864202D00020FE
:10BC5000BDE8F08143462A4639462046BDE8F0411A
:10BC6000FFF788BF2DE9F843C468A24202D900203B
:10BC7000BDE8F88316468846074601784068D2B288
:10BC8000FFF774FC8642F2D136B30023DFF85490FC
:10BC90001C4612E090F8383090F839209A4203F1AF
:10BCA000010E00EB03011AD980F838E0087E2870F5
:10BCB0000134A4B2A64223460ED9786802685269BC
:10BCC0004A4508EB0305E5D090470134A4B2C0B261
:10BCD000A64228702346F0D80120BDE8F883FF2053
:10BCE000E5E700BF61B000002DE9F041C568069F9F
:10BCF0009DF81C60AA4202D90020BDE8F08190F8AE
:10BD000000C0D0F804E04FF001084FEA4C0C1D468B
:10BD10008EF83BC033468EF85E808EF85D80044618
:10BD2000FFF728FF0028E7D043463A462946204639
:10BD3000BDE8F041FFF796BF2DE9F04704681346D0
:10BD40000A4624B12046BDE8F04700F035BB057B2C
:10BD50000C7886686249B1FBF6F1002D0CBF4FF0FC
:10BD600001094FF0800919EA040F0CBF4FF0010CD4
:10BD70004FF0000CCDB2002B00F0AF804F0107F464
:10BD8000FF57114602EB030811F801EB4B46002662
:10BD9000002D50D0002F4ED03A46013AFDD1427BC3
:10BDA00012F0F70F40F08D8090F91020013212D080
:10BDB0001EEA030214BF0124002464450BD0002AAC
:10BDC0006CD0446990F8242094F800C04CEA020238
:10BDD00022704FF0010C846990F8262094F800A09E
:10BDE0004AEA020222701DB117B13A46013AFDD16A
:10BDF00090F91120013206D0C26990F825401278DE
:10BE0000224218BF1E43826990F826A0147824EAC3
:10BE10000A04147090F91120013201D001F8016C6C
:10BE2000027B002A35D15B00DBB2002BB0D1884504
:10BE3000AAD1BDE8F087427B12F0F70FB4D0846935
:10BE400090F8262094F800A04AEA0202227090F9A5
:10BE5000102001320AD01EEA030F44692AD090F85C
:10BE6000242094F800A04AEA02022270846990F823
:10BE700026A0227822EA0A02227090F911200132CB
:10BE8000CED0C26990F825401278224218BF1E43D6
:10BE9000C4E75B08002B7FF47BAFC8E7D0F814A0A1
:10BEA00090F824C09AF8004024EA0C048AF8004074
:10BEB000944690E790F824A0227822EA0A022270A1
:10BEC000D4E7846990F8262094F800A04AEA020298
:10BED00022703A46013AFDD1B9E7BDE8F08700BFCC
:10BEE00020A107002DE9F0430C4683B001680A9FAA
:10BEF000064690461D4681B14268CB7A1268002BF7
:10BF00004ED10B68D968914207D039481860394939
:10BF1000DA6042F08040186119600021B07B02F0C5
:10BF2000EFFB77B105EB07090DF1070715F8013BAA
:10BF30008DF80730012239463046FFF7FDFEA9454E
:10BF4000F4D1B8F1000F0ED004EB08050DF107078E
:10BF500014F8013B8DF80730012239463046FFF7CF
:10BF6000EBFEA542F4D10121B07B02F0C9FB33689E
:10BF700093B1DA7A82B1D00703D51F4A996911606B
:10BF8000DA7A910703D51D4AD9691160DA7A520726
:10BF900002D51B4A1B6A1360012003B0BDE8F08381
:10BFA00072B6CB7AD80709D5DFF858E0C868DEF852
:10BFB000003003408B61CEF80030CB7A980709D56A
:10BFC000DFF844E00869DEF800300340CB61CEF8CA
:10BFD0000030CB7A5B0708D5DFF830E04869DEF83F
:10BFE000003003400B62CEF8003062B689E700BF34
:10BFF00001403F0000003F8000E100E004E100E07C
:10C0000008E100E080E100E084E100E088E100E098
:10C010002DE9F0470D4682B00168DDF828909DF8C3
:10C020002C80064617461C4681B14268CB7A1268BE
:10C03000002B4FD10B68D968914207D0394818605E
:10C040003949DA6042F08040186119600021B07B04
:10C0500002F056FB77B105EB070A0DF1070715F85B
:10C06000013B8DF80730012239463046FFF764FE68
:10C07000AA45F4D1B9F1000F0FD0A1440DF1070783
:10C080000122394630468DF80780FFF755FE9DF8AE
:10C09000073004F8013BA145F2D10121B07B02F049
:10C0A0002FFB336893B1DA7A82B1D00703D51F4AE8
:10C0B00099691160DA7A910703D51D4AD96911602F
:10C0C000DA7A520702D51B4A1B6A1360012002B0BC
:10C0D000BDE8F08772B6CB7AD80709D5DFF858E00B
:10C0E000C868DEF8003003408B61CEF80030CB7AB0
:10C0F000980709D5DFF844E00869DEF8003003400E
:10C10000CB61CEF80030CB7A5B0708D5DFF830E0A2
:10C110004869DEF8003003400B62CEF8003062B6AA
:10C1200088E700BF01403F0000003F8000E100E0E1
:10C1300004E100E008E100E080E100E084E100E0EB
:10C1400088E100E02DE9F0410468E56815F0807FA2
:10C15000794D256052D1DF0740F1B380002900F00E
:10C16000E3800D78012B18BF45F000456563013170
:10C1700090F8248003F1FF3C48EA0828BCF1000F46
:10C1800000F0A88021B14D7811F8028B45EA08280B
:10C1900045682E7ABCF1020F06F1FF364FEA0636EB
:10C1A0000CBF48F0805548F01045B6B26563ACF15D
:10C1B000020C08E00AB114700132013B05F470452D
:10C1C000B54216D90468E56A15F0F00FF6D0A46BF5
:10C1D00013F0010F17464FEA242EEBD11AB107F8DE
:10C1E00002EB54703A4605F47045B542A3F10203E0
:10C1F000E8D8BCF1000F6DD00468C3E7DD074CD56B
:10C20000002900F089800D78012B18BF45F000450A
:10C210006563013103F1FF3E90F824C0BEF1000FC9
:10C2200041D029B191F801C00D78023145EA0C2CBA
:10C2300045682E7ABEF1020F06F1FF364FEA063648
:10C240000CBF4CF080554CF01045B6B26563AEF1B2
:10C25000020E08E00AB114700132013B05F470458A
:10C26000B54215D90468E56A15F0F00FF6D013F061
:10C27000010F1746A46BEDD122B107F8024B24122F
:10C2800054703A4605F47045B542A3F10203E9D86B
:10C29000BEF1000F07D00468C3E79E4690F824C0A3
:10C2A000BEF1000FBDD11BB30468E16A11F0F00FBD
:10C2B000FBD0A16BDC071DD50AB111700132013B27
:10C2C000F1E790F824809C4648EA0828BCF1000F6A
:10C2D0007FF458AF63B10468E16A11F0F00FFBD04E
:10C2E000DE07A16B0FD50AB111700132013BF1E7F6
:10C2F000BDE8F0812AB114460D1204F8021B5570F6
:10C300002246023BCFE72AB114460D1204F8025B25
:10C3100051702246023BDDE790F82450012B18BFF4
:10C3200045F00045656375E790F82450012B18BF70
:10C3300045F0004565631BE700041F8090E80C0092
:10C34000F0B41C6859682568164F174E29432160C0
:10C35000164D17491760D66015611160417A154A6C
:10C360005C180A3194F8244053F8215002EBC401C0
:10C3700049680D60017A5C1803EB8101247ECD6968
:10C3800002EBC40149680D60817A581803EB810300
:10C3900090F83000596B02EBC002F0BC5368196092
:10C3A000704700BF01401F000110003801100078E5
:10C3B00000001F80985D01000BB1FFF7C3BE7047FE
:10C3C000704700BFF0B50C1EBDF8146034DBB0F947
:10C3D00006701919B942C4BF3B1B1BB2002BA646FD
:10C3E0001CDD002A1146B8BFD11D02F00705CC1094
:10C3F000826A012007FB04E1A840012E0A44C0B272
:10C400001ED00CD3022E09D1013B12FA83F3013A5C
:10C4100012F8011F41409A421170F9D1F0BDC0439A
:10C42000013B12FA83F3C0B2013A12F8011F014036
:10C4300093421170F9D1F0BD23441BB20024C6E72A
:10C44000013B12FA83F3013A12F8011F01439A42A9
:10C450001170F9D1F0BD00BF00291EDB30B4B0F976
:10C460000A408C4218DD002A16DBB0F90C409442D9
:10C4700012DD047E022C54D0032C4CD0012C06D1AA
:10C480005140C4884A405140013C611A09B2012B15
:10C490002DD017D3022B01D030BC7047002AB0F941
:10C4A0000630856A1446B8BFD41D44F3CF0404FB9C
:10C4B000031102F007026B5C012000FA02F25A40FD
:10C4C0006A54E9E7002AB0F90630856A1446B8BF15
:10C4D000D41D44F3CF0404FB031102F007026B5C8C
:10C4E000012000FA02F223EA02026A54D4E7002A89
:10C4F000B0F90630856A1446B8BFD41D44F3CF04A2
:10C5000004FB031102F007026B5C012000FA02F247
:10C510001A436A54C0E70489013C641A114622B2E6
:10C52000B5E7C5880489013D013C691AA21A09B220
:10C5300012B2ACE72DE9F041079E9DF91880089DE5
:10C5400004461F4600F0BCFF0D4B0E480E4984F810
:10C550003380FF22002F08BF1F4684F82F200023BE
:10C5600084F8302084F8312084F832202060666519
:10C57000A565676221662362A3622046BDE8F0815B
:10C580007091FF1F005301000110013810B50446DF
:10C59000806A034B236008B106F03EF8204610BDC8
:10C5A00000530100F8B5436ADBB190F82C20012557
:10C5B000AA4083F83B2083F85E5083F85D50044620
:10C5C000406A03680E461B6800219847606A03684A
:10C5D00031461B6898472946606ABDE8F840FEF777
:10C5E0003BBFC26BC56C1368046A23EA0503136082
:10C5F0004CB122684FF00043D3625163D36A002BE1
:10C60000FCDA936BF8BD836B466B0825802410E041
:10C610003768426C3A4332601F68826C3A431A6052
:10C620001A68876C013D22EA07024FEA54041A6037
:10C6300007D02142ECD13268476C22EA070232600F
:10C64000EAE7F8BD70B50446406A0D4600282BD0D5
:10C65000616DFEF79FFD002D20460CBFA621A7218E
:10C66000FFF7A0FF606A20B1A16DBDE87040FEF742
:10C6700091BD216C226D0868236A02430A6093B160
:10C68000DA7A82B1D00703D5224A99691160DA7A41
:10C69000910703D5204AD9691160DA7A520702D589
:10C6A0001E4A1B6A136070BD236A002B2BD0D97AF7
:10C6B000226EE1B172B6D97ACE0706D51848D9688C
:10C6C0000668314099610160D97A880706D5154816
:10C6D000196906683140D9610160D97A4E0705D5DC
:10C6E00011485969066831401962016062B61B68D9
:10C6F000D968914207D00D4818600D49DA6042F0C0
:10C70000804018611960226C216D136823EA0103CF
:10C710001360A0E700E100E004E100E008E100E0D0
:10C7200080E100E084E100E088E100E001403F00BA
:10C7300000003F80436A2DE9F04105460E469046D1
:10C74000002B3ED090F82C100124A14083F83B1020
:10C7500083F85E4083F85D40406A036800211B68EF
:10C7600008F1FF379847FFB2B8F1000F23D03744E4
:10C77000A046013E686A16F8011F03681B689847C7
:10C780000134B742A4B216D01F2CF3D90121686A34
:10C79000FEF762FE95F82C206B6A520083F83B206E
:10C7A00083F85E8083F85D80686A036800211B68F7
:10C7B00098470124DEE7686A0121BDE8F041FEF7F1
:10C7C0004BBEC26BC16C136823EA010306EB08047D
:10C7D00013604FF00048A6420ED02B6A16F801EB0A
:10C7E00063B11A68C2F82C80C2F834E0D36A002B17
:10C7F000FCDAA642936BF0D1BDE8F081AB6BD5F8C3
:10C8000034C008208021DCF800206F6C1EEA010F84
:10C8100014BF3A43BA43CCF800201A68AF6C3A43CD
:10C820001A601A68AF6C013822EA07024FEA510118
:10C830001A60E8D1CFE700BF70B50446406A0D46E4
:10C84000002828D0616DFEF7A5FC20462946FFF799
:10C85000A9FE606A20B1A16DBDE87040FEF79ABCE8
:10C86000216C226D0868236A02430A6093B1DA7A68
:10C8700082B1D00703D5234A99691160DA7A91070A
:10C8800003D5214AD9691160DA7A520702D51F4AC5
:10C890001B6A136070BD236A002B2BD0D97A226EDD
:10C8A000E1B172B6D97ACE0706D51948D9680668BB
:10C8B000314099610160D97A880706D51548196910
:10C8C00006683140D9610160D97A4E0705D5124812
:10C8D0005969066831401962016062B61B68D968FF
:10C8E000914207D00D4818600D49DA6042F080404F
:10C8F00018611960226C216D136823EA010313602B
:10C90000A3E700BF00E100E004E100E008E100E08F
:10C9100080E100E084E100E088E100E001403F00C8
:10C9200000003F802DE9F041044686B0806A9DF802
:10C9300030801E460F461546B4F90830002800F036
:10C940004B81DA1D48BF03F10E02B4F90630D21054
:10C9500003FB02F2002106F083F9B4F90820202A33
:10C9600000F3A780B4F90610A74B0120203A7339D1
:10C9700002EBD27201EBD1714FF0200E02907320C6
:10C980008DE8014042F34F0241F34F01204600F091
:10C990004DFE606A84F82D70002800F05181002D52
:10C9A00040F09F80B4F90830202B14BF3D253C2572
:10C9B00084F82C50B8F1000F40F09A8006B394F937
:10C9C0003300002818DBC0B2012101F0ADFE0121C7
:10C9D00094F8330001F094FE012001F0CDFE002117
:10C9E00094F8330001F08CFE0A2001F0C5FE01210D
:10C9F00094F8330001F084FE606A002800F098800B
:10CA0000616DFEF7C7FB042280492046FFF792FEC6
:10CA1000217A0139C9B22046FFF7C4FD7C490422BE
:10CA20002046FFF787FE94F92D30012B14BF142107
:10CA300010212046FFF7B6FD042276492046FFF775
:10CA400079FEB4F906308F22802B84F85C2000F048
:10CA5000A580602B00F0B1800225DA212046FFF787
:10CA6000A1FD29462046FFF79DFD81212046FFF7C5
:10CA700099FD94F85C102046FFF794FDD9212046DB
:10CA8000FFF790FD94F92D30012B14BFF1212221E5
:10CA90002046FFF787FD204606225F49FFF74AFE42
:10CAA000606A58B3A16DFEF775FB012006B0BDE8C2
:10CAB000F081B4F90610594B0120403A52394FF039
:10CAC000400E029002EBD272522001EBD1718DE840
:10CAD000014042F34F0241F34F01204600F0A6FD12
:10CAE00057E76DB284F82C50B8F1000F3FF466AFF1
:10CAF000FEF706FB002E3FF47FAF60E7216C226D4E
:10CB00000868236A02430A6073B1DA7A62B1D00717
:10CB100003D5434A99691160DA7A91076FD45207B5
:10CB200002D5404A1B6A1360012006B0BDE8F081BF
:10CB3000236A002B2BD0D97A226EE1B172B6D97A52
:10CB4000CF0706D53848D968056829409961016042
:10CB5000D97A8E0706D53548196905682940D96103
:10CB60000160D97A4D0705D53148596905682940D2
:10CB70001962016062B61B68D968914207D02D48DE
:10CB800018602D49DA6042F0804018611960226C0B
:10CB9000216D136823EA0103136034E7B4F9083008
:10CBA000402B7FF459AF94F92D30012B14BFCF23C4
:10CBB0009F2384F85C3012254FE7B4F90830102B1E
:10CBC0007FF44AAF94F92D30012B14BFAF2310230B
:10CBD00084F85C30022540E7DA1D48BF03F10E02FD
:10CBE000B4F90630D21003FB02F21046059205F0AC
:10CBF0000BFDA06200283FF459AF059AAAE60F4A40
:10CC0000D9691160DA7A8AE7505301003055010082
:10CC100034550100385501003C55010044550100D0
:10CC200000E100E008E100E080E100E084E100E0F4
:10CC300088E100E001403F0000003F8004E100E0A7
:10CC4000012194F83100214F01F06EFD94F832007B
:10CC5000012101F069FD94F9312094F9323057F83F
:10CC60003220E26357F83330206A23640125E564FB
:10CC700025651A682A431A6048B1B8F1000F3FF4DD
:10CC800039AFFFF75BFB002E3FF4B6AE97E62946BF
:10CC900094F82F0001F048FD294694F8300001F087
:10CCA00043FD94F92F2094F9303057F83220626315
:10CCB00057F833306564A5641A68A36322F0010253
:10CCC0001A60002E3FF498AE79E600BF985D01002F
:10CCD000B0F90820D31D48BF02F10E03B0F90620B9
:10CCE000806ADB1002FB03F2002105F0B9BF00BF30
:10CCF000F0B50029BDF814502EDBB0F90660B14242
:10CD00002ADA002A59DBB0F9087014461C44BC42E8
:10CD1000C4BFBB1A1BB2002B1EDDD2B2D408D0F8A0
:10CD200028E016FB041112F00702DBB20EEB01043F
:10CD300021D0C2F10807FAB2374F9342BF5C0CD240
:10CD4000C3EB020CFF2646FA0CF6012D07EA060794
:10CD50003FD005D3022D36D0F0BD012D39D030D2D1
:10CD60001EF8016026EA07070EF801709342F3D31C
:10CD7000B0F906100C449A1AD2B2072A10D9022D23
:10CD800036D0002D14BFFF26002613462670083B20
:10CD9000B0F90610DBB2072B0C44F7D802F00702FB
:10CDA000002AD9D01D4B012D9B5C1DD017D3022D1D
:10CDB000D2D1227853402370F0BD13441BB200221D
:10CDC000A1E7022D25D11EF8016077400EF8017011
:10CDD000CCE71EF8016037430EF80170C6E72278F1
:10CDE00022EA03032370F0BD227813432370F0BDC1
:10CDF00011462378DB4323700839B0F90630C9B2F5
:10CE000007291C44F5D812F00702A5D0034B9B5C00
:10CE1000CFE73444AFE700BFF0520100E052010019
:10CE200070B4047EBDF80C50022C18D0032C1FD017
:10CE3000012C0BD0002A03DBB0F90840944201DC3E
:10CE400070BC7047039570BCFFF7BCBAC4880395EB
:10CE5000013CA41A0A4621B270BCFFF749BF0689FB
:10CE6000C488013E641AB21AE41A12B221B2E1E790
:10CE700004890395E41A641A114622B270BCFFF7C4
:10CE800037BF00BF70B4057EBDF80C60022D1AD00C
:10CE9000032D12D0012D03D0039670BCFFF728BFDD
:10CEA000C488E41AA41A0A4621B2002A03DBB0F9A6
:10CEB0000840944213DC70BC70470489013C641A3A
:10CEC000114622B2F1E7C48805890396013CAD1AE8
:10CED000ED1A621A11B22AB270BCFFF709BF0396AD
:10CEE00070BCFFF76FBA00BF2DE9F8430446406AF3
:10CEF000002863D0616DFEF74DF905227449204684
:10CF0000FFF718FCA1790139C9B22046FFF74AFBA7
:10CF1000B4F90820E588A66AD31D48BF02F10E03C4
:10CF2000DB10626A15FB03F51FFA85F8002A7BD037
:10CF300094F82C300125AB4082F83B3082F85E50EB
:10CF400082F85D50606A036840211B6808F1FF3772
:10CF50009847BFB2B8F1000F23D03744A846013E2E
:10CF6000606A16F8011F03681B6898470135B742CD
:10CF7000ADB216D01F2DF3D90121606AFEF76CFA0D
:10CF800094F82C20636A520083F83B2083F85E807B
:10CF900083F85D80606A036840211B68984701251B
:10CFA000DEE70121606AFEF757FA606A002800F0A8
:10CFB0008D80A16DBDE8F843FEF7ECB8236A002B25
:10CFC0002BD0D97A226EE1B172B6D97ACE0706D5C6
:10CFD0004048D9680568294099610160D97A8D0770
:10CFE00006D53D48196905682940D9610160D97A9B
:10CFF000480705D539485969056829401962016013
:10D0000062B61B68D968914207D035481860354927
:10D01000DA6042F0804018611960226C216D13685B
:10D0200023EA0103136068E7E26BE36C1168276A87
:10D030000B4306EB080913604FF0004E4E450DD030
:10D0400016F801CB2FB33A68C2F82CE0C2F834C00E
:10D05000D36A002BFCDA4E45936BF1D1226C236D21
:10D0600011680B43136097B1FB7A83B1D90703D5DD
:10D070001D4BBA691A60FB7A9A0703D51B4BFA69F4
:10D080001A60FB7A5B0702D5194B3A6A1A60BDE851
:10D09000F883A36BD4F8348008208021D8F80020CE
:10D0A000656C1CEA010F14BF2A43AA43C8F800208C
:10D0B0001A68A56C2A431A601A68A56C013822EA1E
:10D0C00005024FEA51011A60E8D1B7E7276AC5E7C0
:10D0D000E852010080E100E084E100E088E100E046
:10D0E00001403F0000003F8000E100E004E100E07B
:10D0F00008E100E02DE9F04F85B09946BDF93870A0
:10D10000BDF83CA0BB1AC1EB090B002BB8BF5B42BA
:10D11000BBF1000FB8BFCBF1000B5B450D461646C7
:10D120000093804648DC4D453A4633464CDC194670
:10D1300013460A46C5EB09019B1A89B2002B0CB2B3
:10D14000B8BF5B4204EBD474BE42ACBF4FF0FF32B9
:10D1500001224D45039102924FEA640429DC9BB2FF
:10D1600001930DE0D8F80070BF69B847019BE41A3D
:10D17000A3B21CB20135002C2DB211DBA94518DB7E
:10D18000009B5B452A46534631464046EADCD8F8C8
:10D19000002053469769294632464046B847E5E79E
:10D1A000029A1644039AA94502EB030436B224B24C
:10D1B000E6DA05B0BDE8F08F4A462B46B94635465B
:10D1C0004D4517461E46B2DD304629463E464D4681
:10D1D00007468946AEE700BF10B404682469A44638
:10D1E00010BC604730B40468BDF808500295A46BC9
:10D1F000A44630BC604700BF30B40468BDF8085096
:10D200000295E46BA44630BC604700BF70B404686C
:10D21000BDF90C60BDF8105003960495246CA4462B
:10D2200070BC6047704700BF10B582B0B0F90C20E9
:10D2300001910168009200220C6CB0F90A3011468D
:10D24000A04702B010BD00BF704700BF01F003014E
:10D250000129017606D0032904D0C28803894281BE
:10D26000838170470289C38842818381704700BFF0
:10D270002DE9F0410568134E6F6986B0B742044648
:10D28000BDF8308010D1013B13441BB20093CDF8A0
:10D2900004800B46AD6A2046A8472368DB6AB34288
:10D2A0000AD106B0BDE8F081059304920391B84716
:10D2B00003A925680EC9E6E7204606B0BDE8F0419F
:10D2C000184700BF25D200002DE9F0410568124E35
:10D2D0006F6986B0B7420446BDF830800FD1013B7C
:10D2E000CDF804800B4400921BB2AD6A2046A847DB
:10D2F0002368DB6AB3420AD106B0BDE8F08105932A
:10D3000004920391B84703A925680EC9E7E72046B0
:10D3100006B0BDE8F041184725D200002DE9F04FD6
:10D320000568DFF858B06F6985B05F450646BDF9FE
:10D330003890BDF83CA00C46904615D11F19BC4250
:10D340000CDACDF800A0214601342D6A4B46424646
:10D35000304624B2A847BC423568F2DBEB6A5B4535
:10D3600007D105B0BDE8F08F0393B8473568039B3C
:10D37000E4E7304605B0BDE8F04F184725D200007D
:10D380002DE9F04387B099420546BDF93840BDF814
:10D390003C6025D0A24212D00768DFF88080D7F821
:10D3A0001490C14532D18DE850002846BC6AA04790
:10D3B0002B68DB6A434524D107B0BDE8F08399426E
:10D3C00002DD08461946034628680E96C46B0133F1
:10D3D0005B1A1BB22846A44607B0BDE8F04360477D
:10D3E000A24202DD134622461C4628680E96631CA4
:10D3F000846B9B1A1BB22846A44607B0BDE8F043D5
:10D400006047284607B0BDE8F043184705930492EB
:10D410000391C84703A92F680EC9C4E725D20000AD
:10D420002DE9F04FD0F800E0DFF89090DEF814B06E
:10D4300083B0CB450446BDF93080BDF834A00D461D
:10D4400017461E4631D1CDF800A0DEF824B029469B
:10D4500033463A462046D8472368CDF800A008F165
:10D46000FF323A44D3F824B0294612B2334620465C
:10D47000D8472368CDF800A02946D3F820B03A4613
:10D4800043462046D8472068CDF800A0711E2944A5
:10D490004346056A09B23A462046A8472368DB6A34
:10D4A0004B4506D103B0BDE8F08FD847D4F800E073
:10D4B000C9E7204603B0BDE8F04F184725D2000069
:10D4C000F0B4002401254FF6FF76094F0760047180
:10D4D0000476C48104828476C461C57585754576F9
:10D4E00086824682C180028141818281F0BC704780
:10D4F0000C5801002DE9F04F85B00668BDF8445086
:10D50000BDF93880CDF8008004460195D6F848B0C2
:10D510000392BDF93C60BDF9407089469A46D847F0
:10D5200023680195009742465146D3F8488020462B
:10D530003346C0472068039B0E930F95856C4B467E
:10D540003A4631462046AC4605B0BDE8F04F60474C
:10D550002DE9F04F87B01746BDF9404000912546B0
:10D56000E91D059344BF2B4603F10E010268BDF887
:10D57000486053690294C91003912B49BDF9444096
:10D5800001968B42824645D1002C3CDD029B3C44F7
:10D590005E1EB6B24FF0000923B2049301364D4629
:10D5A000029B002B28DD059B002403EB090806E005
:10D5B000EDB22B0604F1010411D4A6421CD0A1B295
:10D5C00011F0070F23B24FEA4505F1D1002BB8BF88
:10D5D0000733DB10013418F803502B06EDD5009B00
:10D5E000D2F818B019443A4609B2019B5046D847C0
:10D5F000A642DAF80020E2D1039B01379944049B4C
:10D600003FB2BB42CCD1D36A074A934206D107B09E
:10D61000BDE8F08F9847DAF80020B5E7504607B02C
:10D62000BDE8F04F184700BF25D2000070B4BDF927
:10D630000C60BDF91050BDF8144003960495059494
:10D6400070BCFFF785BF00BF2DE9F04F91B0834656
:10D650000591C169BDF8680006909DF87400BDF899
:10D660006C709DF870A0039002929946002900F01A
:10D67000CC800B7A48680A68C3EB0903DBB2154615
:10D6800000EBC30230F83360D3780993BAF1010F8D
:10D6900092F9053092F802800E9392F9064079D9FA
:10D6A000BDF93830089323B20B93A94BDBF8002067
:10D6B0000F93194653698B4240F0A280099B002BBF
:10D6C00053D0BDF808300C930021234407910D93EB
:10D6D0000F460C46A946B8F1000F3FD0BDF81C100C
:10D6E0000B9BBDF80C000297CB1813FB00F30C98B2
:10D6F00003440D981BB2014404930BB20A93002516
:10D7000005E00135EBB264009845E4B223D9029BF1
:10D710002B44590703D1731C19F806409EB2230607
:10D72000EFD5089BE918059B11FB0AF1BAF1010F2F
:10D73000194402D1039B012B1ED0069B0193039B2E
:10D740000093D369049A1F4609B253465846B84716
:10D75000DBF80020D5E7029F4744FFB2079B0999F9
:10D7600001330793DBB29942B5D8D36A0F9A93423B
:10D7700041D111B0BDE8F08F0E9B059959189369FE
:10D780000A9A29441F4609B2069B5846B847DBF857
:10D790000020B6E7039B012B82D800230B9308934C
:10D7A00083E70799099A0131013A49B212F0FF0261
:10D7B0000791099260D1069A4A454F4617D0BAF1AF
:10D7C000010F03D1039A012A00F0B5800A9A089844
:10D7D00002EB8201039AD2008DE88400084401B272
:10D7E000DC69029A53465846A047DBF80030DB6AF2
:10D7F0000F9A9342BDD0584611B0BDE8F04F18477C
:10D8000058469847DBF8002058E7BBF90A300599DD
:10D810008B42AEDDBBF90C3002988342A9DD0623B2
:10D8200013FB0A13002BA4DD039B00EBC303002BA7
:10D830009FDD9BF81A3033B9B9F1AF0F84BF09F1FE
:10D8400001035FFA83F9424ADBF800300F92114678
:10D850005A698A426AD1BDF81420089205220992B9
:10D86000002207921FFA8AF20A92CDF830900FFA3E
:10D870008AF2B946039F05920799BDF83040089D8A
:10D880000522104610FB04120A98324C0646084640
:10D8900001FB0651A65C15FA80F209B212B204919E
:10D8A0000B92082400251CE0BAF1010F01D1012FD1
:10D8B00024D0069A0192029A009705FB0722D3F81A
:10D8C0001C800499059B12B25846C047DBF8003013
:10D8D000013C013514F0FF046DB24FEA56063FF4E7
:10D8E00060AFF007E0D4069A4A45F1D0BAF1010FD3
:10D8F00001D1012F0ED0CDF80490DCE7029AD3F8C5
:10D9000018800B99069BAA1812B25846C047DBF83C
:10D910000030DDE7029AD3F818800B99AA184B461D
:10D9200012B25846C047DBF80030D1E7584690475E
:10D93000DBF800308FE70899CDF8009005311C6ABC
:10D94000029A082309B25846A047DBF800304EE798
:10D9500025D200005C580100F0B5C36985B00446CB
:10D960003BB30A296FD00D294FD01A7A91424CD37C
:10D97000987A884249D38A1A5D68D2B205EBC2050B
:10D98000AA78002A56D0E878002853D0607E002874
:10D990003ED095F905E0B4F90E00A67DB4F90A7001
:10D9A000724406FB0202BA4269DCE77DB4F910203A
:10D9B00034E00A295CD00D2927D0427E002A50D0BD
:10D9C000B0F90E00A57DB4F90A60062212FB05022B
:10D9D000B242E67D42DD228AE38102EBC60212B248
:10D9E00018462282B4F814E0678A03960B46029523
:10D9F00001468DE880402046FFF726FEA37DE289A0
:10DA000003EB430302EB4303E381012005B0F0BDC8
:10DA1000A67DE77DB4F90E00B4F91020B4F814E047
:10DA20000397678A02960B468DE8804001462046A0
:10DA3000FFF70AFE2979E389A27D012001FB023369
:10DA4000E38105B0F0BD0022C2811A7BC17D038A4B
:10DA500001FB02330382012005B0F0BDB4F91020B0
:10DA6000C0E7857DC67DB4F91020B0F90E00B9E796
:10DA7000028AC17DC38102EBC1030382C5E7002096
:10DA8000E0811B7B228AE77D03FB072212B2228200
:10DA9000C4E700BF11B18175C1757047012181755F
:10DAA000C1757047844641EA000313F003036DD14A
:10DAB000403A41D351F8043B40F8043B51F8043B51
:10DAC00040F8043B51F8043B40F8043B51F8043B58
:10DAD00040F8043B51F8043B40F8043B51F8043B48
:10DAE00040F8043B51F8043B40F8043B51F8043B38
:10DAF00040F8043B51F8043B40F8043B51F8043B28
:10DB000040F8043B51F8043B40F8043B51F8043B17
:10DB100040F8043B51F8043B40F8043B51F8043B07
:10DB200040F8043B51F8043B40F8043B51F8043BF7
:10DB300040F8043B403ABDD2303211D351F8043B97
:10DB400040F8043B51F8043B40F8043B51F8043BD7
:10DB500040F8043B51F8043B40F8043B103AEDD246
:10DB60000C3205D351F8043B40F8043B043AF9D297
:10DB7000043208D0D2071CBF11F8013B00F8013B6A
:10DB800001D30B8803806046704700BF082A13D377
:10DB90008B078DD010F003038AD0C3F10403D21A8F
:10DBA000DB071CBF11F8013B00F8013B80D331F8C3
:10DBB000023B20F8023B7BE7043AD9D3013A11F843
:10DBC000013B00F8013BF9D20B7803704B784370AE
:10DBD0008B78837060467047374A384913681B0654
:10DBE000FCD40B6813F08003F8D172B634490A787C
:10DBF000002A5FD0334A3448F0B4344C17680668C2
:10DC00002568D4680C303E44143200681268304FE6
:10DC100035442C4420440244C2F34E022D4E2E487B
:10DC20002E4D2F4C42F400423A60376806682D684A
:10DC30002C4A24680C303E44006812682A4F354450
:10DC40002C4420440244C2F34E02284E2848294D59
:10DC5000294C42F400423A60376806682D68274A2A
:10DC600024680C303E4400681268254F35442C442B
:10DC700020440244C2F34E02224E2348234D244C3A
:10DC800042F400423A60376806682D68214A2468E9
:10DC90000C303E440068126835442C442044024451
:10DCA000C2F34E021C4842F4004202600B7062B69E
:10DCB000F0BC704762B6704724B0034024B00B40FC
:10DCC0005EA0FF1F38B003403CB0034040B00340AB
:10DCD0002CB0034058B003405CB0034060B0034038
:10DCE00064B003406CB0034030B0034038B00B4028
:10DCF0003CB00B4040B00B4044B00B404CB00B402C
:10DD00002CB00B4058B00B405CB00B4060B00B40E7
:10DD100064B00B406CB00B4030B00B4030B42948BD
:10DD2000294A2A4B2A4D6024E121047011701B7886
:10DD3000284C082B30D00A2B2748284937D00C2BE9
:10DD40000CBF35223D2212232A60236002600B6043
:10DD5000234B24491B78244ABBB101230B60136079
:10DD6000224B23491B78234A012B26D9042B0FD998
:10DD7000082B1ED9102B94BF862387230B601360BA
:10DD80001D4B01221A7030BC70470B601360E7E72F
:10DD900084230B601360F3E700F58E200F490830F1
:10DDA000012213232A60236002600B60D0E739222E
:10DDB000F7E785230B601360E2E780230B601360B5
:10DDC000DEE700BF00400740014007404892FF1FC8
:10DDD00008B003400CB0034008B00B400CB00B403F
:10DDE00061A0FF1F20B0034020B00B404992FF1FED
:10DDF00024B0034024B00B405EA0FF1F0C2830B4B9
:10DE000017D91023984228BF18461C46104A114DB6
:10DE10001178181A8C42287018D00F4913700B789B
:10DE200023B10E490E4A00230B60136030BCFFF78C
:10DE300075BF0A2802D90C231C46E7E7082802D937
:10DE40000A231C46E2E708231C46DFE730BC704784
:10DE50004892FF1F5DA0FF1F5EA0FF1F24B003407C
:10DE600024B00B4028282FD8334B2DE9F0411E5CFD
:10DE7000FF2E2BD0314B1B78002B2AD132062CD40D
:10DE800072B62F4D2F4C2F46012326602B7062B6A1
:10DE900072B623681B060CD43B781BB9F4E72B78C9
:10DEA000002BF1D062B603F0A1F872B62368180611
:10DEB000F5D5254B1B6800222A7062B6234A1078DC
:10DEC00043FA00F0BDE8F081002070470020BDE873
:10DED000F081FFF781FE3206D2D572B61C4DDFF815
:10DEE0007C801C4C06F04007FFB206F03F06D8F8D5
:10DEF0000030DFB123F01003C8F8003001232660A2
:10DF0000134A2B7062B672B6236819060CD41378C4
:10DF10001BB9ECE72B78002BE9D062B603F066F86A
:10DF200072B623681B06F5D50B4BC3E743F010030D
:10DF3000C8F80030E2E700BF5C5D01005EA0FF1F93
:10DF400060A0FF1F00B0034010B003405DA0FF1FA2
:10DF50005FA0FF1F00B00B4010B00B400CB00B4097
:10DF60000A4A0B49136843F4805313600B7843B992
:10DF7000084BC0221A70084B80F30C0000B21880C6
:10DF80007047044B80221A70F5E700BF2C800440D4
:10DF900061A0FF1F21C00C4000C00C40F0B51B4B1E
:10DFA0001B4E596818689A68DB6885B06C460FC4C8
:10DFB000337899071DD5174A174C1378174913F072
:10DFC000700318BF1370164A164B8027177000266F
:10DFD0003320032226706D4608701A7072B6043C16
:10DFE00045F001052046A84762B6237813F0700378
:10DFF00009D10D4B064901E0013B02D00A78D20756
:10E00000FAD505B0F0BD237005B0F0BD885D010004
:10E010000100024000000240040002400B000240E8
:10E02000070002400A000240410D0300B0F5006FF6
:10E030000AD210B5094B1B78DB07044606D504F15C
:10E04000A0500078C0B210BD00207047FFF7A6FFB7
:10E0500004F1A0500078C0B210BD00BF0100024022
:10E06000B0F5006F17D238B50F4B1B78DA070D46A5
:10E07000044611D504F1A0500378AB420AD00B4AF4
:10E08000137813F0700318BF1370074A05701378E4
:10E09000DB07FCD538BD7047FFF780FF04F1A050C7
:10E0A0000378AB42EBD1F5E70100024000000240EB
:10E0B00008B5104C08E0236859050DD423681A05EB
:10E0C0000FD42368DB0411D423685803F3D501F07F
:10E0D00087FB23685905F1D500F00EF823681A056F
:10E0E000EFD500F02DFF2368DB04EDD501F0EAF950
:10E0F000EAE700BF3480044008B5FFF7D9FF00BF4E
:10E10000014B10221A80704700200540704700BF65
:10E11000094908B50B6830B16A461844A2F5805227
:10E12000904202D20860184608BD04F03FFA0C2362
:10E1300003604FF0FF3008BD4C92FF1FFEE700BFA9
:10E14000EFF3138070B9EFF310836BB9EFF305822F
:10E150005AB94FF48070EFF311832BB1984228BF66
:10E16000184670474FF0FF3070470F2A01D8184605
:10E17000F1E7014BD05CEEE7F0E300E0704700BF51
:10E1800010B40F4B53F8302092F880422CB1012389
:10E1900069B182F8803010BC704703EBC0035B6844
:10E1A0001A6841B922F002021A6010BC704782F866
:10E1B000003110BC704742F003021A6010BC704777
:10E1C000985D01001C4A02EBC00301295B6811D075
:10E1D00004291BD052F83000002280F8802229B197
:10E1E000022920D0032922D01A6070474FF4807290
:10E1F0001A60704752F830004FF4A27280F8801213
:10E200001A601A6822F020021A60704752F8301023
:10E210004FF4A272012081F880021A601A6842F05D
:10E2200020021A60704740F203121A6070474FF4E0
:10E2300081721A60704700BF985D0100212848D89C
:10E24000F8B5042A44D8DFE802F0484B4E034500F5
:10E250004FF410262B4B03EBC0030D465C6821687E
:10E2600011F4E06148D0284B284A2949C3F89C2181
:10E2700004F140422748C3F8A411A2F59221264F89
:10E28000C3F8A0017C292548C3F8A871C3F8AC01E4
:10E290002CD9A2F594237C2B2AD9A2F596237C2B8A
:10E2A00028D9A2F598237C2B29D9A2F59A227C2A79
:10E2B00027D81B4872B6236823F4702343F080727A
:10E2C000C4F384011643236040F82150266062B6EF
:10E2D000F8BD70474FF43026BCE74FF40026B9E78D
:10E2E0004FF44026B6E74FF42026B3E70D48E1E7A8
:10E2F0000D48DFE70D48DDE7FFF764FFB3E70C48A3
:10E30000D8E7F8BD985D01000082FF1FF188FF1F6C
:10E310009988FF1FC588FF1F6D88FF1F4188FF1F59
:10E320002893FF1F5092FF1F8892FF1FD892FF1F54
:10E330000893FF1F1A4B03EBC00010B4426802F1B0
:10E340004043A3F592217C2923D9A3F594217C296C
:10E350000DD9A3F596217C291FD9A3F598217C29F5
:10E3600019D9A3F59A237C2B11D80E4C00E00E4C42
:10E3700072B613680D4823F08773C2F3840123F447
:10E38000803343F08073136044F8210062B610BC00
:10E390007047074CECE7074CEAE7074CE8E700BF9B
:10E3A000985D01002893FF1F8892FF1F7DE1000008
:10E3B0005092FF1F0893FF1FD892FF1F30B4054BE8
:10E3C000054D064C002210211A602A602060196059
:10E3D00030BC704714D0034004D0034000D0034049
:10E3E000282838B52ED0002904464FDD5F4B1B7816
:10E3F000012505FA03F28A4202D8212837D938BD0F
:10E400000338C2B2012A3AD9202C4AD0192C48D05C
:10E41000574A126802FB011222FA03F31D2800F288
:10E420009B80DFE800F0928B847D9999766F9999B3
:10E430009999999999999968615A53994C99999987
:10E4400099999945494B1B780B2B08D90C2B1CBF6C
:10E450000C3B19410846BDE83840FFF781BDC3F1C8
:10E460000C0399400846BDE83840FFF779BD2946BE
:10E47000FFF786FE2946BDE83840FFF7A3BE3D4AB8
:10E48000126802FB011222FA03F3C7E72128B6D86B
:10E490000021FFF775FE20460121BDE83840FFF757
:10E4A00091BE354A126802FB011222FA03F3B5E766
:10E4B0003249334A0B604FF45173136038BD314910
:10E4C000314A0B604FF45173136038BD2F49304A05
:10E4D0000B6040F24443136038BD2E492E4A0B6056
:10E4E00040F24443136038BD2C492D4A0B6040F282
:10E4F0004443136038BD2B492B4A0B6040F2444320
:10E50000136038BD29492A4A0B6040F24443136026
:10E5100038BD2849284A0B6040F24443136038BD97
:10E520002649274A0B6040F24443136038BD254911
:10E53000254A0B6040F24443136038BD2349244A06
:10E540000B604FF45173136038BD2249224A0B60AF
:10E550004FF45173136038BD212C3FF650AF7F2923
:10E56000D4BF00210121204693E700BF3093FF1F55
:10E57000088003400890034008800B4010800B4047
:10E5800048A0044018800B404CA004401880034071
:10E5900008B004401080034004B0044040800340B1
:10E5A00018C004403880034014C004402880034051
:10E5B00010B00440208003400CB004403080034081
:10E5C00010C00440488003401CC004401890034021
:10E5D00034900440109003403090044038B110282B
:10E5E00028BF1020044AC3B2107813707047024A43
:10E5F00001231078137070473093FF1F2DE9F84303
:10E600000E4680463249334D304603F05BFF47F6F5
:10E61000122300281ABF1D464FF002094FF00109CE
:10E62000002425FA04F003F057FD4FF05E51074631
:10E6300003F0AAFD0146304603F058FF30B901341B
:10E64000072CEED1E80903F047FD0746314638466E
:10E6500003F04EFE4FF07C5103F08CFC03F080FF82
:10E660004FF6FF729042A8F1030328BF1046012B1A
:10E6700029D9B8F1170F17D8174B23FA08F303F06D
:10E68000010383F0010223B9B8F1190F0FD0BDE8DF
:10E69000F883124B124D13491A6044EAC9042A60E8
:10E6A00008601C60BDE8F883B8F1200FECD10E4B78
:10E6B0000E4D0F49002244EAC9041A602A6008601E
:10E6C0001C60BDE8F8830B4B0B4D0C49F2E700BF13
:10E6D000001BB740006CDC026006F00000800340C5
:10E6E000048003400880034000800B4004800B40FE
:10E6F00008800B40009003400490034008900340C2
:10E70000212801D8FFF73CBD704700BF212806D85B
:10E71000044B53F8303093F80002C0B27047002029
:10E72000704700BF985D0100212801D8FFF74ABD5E
:10E73000704700BF72B60C490C4B0D4A1B68086845
:10E74000126862B6520102D5322B88BF01300949E6
:10E75000C3F5BB334FF47A72FF33A1FB031302FB03
:10E7600000F000EB9310704764A0FF1F18E000E07A
:10E7700004ED00E0ABAAAAAA2DE9F843054672B65B
:10E78000204F214B214A1B683C68126862B6520137
:10E7900002D5322B88BF013495B3C3F5BB331C4E71
:10E7A000DFF86490DFF86480FF334FF47A72A6FBE1
:10E7B000031302FB04F404EB931472B6D9F80010AF
:10E7C0003A68D8F800E062B6C1F5BB33FF33A6FB68
:10E7D00003031EF0806FC4EB93134FF47A7002D0E2
:10E7E000322988BF013200FB0233B3F57A7F04D3AC
:10E7F000013D05D004F57A74DFE702F0F7FBDCE7B2
:10E80000BDE8F88364A0FF1F18E000E004ED00E01D
:10E81000ABAAAAAAF8B52D4B2D49DFF8D0E0DFF856
:10E82000D0C02C4E2C4D2D4C2D4A2E4F4FF40000B5
:10E8300018604FF0807018604FF0007018604FF053
:10E84000806018604FF00060186000200860282386
:10E850004BF6FF71CCF80010CEF800303360136037
:10E860002B6023603B60B3629362092245F8242C3D
:10E87000C4F8D80F05F57F65C7F8D41F07F5FF2743
:10E8800007F5FA67C6F8F83F2B6006F5FF26C4F8CF
:10E89000D42F05F5FD2504F5FF24386006F2F47643
:10E8A0001148316005F5FF6504F5FD642B602360B8
:10E8B0000260FFF733FA1920FFF75EFF01F0F6FC64
:10E8C00040F21310BDE8F840FFF756BF08E100E042
:10E8D0000480034014800340248003402C800340C4
:10E8E0001C8003403480034000800B400C800340B8
:10E8F000088003402B4A2C491368F0B543F40063A9
:10E9000013600A78294F2A4E2A4D2B4C2B4900239D
:10E91000092A3B7033702B7023700B703DD01A2A7C
:10E9200021D0274B1B780A2B25D01F2B30D01F2836
:10E9300027D8002002460125224B234C1A70234978
:10E940005D7004224FF0020E88273C264025987205
:10E950009A704FF4004083F813E05A751F74DE700C
:10E9600025700860F0BD1A4B40F213321A60144B48
:10E970001B780A2BD9D1174B4FF451721F281A60FC
:10E98000D7D9C0F34432C0F3471500F01F00D3E7D6
:10E99000114B4FF451721A60C9E7104B40F2133219
:10E9A0001A60BEE7348004403193FF1FD8A0FF1FD8
:10E9B0006DA0FF1FE0A0FF1FD9A0FF1F6CA0FF1FCD
:10E9C0003293FF1F00B006402FE400E004E100E0B6
:10E9D00004D0044010B0044000D004400CB0044007
:10E9E000144B14499B7803F0EC0200F0030313432B
:10E9F000420700F00F0248BF43F01003042A8B7057
:10EA000013D00C4B0B4A5B79C10603F0EF0348BFF0
:10EA100043F0100353719379820603F0EF03054A24
:10EA200048BF43F01003937170478B7943F0400364
:10EA30008B71E6E700B00640234B1B681B0542D5EF
:10EA400010B5224C237823B102F0D0FA2378002BA2
:10EA5000FAD11F481F4A204B4FF4004400210460A4
:10EA6000D1701B78092B1FD01A2B03D11B4B40F2FE
:10EA700003121A601A4B1B7803F07F030A2B1DD078
:10EA80001F2B03D1174B40F203121A60164A114B89
:10EA90001648174912681C79DB79002303700B7044
:10EAA0000AB10123137010BD124B40F203121A6019
:10EAB0000B4B1B7803F07F030A2BE1D10E4B40F286
:10EAC00003121A60E2E77047348004406CA0FF1F15
:10EAD00084E100E000B006403193FF1F04D0044001
:10EAE0003293FF1F00D0044068A0FF1FD8A0FF1F73
:10EAF0006DA0FF1F0CB0044010B004400A4A38B5A6
:10EB00000546137803F0FF04002BFAD101212846B3
:10EB1000FFF70AFE21462846FFF7F2FD034A044BA1
:10EB200052F835201A6038BD6CA0FF1F985D0100B7
:10EB3000DCA0FF1F09B140F08000174A137898420B
:10EB400016D010B4154C246824050FD503F07F03AC
:10EB50000A2B1CD01F2B11D0002900F07F0114BFFD
:10EB6000602344230A290DD01F2902D0107010BC45
:10EB700070470B4943F440730B60F7E7084B0024E0
:10EB80001C60E9E7074943F440730B60EEE7054B6F
:10EB900000241C60E0E700BF3293FF1F3480044074
:10EBA00000D0044010B00440124B1A7882420CD0BE
:10EBB00011490968090507D5092A16D01A2A0AD069
:10EBC00009280DD01A2801D0187070470B4A40F25E
:10EBD00013311160F8E7094A002109281160F1D1C9
:10EBE000074A40F213311160EEE7054A0021116037
:10EBF000E6E700BF3193FF1F3480044004D0044097
:10EC00000CB004400D4B1B6813F4006305D02128A1
:10EC100005D90B4B00201860704718467047094B08
:10EC200010B5074C53F8303023600121FFF77CFD0D
:10EC3000236800221A70012010BD00BF34800440F8
:10EC400068A0FF1F985D01000C4B1B6813F4006364
:10EC500006D0172806D00A4A537B03F0FE035373ED
:10EC600000207047074B064A40F202311960537B7F
:10EC700043F0010353730120704700BF3480044008
:10EC800000B0064008B004402DE9F84F234B1B6844
:10EC90001A053BD5224B1B680BB101221A70DFF815
:10ECA0009090204D99F80040DFF888801E4E013486
:10ECB000272C8ABF4FF0000A5FFA84FA54460746B1
:10ECC000AB462B789C4216D1FFF73AFA40281FDC5E
:10ECD00033791B06F5D59BF800300133272B86BF0F
:10ECE00000221346DAB218F80330DBB2F3712A704F
:10ECF0002B789C42E8D00D490B4BFFB20120BC227F
:10ED000008F80470087089F800A0DA70BDE8F88F80
:10ED1000FF28D6DD02F06AF9D3E700BF3480044053
:10ED2000DCA0FF1FD9A0FF1F00B006406CA0FF1F92
:10ED3000E0A0FF1F70A0FF1F2DE9F84F294B1B68B3
:10ED40001A0548D5284B1B6805460BB101221A70DD
:10ED500005EB010A554540D2DFF89C80234CDFF8D3
:10ED60009C90234F0AE015F8012B09F80B20214A4B
:10ED70000123AA45137088F800602ED098F800305F
:10ED8000227803F1010BBBF1270F86BF0026B346A3
:10ED90005FFA8BF69345E6D1BC22FA7005E03A792A
:10EDA00013060BD422789345DDD1FFF7C9F940282B
:10EDB000F5DDFF28F6DD02F019F9F3E722780132DC
:10EDC000272A86BF00210A46D1B219F80220D2B202
:10EDD000FA712170E6E7BDE8F88F054BBC22DA70C6
:10EDE000BDE8F88F34800440DCA0FF1FD9A0FF1FCE
:10EDF00000B006406CA0FF1FE0A0FF1F70A0FF1F27
:10EE000010B5044C237823B102F0F0F82378002BDE
:10EE1000FAD110BD6CA0FF1F064A074B1B78107873
:10EE2000DBB2C0B283422CBF273000F1FF30C01AE2
:10EE3000704700BFD9A0FF1FE0A0FF1F054A064B87
:10EE400010781B78C0B2DBB2984238BF4030C01A8D
:10EE5000704700BFD8A0FF1F6DA0FF1F30B4154B37
:10EE6000154C1A782378D2B2DBB29A421ED0013305
:10EE70003F2B0ED91149124B087819680023C0B2F4
:10EE8000237021B1D31A1A2B01DC00230B7030BC84
:10EE900070470A480A49C05C0968DDB2C0B22570F3
:10EEA0000029F4D09A4238BF4032EBE74FF0FF30F0
:10EEB000EDE700BFD8A0FF1F6DA0FF1F98A0FF1FA8
:10EEC00068A0FF1F084A094B12781B78DBB29A42F0
:10EED00007D00133402B28BF0023054AD05CC0B2C5
:10EEE00070474FF0FF307047D8A0FF1F6DA0FF1F85
:10EEF00098A0FF1F0D4B1B681B0516D530B40C4B9B
:10EF00000C4CDA780C480D4902F0CB024025DA703F
:10EF10005D74DA7842F03402DA7023780268DBB28A
:10EF20000B700AB10023137030BC7047348004406A
:10EF300000B006406DA0FF1F68A0FF1FD8A0FF1FF4
:10EF4000F0B4384B1A7912F0300F2CD072B6997D8C
:10EF500001F0FF0200293DD062B6334F33493878C3
:10EF60000D78334E1C46C0B2EDB2431C402BE17904
:10EF700028BF0023AB4202F1FF32C9B21CBFF154DB
:10EF8000184612F0FF02F0D12A4B1B68C2B23A7049
:10EF90004BB1A84236BFC5F14005401B4019272898
:10EFA000C4BF01221A701F49CA78D2B2150616D4FE
:10EFB00052060DD51B4B1B795B0609D51E4B1F490D
:10EFC0001B6800220A7003B11A70164B3C22DA70DB
:10EFD000F0BC70474022D9795A7462B6E3E70B79E6
:10EFE0001C06E5D5164B174E1C783378E4B2DBB21D
:10EFF0009C420ED0144D01E0A3420AD00133282BCD
:10F0000028BF00230879E85CC0B2C871087D0728D2
:10F01000F2D9DBB2034933700B79180644BF7C2365
:10F02000CB70C5E700B00640D8A0FF1F6DA0FF1F42
:10F0300098A0FF1F68A0FF1FDCA0FF1F6CA0FF1F90
:10F04000E0A0FF1FD9A0FF1F70A0FF1F2DE9F84F00
:10F05000214B1B6807460BB101221A70DFF888901C
:10F060001E4D99F80040DFF884801D4E0134272C96
:10F070008ABF4FF0000A5FFA84FA5446AB462B78F9
:10F08000A34216D1FFF75CF840281FDC33791B063A
:10F09000F5D59BF800300133272B86BF002213469D
:10F0A000DAB218F80330DBB2F3712A702B78A3427E
:10F0B000E8D00C490A4BFFB208F804700120AC22DA
:10F0C000087089F800A0DA70BDE8F88FFF28D6DD57
:10F0D00001F08CFFD3E700BF58A1FF1F55A1FF1F10
:10F0E00000C0064054A1FF1F5CA1FF1FECA0FF1F42
:10F0F0001C4BDFF894C01A681B49F0B542F48052EB
:10F100001A4D1A60DFF884E0194F1A4E1A4C00238A
:10F110008CF800304FF451722B701F2840F21335D9
:10F120008EF800303B70337025600A6012D81946A3
:10F130000124124A124D11701248547000212C27DC
:10F14000402693724FF4003491701174D7702E7072
:10F150000460F0BDC0F34431C0F3471400F01F0356
:10F16000E7E700BF348004400CC00440E9A0FF1F63
:10F1700055A1FF1F54A1FF1F08C0044000C0064056
:10F1800031E400E004E100E0E8A0FF1F5CA1FF1F04
:10F19000144B14499B7803F0EC0200F00303134373
:10F1A000420700F00F0248BF43F01003042A8B709F
:10F1B00013D00C4B0B4A5B79C10603F0EF0348BF39
:10F1C00043F0100353719379820603F0EF03054A6D
:10F1D00048BF43F01003937170478B7943F04003AD
:10F1E0008B71E6E700C00640F8B5134B1B68DB04E3
:10F1F0001FD5124C237823B101F0F8FE2378002BA1
:10F20000FAD10F4B0F4A104D104F114E114C1248AE
:10F210004FF4003119600023D37040F203113960BC
:10F22000316029681579D2792370037011B10123F7
:10F230000B70F8BDF8BD00BF3480044054A1FF1F1F
:10F2400084E100E000C00640E4A0FF1F08C00440C5
:10F250000CC00440E8A0FF1FE9A0FF1F0A4A38B510
:10F260000546137803F0FF04002BFAD1012128464C
:10F27000FFF75AFA21462846FFF742FA034A044BA1
:10F2800052F835201A6038BD54A1FF1F985D010067
:10F2900058A1FF1F09B140F080000F4A137898422F
:10F2A00019D010B40D4C2468E40412D503F07F0388
:10F2B000082B02D10A4B00241C60002900F07F03B8
:10F2C00014BF60214421082B03D1054B41F4407148
:10F2D0001960107010BC70473393FF1F34800440D6
:10F2E0000CC00440704700BF0D4B1B6813F48053E3
:10F2F00005D0212805D90B4B00201860704718460F
:10F300007047094B10B5074C53F83030236001218A
:10F31000FFF70AFA236800221A70012010BD00BF0F
:10F3200034800440E4A0FF1F985D01000C4B1B6873
:10F3300013F4805306D00E2806D00A4A537B03F0FC
:10F34000FE03537300207047074B064A40F2023118
:10F350001960537B43F0010353730120704700BFD2
:10F360003480044000C0064004C00440034B1B68C6
:10F37000DB0401D5FFF76ABE704700BF348004404C
:10F3800070B5094E04464518AC4204F101040AD098
:10F390003368DB04F8D514F8010CFFF757FEAC42D4
:10F3A00004F10104F4D170BD3480044010B5044C64
:10F3B000237823B101F01AFE2378002BFAD110BD77
:10F3C00054A1FF1F064A074B1B781078DBB2C0B26E
:10F3D00083422CBF273000F1FF30C01A704700BFB6
:10F3E00055A1FF1F5CA1FF1F054A064B10781B7833
:10F3F000C0B2DBB2984238BF4030C01A704700BF7D
:10F40000E8A0FF1FE9A0FF1F30B4154B154C1A7878
:10F410002378D2B2DBB29A421ED001333F2B0ED9F1
:10F420001149124B087819680023C0B2237021B12A
:10F43000D31A1A2B01DC00230B7030BC70470A482A
:10F440000A49C05C0968DDB2C0B225700029F4D059
:10F450009A4238BF4032EBE74FF0FF30EDE700BF94
:10F46000E8A0FF1FE9A0FF1F14A1FF1FE4A0FF1FDA
:10F47000084A094B12781B78DBB29A4207D0013355
:10F48000402B28BF0023054AD05CC0B270474FF024
:10F49000FF307047E8A0FF1FE9A0FF1F14A1FF1F66
:10F4A000054B064A1B7806491268DBB20B700AB19D
:10F4B00000231370704700BFE9A0FF1FE4A0FF1FE7
:10F4C000E8A0FF1F30B42B4B1A7994061FD52A48A9
:10F4D000DA790378294901333F2B0978C8BF002323
:10F4E0008B42D2B203D0264CD9B2E2540170254AE5
:10F4F000116861B1244A1278D2B2934236BFC2F188
:10F5000040029B1A9B18272BC4BF01230B70194A7A
:10F51000D378DBB2180611D45A060DD5154B1B79DA
:10F520005B0609D5194B1A491B6800220A7003B102
:10F530001A70104B2C22DA7030BC70471179090612
:10F54000EAD5144910480C780178C9B28C420DD024
:10F550004A1C272A84BF00210A460F4D054C98BF3C
:10F56000D1B2AA5CD2B2E2710170D5E76C21D17040
:10F57000D2E700BF00C00640E8A0FF1FE9A0FF1FC0
:10F5800014A1FF1FE4A0FF1F55A1FF1F58A1FF1FDB
:10F5900054A1FF1F5CA1FF1FECA0FF1F21282FD843
:10F5A000184B195CFF292BD0174B184ADFF870C095
:10F5B00003EBC000F0B54368DFF868E0144F154D69
:10F5C000154E00241C60DEF80030012043F02003BB
:10F5D0008840CEF8003014604FF4A07338602E607D
:10F5E000C2F800C0013BFDD113689B05FCD4202369
:10F5F000013BFDD1094B09B233F8110080B2F0BDD7
:10F6000000207047A85E0100985D01000050044092
:10F61000085004400450044000000203005104401C
:10F6200080014A0038800440431E032B14D872B670
:10F630000A4951F8230068B170B4094C058834F8C0
:10F640001320466841F82360521B24F8132062B649
:10F6500070BC704762B6704700207047B8A1FF1FAA
:10F6600010A3FF1F013803280BD872B6074B53F8BD
:10F67000203043B100205B680130002BFBD162B623
:10F680007047002070471846F9E700BF0CA2FF1F23
:10F6900030B472B62B4A13781D0706D52A4B196A67
:10F6A000002936D0996A002941D053781C0706D525
:10F6B000254B196C00293ED0996C002939D09378DC
:10F6C000190705D5204B196E002936D0996E89B1DE
:10F6D000D3781B0707D51C4BD3F880207AB3D3F817
:10F6E000882011213AB162B6184B00221A7030BC42
:10F6F00000F058BE0D21154C154D227843F83150BD
:10F7000003EBC1030830013A5860227062B630BC86
:10F71000704704220D4C0F4D217843F8325003EB13
:10F72000C20308304A1E5860227062B6EFE7052116
:10F73000E1E70921DFE70822ECE70C22EAE71022E3
:10F74000E8E700BF905F01000080FF1F35A2FF1FA8
:10F75000C800400088004000431E032B1DD81B4AF0
:10F76000400140F0100030B4104472B6184CE25C16
:10F77000032A1BD8DFE802F00212151703220D88B6
:10F78000E25410F0080F14BFC823882343EA05434E
:10F7900008310360416062B630BC70470830022215
:10F7A000EDE70522EBE708300422E8E7094A52F8C2
:10F7B000230038B1084A52F82300416042F8231070
:10F7C00062B6E9E742F82310034AF7E70080FF1F1B
:10F7D00044A2FF1F0CA2FF1F1CA2FF1F00BE00BF00
:10F7E0002DE9F04FDFF820B3DFF820A387B044E025
:10F7F000AF4F4FEA930807EBC809013ED9F8042040
:10F8000003F00803F6B2A2F1080003F0FF04002B96
:10F8100040F00B8157F838301B0C99B222F8081CC5
:10F82000002B00F0F980A34B22F8064C42F8044C60
:10F8300053F82620002A00F075819F4D55F8263098
:10F8400058609E4C45F8260034F81630194424F8C8
:10F85000161000F087FD002800F05D81984A994B52
:10F8600019F0080F00F1080018BF1346C9F804008A
:10F8700047F8383008238BF800309BF80040E4B29A
:10F8800065071DD5904B1B78BBB190490A7802F0F3
:10F89000FF032AB1013BDBB20B70002B00F00185A6
:10F8A0008B490A7802F0FF032AB1013BDBB20B70EF
:10F8B000002B00F02D8100F073FE04238BF8003044
:10F8C00004F0080303F0FF02002B00F0DA809AF83E
:10F8D0000030DBB21E098BD19A08DFF8D49159F8B9
:10F8E000321009EBC200C1F38301013940680C29D1
:10F8F0007DD8DFE801F080807C7C7C7C7C7C467C51
:10F900007C7C0700D0F800E0724C4168724F734E67
:10F910006160C4F800E01FFA8EF140F2816E0025AC
:10F92000674B49F83230012071453D60C9F81050ED
:10F93000C9F8185030705E4A00F20881B1F5D06FF6
:10F9400080F08283B1F5817F00F0668300F28F82C0
:10F95000802900F07483822940F0A782A18801F0F9
:10F960007F01042900F2A1825D4B5E4A89000B44AD
:10F970001570557019788D0740F180831070022042
:10F98000F2E2554F3A6842B3574B544E57491888E4
:10F9900034780D784028864645F0020828BF4FF09D
:10F9A000400E002C84F001043470CEEB00000CBF3C
:10F9B0008824C82409EBC80680B285F0010544EA12
:10F9C0000E447260188049F8384072440D7018B9BE
:10F9D000BEF1400F18BF00223A603E4B1A88B2F5C4
:10F9E000A06F04D100219A785970414B1A70414A96
:10F9F000012313703EE7374C258842F221018D42E6
:10FA000000F05A8224683C49324D8C4200F000825A
:10FA10002B4949F83210EAE7294A2A4B19F0080F16
:10FA200018BF134647F8383024E700F0BBFC334AD0
:10FA3000334952F82630002B78D058688C5D42F854
:10FA4000260003F10802C9F80420032C05D8DFE8DA
:10FA500004F0120F150204228A551A8819F0080FB3
:10FA60000CBF8823C82343EA024347F8383001E734
:10FA700002228A55F1E703228A55EEE705228A55CC
:10FA8000EBE7E00700F13082210600F15F82A20778
:10FA900006D51C4A1C4913780220DBB2137008708B
:10FAA000E30602D5184B10221A7007B0BDE8F08F9C
:10FAB0000080FF1FB8A1FF1F64A1FF1F10A3FF1F3D
:10FAC000C80040008800400040A2FF1FC9A1FF1FDE
:10FAD000B4A2FF1F2CA2FF1F60A1FF1FC8A1FF1F20
:10FAE000C020074038A2FF1F74A1FF1F34A2FF1FD0
:10FAF0009820074094200740210900030CA2FF1F13
:10FB000044A2FF1F88200740802007409020074024
:10FB100000F0ACFFCFE6AC4A47F838001378013369
:10FB20001370A7E643F82600A84D8AE68B5D032BE9
:10FB300000F26B8201A252F823F000BF75F80000BA
:10FB400075F800003DFF000037FF000040F621156A
:10FB5000A94200F0358100F29F81B1F5086F00F0F5
:10FB6000FF81B1F5106F40F0A0819948116AA47827
:10FB700004700C0600F19382D9F8282095491006EC
:10FB800000F18882D9F830209249120600F17D8276
:10FB9000D9F838208F49130600F17282D9F8402035
:10FBA0008C49150600F12E83D9F84820894914069E
:10FBB00000F12383D9F850208649100600F11883FC
:10FBC000D9F858208349120600F10D83D9F8602036
:10FBD0008049130600F12083D9F868207D49150675
:10FBE00000F11583D9F870207A49140600F1DE82FD
:10FBF000D9F878207749100600F1D382D9F880200F
:10FC00007449120600F1E982D9F888207149130677
:10FC100000F1DD82D9F890206E49150600F1D182FD
:10FC2000D9F898206B49140600F1C5826A486B4ADE
:10FC30006B4901906B486C4C644D0294002304970F
:10FC4000059680461C4617460E460395386828B12F
:10FC5000456800F0A7FB2846002DF9D100233B6042
:10FC6000039B30681A46002342F8243028B14568C7
:10FC700000F098FB2846002DF9D100223260019A4D
:10FC800098F800301146002241F8042B029A0191A5
:10FC9000023B4FF0000122F81410032B09D8DFE8D3
:10FCA00013F050010400500104004FF0010388F8E4
:10FCB00000300134042C07F1040706F1040608F1B2
:10FCC0000108C3D1494C404D2278494B049F059E01
:10FCD0000021100729701A7000F14E8245496278A0
:10FCE0000A700021C9F83010C9F838101107DFF880
:10FCF000E48000F12C82A2783F49DFF8D8800A70B6
:10FD000000211207C9F85010C9F8581000F10882F4
:10FD1000E2783A492F4C0A7013074FF00001C9F8F6
:10FD20007010C9F8781000F1BF8133780293002277
:10FD300083F00105C9F89020C9F8982000200190AF
:10FD40008046864602462E490C7844F0020C09EBA8
:10FD5000CC030393029B002B039B5A600CBF8822A9
:10FD6000C82242EA080384F0010249F83C303570A9
:10FD70000A70DFF860C0234BDFF88480002840F071
:10FD80001681BEF1400F1BD142F0020C09EBCC03EF
:10FD9000019ADFF840E05A60002D40F01E81050412
:10FDA00045F088059DF808304EF83C500244337009
:10FDB0000C701346402803D10020134A3B6010808A
:10FDC000124A0123137012E635A2FF1F64A1FF1F20
:10FDD00040A2FF1F0080FF1F1CA2FF1FB8A1FF1F32
:10FDE0000CA2FF1F44A2FF1F10A3FF1F905F010082
:10FDF000C4200740C8200740CC200740D02007403F
:10FE000034A2FF1FC8A1FF1F74A1FF1F9420074049
:10FE10006C68B1498C427FF4FBAD0178A9297FF46D
:10FE2000F7AD417845297FF4F3AD8178C2297FF49D
:10FE3000EFADC1786B297FF4EBADA849A84E0878E7
:10FE4000347880F00105002C40F002000D700CBFEA
:10FE50008821C82184F0010449F8301009EBC00062
:10FE6000A04934700025052445600C70D0E540F2AF
:10FE70000232914240F09480A28802F07F02042A6C
:10FE800013D865888DB998490290920011440A7878
:10FE900042F002020A7051E740F62122914200F03E
:10FEA000828042F2212291427DD08F4A0F2313702B
:10FEB0008E4A012313709AE58849894E0D78377868
:10FEC00085F0010E002F45F0020581F800E00CBF1F
:10FED0008821C82149F8351009EBC50587F00107CD
:10FEE0000021377069608DE5814B80487B491A613C
:10FEF0004FF0020E80F800E07B4F0A707D491960D8
:10FF000099607D4E7D4D7E4C9A610D213970FF21A7
:10FF10003170DFF808E2297022707A4D7A4A8EF843
:10FF200000109F27012406F8047C5D600470DA60ED
:10FF300007B0BDE8F08F01238B559BE400238B5560
:10FF400098E44FF0000388F80030B2E666496B4B46
:10FF500080220D2008701A70A2077FF5A1AD98E5E8
:10FF60006A496B4A09781170E588854280F0898179
:10FF70005A490C78402DAE4644F0020C28BF4FF091
:10FF8000400E02EB0E0309EBCC000193012342600B
:10FF90004FEA0E48CEEB050002930025C822E0E6AA
:10FFA000B1F5A06F81D1012300250293C6E6402858
:10FFB0007FF6EAAE42F002020CEBC201019E4E60F7
:10FFC000BDB19DF8085053491D703346403888F83C
:10FFD000004040334CF83210EFE69DF808303370A3
:10FFE0000504019B0C7045F0C80503444EF83C50D5
:10FFF000E0E69DF808501D70019B3E4988F80040DE
:020000021000EC
:10000000403840334CF83210D7E619F0080F0CBFD7
:10001000022303238B552DE4A28802F07F02042AD9
:100020003FF643AF6588002D7FF43FAF2E49029025
:10003000920011440A7822F002020A707EE6344AE5
:100040000220157055708FE733494A68002A3FF443
:100050002CAF6588B4F804E004E00C314A68002A4B
:100060003FF423AF0B88AB42F7D14B887345F4D1F3
:100070002D0A032D0CBF1078088975E7022073E75D
:10008000C86B083800F08EF988E5486B083800F036
:1000900089F97DE5C86A083800F084F972E5506A8C
:1000A000083800F07FF967E500F05CF9002800F0FF
:1000B000D68008300F4AC4F88400C4F8802000F0CD
:1000C00051F9002800F0C5800830124AC9F88C00A8
:1000D000C9F8882029E600BF0100040034A2FF1FF0
:1000E000C8A1FF1FC9A1FF1FC020074094200740DF
:1000F0000080FF1F880040008820074080200740C4
:100100009820074078A1FF1FCCA1FF1F40A2FF1F2E
:1001100038A2FF1FC8004000945F01008C200740F8
:1001200000F020F9002800F0A68008305D4AC8F8E9
:100130006400C8F8602000F015F9002800F09580F0
:100140000830594AC9F86C00C9F86820E0E500F0A9
:1001500009F9002877D00830524AC8F84400C8F896
:10016000402000F0FFF8002867D008304E4AC9F858
:100170004C00C9F84820BEE500F0F4F8002856D03D
:100180000830484AC9F82400C9F8202000F0EAF8ED
:10019000002846D00830444AC9F82C00C9F8282065
:1001A0009CE5C86F083800F0FDF827E5486F08386F
:1001B00000F0F8F81CE5D1F89C00083800F0F2F8DF
:1001C00034E5D1F89400083800F0ECF828E5D1F8CF
:1001D0008C00083800F0E6F81CE5D1F884000838F7
:1001E00000F0E0F810E5C86D083800F0DBF8EDE449
:1001F000486D083800F0D6F8E2E4C86C083800F022
:10020000D1F8D7E4486C083800F0CCF8CCE4C86EDC
:10021000083800F0C7F8E5E4486E083800F0C2F886
:10022000DAE42A78C9F8280001322A7056E52A78DB
:10023000C9F8200001322A70A8E72A78C9F84800D6
:1002400001322A7057E52A78C8F8400001322A7036
:1002500087E72A78C9F8880001322A7065E52A788C
:10026000C4F8800001322A7029E72A78C9F86800AA
:1002700001322A704CE52A78C8F8600001322A70F1
:1002800059E74028864628BF4FF0400E02EB0E0388
:1002900001930123CEEB00004FEA0E4800250293A4
:1002A00051E500BE88004000C80040002DE9F84339
:1002B000204C00F037FF002204F1A00023461A6012
:1002C0005A60083383424FF00001F8D11A4A1B4F9D
:1002D00013681B4D1B481C4EDFF87880DFF878C090
:1002E000DFF87890DFF878E043F480231360C4F3FC
:1002F00007233B70C4F307432B70240EFF2302F542
:1003000028320470114D88F8003011488CF8003004
:10031000D4323370012389F8003070268EF8001033
:100320004FF40074102107F8183C2E70046011700F
:10033000BDE8F8830080FF1F348004409C20074004
:10034000B0200740B42007401020074049E400E0F7
:1003500008E100E080200740882007409420074003
:100360000021074072B60D480268B2FA82F30F2BE3
:1003700010DC4FF00041D94022EA0102026062B66F
:10038000074803EBC303DB00C2180021C15010462D
:100390005160704762B60020704700BF3493FF1F62
:1003A000BC83FF1F0D4B0E4AC31AA2FB03231B097C
:1003B0000F2B0CD80B4A127852B972B60A484FF07C
:1003C0000041026821FA03F31A43026062B67047E3
:1003D000064A1278002AF0D0FFF75AB9BC83FF1FF3
:1003E000398EE33835A2FF1F3493FF1F40A2FF1F51
:1003F00038B50E4B0E4C1B68218805468BB1B1F504
:10040000917F05D20B4A4B1C55549BB2238038BDBB
:100410000022084898470021064A555401232380AA
:1004200038BDB1F5917FEDD338BD00BF6CA2FF1F81
:100430001AA3FF1F20A3FF1F2DE9F843214E224FCF
:100440003168012380463B70B1B1204D4B8801EBF0
:100450008302013300240F2BC2F808802C7004D8CB
:100460004B8000233B70BDE8F88340230B800320C2
:10047000FFF772F93460F4E7DFF8549099F8003030
:10048000002BF0D0114D45F6215408E0013C12D06C
:100490002B7883B900F0AAFD99F800307BB10320D6
:1004A000FFF7E0F80528F1D8FFF75CFF0146306060
:1004B0000028EBD0CAE701232B70BDE8F883BDE824
:1004C000F88300BF88A2FF1F5CA2FF1F8CA2FF1F42
:1004D00040A2FF1F1201F8B5D5B2A1B3012943D044
:1004E0004378044600781B0643EA004040F470401D
:1004F00045F004068F1E3043FFF79EFF022F04F1E4
:10050000020314D9053414F8023C14F8032C14F82F
:10051000010C1B0443EA0223334343EA0060033F18
:10052000FFF78AFF022F234604F10304EBD8022FC2
:1005300023D0012F0DD045F4774040F00500BDE8F1
:10054000F840FFF779BF14482843BDE8F840FFF7AB
:1005500073BF187845F4770545F0060545EA002095
:10056000BDE8F840FFF768BF03780C4845EA03454B
:100570002843BDE8F840FFF75FBF1A78587845F088
:10058000774545F0070545EA022545EA0040BDE804
:10059000F840FFF751BF00BF06F0F70007F000F783
:1005A00038B5084B1C7824B9074D296809B14B8828
:1005B00003B938BD9B000B800320FFF7CDF82C60FA
:1005C00038BD00BF5CA2FF1F88A2FF1F2DE9F041CC
:1005D000AD4E33680746002B00F092801D885A8884
:1005E000910803EB81010432AA428C6842D25A80FE
:1005F00004F00F064FEA1428A449A6F1080208F0F7
:100600000F00C4F30313062A00F101050B701AD979
:10061000B31E012B5FFA88F04ED9052E48D0042E68
:1006200000F0A481731F022B7FD90F2E0ED1F72863
:1006300042D8F02802D0964B1B883BB1FFF7D8FE7A
:100640000020BDE8F08127B1BD4202D00020BDE806
:10065000F081082EC4F3033300F08780092E11D0F7
:100660000A2E40F094800A2BF0D18A4B8A4A1B68EC
:10067000A02181E01846FFF795FE0420FEF7D4FF85
:100680003060B5E7092BE1D1270E00F07B81834B69
:10069000814A1B689021C4F307461170EDB2FCB289
:1006A000002B00F09D80224631462846984797E06F
:1006B000F02843D9F72841D0F1380E28C6D801A335
:1006C00053F820F07B0801005F0801004D0801008D
:1006D0004D0601004D0601003F0801004D060100D6
:1006E0001F0901004D060100E9080100030901008E
:1006F000270801004D0601000F080100F307010063
:10070000674B1B78002BA1D00420FEF78DFF03461A
:10071000306000289AD00588002D7FF460AFFFF785
:1007200041FE35602846BDE8F081FFF761FEC4F365
:100730000740FFF75DFE072E02D1200EFFF758FE9F
:10074000534B584A198858481468584D524A0170FA
:1007500000270E0AF0201F802E7010700CB30122AB
:100760005348A0470120BDE8F081082B7FF46EAF0D
:10077000504B494A1B688021C4F307461170EDB203
:10078000240E6BB3284622463146984728E00B2EAC
:1007900011D10B2B7FF45AAF474B3F4A1B68B02156
:1007A000EAE7464B1B68002B00F0FB804048984767
:1007B0000120BDE8F0810C2E40F000810C2B7FF46D
:1007C00045AF3F4B344A1B68C0211170EDB2C4F3F2
:1007D0000746002B00F0C88028463146240E984773
:1007E0003849314A314B0D7016701C700120BDE83C
:1007F000F081354B1B68002B00F0D6809847C4F37E
:100800000746254BEDB2240E83F80080E8E72F4B16
:100810001B68002BF2D12E4B1B68A3B1FE2098471A
:10082000C4F30746EDE72B4B1B68002BE6D1284BA2
:100830001B6843B1FC209847C4F30746E1E7264B09
:100840001B68002BDAD1C4F30746DAE7234B1B6899
:10085000C4F30746002BD4D030469847D1E7204B4D
:100860001A68002AEFD0260C630C06F07F0003F410
:100870007E531843F6B29047C3E71A4B1B68C4F384
:100880000746002BE8D1BCE794A2FF1F1EA3FF1F61
:100890001AA3FF1F70A2FF1F18A3FF1FA4A2FF1F10
:1008A00040A2FF1F6CA2FF1F1CA3FF1F1DA3FF1F61
:1008B00020A3FF1F9CA2FF1FA0A2FF1F84A2FF1F57
:1008C00060A2FF1F1FA3FF1F4CA2FF1F50A2FF1F0C
:1008D00054A2FF1F90A2FF1F80A2FF1F98A2FF1F1C
:1008E00068A2FF1F7CA2FF1F3F4B1B68002B85D116
:1008F0003E4B1B68002BA6D0FA209847C4F307464E
:100900007FE73B4B1B68002B7FF478AF374B1B68AE
:10091000002B98D0FB209847C4F3074671E7354B6E
:100920001B68002B7FF46AAF304B1B68002B8AD00A
:10093000F8209847C4F3074663E70E2B7FF486AE92
:100940002D4A2E4B1268E0211970002A47D0260C40
:10095000610C06F07F0301F47E511943EDB2A1F55D
:10096000005128469047F6B2240E39E7FFF740FDC4
:10097000C4F30740FFF73CFD200EFFF739FD0020D0
:10098000BDE8F0811E4B1D4A1B6880211170EDB23D
:10099000C4F3074683B1314628463A4698473C4659
:1009A0001EE70120BDE8F081104B1B68002B3FF4CF
:1009B0004AAFFF20984746E71C4611E70D2EBCD1F1
:1009C0000D2B7FF443AE0F4B0C4A1B68D0211170E6
:1009D000EDB2C4F30746002B7FF4FEAEC4E7C4F3C8
:1009E0000746EDB2240EFBE678A2FF1F54A2FF1FBC
:1009F00058A2FF1F48A2FF1F64A2FF1F18A3FF1FDA
:100A00009CA2FF1F74A2FF1F38B5164D2868E0B1E5
:100A100001884488A14213DD03191B7A83B104F1D4
:100A20000803C2180C1B002302E012F8011F21B1B9
:100A30000133A342F9D1204638BD1C46204638BDBB
:100A4000FFF7B0FC0020286038BD074B1B780BB9BE
:100A5000002038BD0220FEF7E7FD28600028D7D12E
:100A6000F6E700BFB0A2FF1F40A2FF1F0D4B1B788F
:100A7000BBB910B50C4C216803F0FF024B883F2B2B
:100A800007DC07330B4401F1470003F8012F8342D1
:100A9000FBD140230B800120FEF75EFE0023236084
:100AA00010BD7047A8A2FF1FACA2FF1F70B5EFF3E7
:100AB000108272B60C4C206880B10C4E0025436940
:100AC000236073B19D6102B962B645778368984728
:100AD000EFF3108272B620680028F0D102B962B636
:100AE00070BD3360EFE700BFB8A2FF1FBCA2FF1FBD
:100AF000FFF7DCBF024A136801331360704700BF81
:100B000064A0FF1F4B0803F1376303F5D83310B51A
:100B10000446B3FBF1F0FDF7EDFE044B1B7803B187
:100B200010BD2046BDE8104000F03EBB7093FF1F93
:100B300008B50846FEF7A8F8012008BD08B5084624
:100B4000FEF7A2F8012008BD38B508460D4602F0B0
:100B5000F7FA044601462846FEF7EEF8204638BD6F
:100B600010B5084614461146FEF7E6F8204610BDBB
:100B7000FEF7C0B908B50846FEF766F8003018BFA2
:100B8000012008BD08B50846FEF73CF8003018BF44
:100B9000012008BD08461146FDF7CCBF0846FEF708
:100BA00003B800BF0846FDF7A9BF00BFFDF744BF6B
:100BB00010B54B0803F13760144600F5D830B0FB90
:100BC000F1F0FDF797FE2046BDE81040FDF708BFA5
:100BD000FEF778B9FEF742B9FEF730B9FEF710B963
:100BE000FEF71AB90368064A1B68934205D110B58F
:100BF000C8B2FEF749F8012010BDC9B2184700BFBE
:100C00003D0B01000368064A1B68934205D110B5ED
:100C1000C8B2FEF739F8012010BDC9B2184700BFAD
:100C20003D0B01000368064A1B68934205D110B5CD
:100C3000C8B2FEF729F8012010BDC9B2184700BF9D
:100C40003D0B01000368064A1B68934205D110B5AD
:100C5000C8B2FEF719F8012010BDC9B2184700BF8D
:100C60003D0B01004B0803F1B76303F5584310B582
:100C70000446B3FBF1F0FEF73BFA044B1B7803B1DB
:100C800010BD2046BDE8104000F08EBA7193FF1FE2
:100C900008B50846FEF76AFB012008BD08B50846FE
:100CA000FEF764FB012008BD38B508460D4602F08A
:100CB00047FA044601462846FEF762FB204638BD47
:100CC00010B5084614461146FEF75AFB204610BDE3
:100CD000FEF7E6BB08B50846FEF728FB003018BF54
:100CE000012008BD08B50846FEF7FEFA003018BF1F
:100CF000012008BD08461146FEF7CCBA0846FEF7AB
:100D0000F1BA00BF0846FEF7A9BA00BFFEF76CBAF9
:100D100010B54B0803F1B760144600F55840B0FB1E
:100D2000F1F0FEF7E5F92046BDE81040FEF730BAD5
:100D3000FEF79EBBFEF768BBFEF756BBFEF736BB61
:100D4000FEF740BB0368064A1B68934205D110B505
:100D5000C8B2FEF70BFB012010BDC9B2184700BF97
:100D60009D0C01000368064A1B68934205D110B52B
:100D7000C8B2FEF7FBFA012010BDC9B2184700BF88
:100D80009D0C01000368064A1B68934205D110B50B
:100D9000C8B2FEF7EBFA012010BDC9B2184700BF78
:100DA0009D0C01000368064A1B68934205D110B5EB
:100DB000C8B2FEF7DBFA012010BDC9B2184700BF68
:100DC0009D0C0100704700BF0368F0B4FBB1002523
:100DD00001249D60DC601B4C1A601C44241104F14A
:100DE00044056A11032692009E60174F0679174B3F
:100DF00047F8241002F1604202F5614205F01F0538
:100E0000012000FA05F5E6541560F0BC7047104C5F
:100E1000236843F40003236000BF0E4B0E4DA4F57E
:100E20008734A4F59E7401261E60234604609C68E6
:100E3000002CD0D01033AB420360F8D10023036004
:100E40001846E2E7008FFCBF6093FF1F44E400E018
:100E50003C80044000700340407103400168A9B128
:100E60000B4BF0B40B441B110A4E0B4F0B4D46F8C5
:100E7000237003F1440202F01F0401235211A34026
:100E8000002445F822308C600460F0BC704700BF3D
:100E9000008FFCBF6093FF1FC50D010080E100E0E3
:100EA000024A034B012111601B6818470C71034073
:100EB0006093FF1F024A034B012111605B681847D2
:100EC0001C7103406093FF1F024A034B0121116014
:100ED0009B6818472C7103406093FF1F024A034B25
:100EE00001211160DB6818473C7103406093FF1FCC
:100EF000F8B50E4671B17AB10746144600253B6835
:100F000016F8011B1B6838469847013C0544F6D18A
:100F10002846F8BD0846F8BD1046F8BD00B5064A9B
:100F2000036812885B6883B001A9ADF8042002222F
:100F3000984703B05DF804FB8C5F0100F0B50746ED
:100F40008BB0002A33D0012A08BF0A2251B32124D2
:100F500000E0F4B2B1FBF2F502FB1511C8B20929A9
:100F600000F1300198BFC8B20AA988BF37302144C8
:100F700088BFC0B201F8240C661E2946002DE8D1B6
:100F800033B1013CE4B20AAB23442D2203F8242CF4
:100F90003B6801AA11195B683846C4F122029847E0
:100FA0000BB0F0BD30228DF825202124E8E703683E
:100FB000C9B21B6898470BB0F0BD00BF0029BABF8B
:100FC00049422D2300230A22FFF7B8BF08B5F0F7E6
:100FD0005BFEF1F7B1FD00F009F8FAE701F014BB90
:100FE00001F01ABB704700BF704700BF2DE9F843FE
:100FF000314E337893B1314F3A787AB90122D9071B
:101000003A7036D49A0719D400225B073A7005D596
:101010002B4B1A6812B1EFF305820AB1BDE8F883D1
:10102000EFF3108172B6186818B1264C2278002AA6
:101030002ED00029F2D162B6BDE8F883DFF89080A7
:1010400098F80020002ADFD0DFF88890002405E01F
:10105000013498F80030E4B2A34212D959F8245070
:101060002B6828461B6998470028F1D02B699847C0
:10107000EEE7FFF7C9FCC8B9134B1B781BB93378EF
:10108000C0E73378C0E7337803F0FE033370B9E785
:1010900045691D60012323705DB1AA6101B962B683
:1010A00000254577836898472570B7E700F092F8E8
:1010B000E2E7064B1D60F1E77293FF1FC9A2FF1F15
:1010C000C4A2FF1FC8A2FF1F5294FF1FC0A2FF1F90
:1010D000D8A2FF1FCCA2FF1FF0B44D1E2E46002445
:1010E00000E00134B0FBF2F302FB1300092800F129
:1010F00030078ABF3730F8B2C0B206F8010F184681
:10110000002BEED10A1953704CB1107815F8016F0D
:1011100028700133E01A834202F80169F5DB0846C2
:10112000F0BC704770B584B072B6194B194D1A48AF
:10113000702241260F2480211A702E701A460470E6
:10114000197013781B06FCD5144B186862B6144B43
:10115000144C984298BF00EB800001A998BF400052
:101160000A22FFF7B9FF01A92046002311F8012B3D
:1011700001333AB10A2B20F8022FF7D1162323703E
:1011800004B070BD5B00DBB2237004B070BD00BF63
:101190000000024007000240060002400800024032
:1011A0007F9698003C94FF1F30B40749074C0A789B
:1011B0002378074D42F0020245F823000A700133FC
:1011C000237030BC704700BF7293FF1FD8A2FF1F6F
:1011D000CCA2FF1F704700BF2DE9F043DFF8EC8081
:1011E0008BB006460F4600F073F898F900300133D3
:1011F00004460D4637D03046394600F0DFF9002866
:1012000031D02BA3D3E900233046394600F02CFE21
:10121000814668BB28A3D3E900233046394600F055
:1012200005FE00B398F90030254ACDF8209004243B
:1012300000200021022BCDE90467CDE9026700946C
:101240000192CDE906012CD0684600F0BDF940B30B
:10125000089B1BB101F0AAF9089B0360DDE90601B8
:101260000BB0BDE8F083204629460BB0BDE8F08303
:10127000134A98F90030019203210022CDE9046756
:10128000CDE90267009108922BB90E4B4FF06042F6
:10129000CDE90623D8E70C490020022BCDE9060151
:1012A000D2D101F083F922230360D1E7AFF30080AC
:1012B000EF39FAFE422E864051302DD5104987C0B5
:1012C00000600100FFFFEF470000F07F5394FF1F15
:1012D0002DE9F04FB04F21F00042BA4283B00C46E6
:1012E0004FEAD17605460DD9AC4FBA4225D9C1F3A4
:1012F0001303034340F0EF800EB10020014603B01A
:10130000BDE8F08FA64B9A4200F2CC80A54B9A42E2
:1013100000F2DE808AA3D3E9002300F063F9002203
:10132000A14B00F0A1FD002800F0058128462146D0
:1013300000229D4B00F056F9E1E783A3D3E9002397
:1013400000F092FD002840F0CB802846214680A383
:10135000D3E9002300F06AFD0028CED1934B284644
:1013600003EBC60821467CA3D3E9002300F0ECFA86
:10137000D8E9002300F036F900F080FD804600F047
:101380007DFA77A3D3E9002306460F4600F0DCFA86
:1013900002460B462846214600F022F972A3D3E903
:1013A0000023CDE900013046394600F0CDFA8246EF
:1013B0008B4652465B46DDE9000100F011F9054617
:1013C0000C462A4623462846214600F0BDFA68A36B
:1013D000D3E9002306460F4600F0B6FA66A3D3E928
:1013E000002300F0FDF832463B4600F0ADFA64A35E
:1013F000D3E9002300F0F6F832463B4600F0A4FAA9
:1014000061A3D3E9002300F0EBF832463B4600F03D
:101410009BFA5FA3D3E9002300F0E4F832463B4691
:1014200000F092FA02460B462846214600F0D8F812
:1014300006460F462846214632463B46B8F1000F85
:1014400056D000F081FA324604460D463B46002055
:101450004FF0804100F0C4F802460B462046294672
:1014600000F09CFB02460B465046594600F0B8F887
:10147000DDE9002300F0B4F80B4602464A4900209B
:1014800000F0AEF86FF47F7398454FDA08F57A787C
:1014900001EB085100224FF0B87300F055FA03B089
:1014A000BDE8F08F424B9A423FF658AF414BF400F3
:1014B0002344D3E9002300F093F83F4BC6F1010821
:1014C0001C44CDE90001D4E900ABC6EB080870E785
:1014D0004FF0000875E702460B4600F083F80EE770
:1014E00017A3D3E900231046194600F02DFA06E7AA
:1014F00000F02AFA0022804689464FF080433046A9
:10150000394600F06DF802460B464046494600F069
:1015100045FB2A46234600F063F802460B460020AE
:10152000214900F05DF803B0BDE8F08F01EB0851F0
:1015300003B0BDE8F08F804643E700BFAFF3008003
:101540009C7500883CE4377EEF39FAFE422E8640D7
:1015500051302DD5104987C0FE822B654715F73FC6
:101560000000E0FE422EE63F763C7935EF39EA3D59
:10157000D0A4BE726937663EF16BD2C541BDBB3E99
:101580002CDE25AF6A56113F93BDBE166CC1663F77
:101590003E5555555555C53F412E8640FFFFEF7FBF
:1015A000422ED63FFFFF2F3E0000F03F08600100B3
:1015B000B1A2F03F286001001860010041F0004135
:1015C00001F58010C00F7047002070470B460146A0
:1015D000184600F0E5BF00BF81F0004102E000BF07
:1015E00083F0004330B54FEA41044FEA430594EAE3
:1015F000050F08BF90EA020F1FBF54EA000C55EA1E
:10160000020C7FEA645C7FEA655C00F0E2804FEAEE
:101610005454D4EB5555B8BF6D420CDD2C4480EAD0
:10162000020281EA030382EA000083EA010180EA00
:10163000020281EA0303362D88BF30BD11F0004F4E
:101640004FEA01314FF4801C4CEA113102D0404284
:1016500061EB410113F0004F4FEA03334CEA1333BF
:1016600002D0524263EB430394EA050F00F0A780D7
:10167000A4F10104D5F1200E0DDB02FA0EFC22FAD2
:1016800005F2801841F1000103FA0EF2801843FAC6
:1016900005F359410EE0A5F120050EF1200E012AB7
:1016A00003FA0EFC28BF4CF0020C43FA05F3C018F5
:1016B00051EBE37101F0004507D54FF0000EDCF16E
:1016C000000C7EEB00006EEB0101B1F5801F1BD317
:1016D000B1F5001F0CD349085FEA30004FEA3C0C1B
:1016E00004F101044FEA445212F5800F80F09A8011
:1016F000BCF1004F08BF5FEA500C50F1000041EB15
:10170000045141EA050130BD5FEA4C0C404141EB18
:10171000010111F4801FA4F10104E9D191F0000F3F
:1017200004BF01460020B1FA81F308BF2033A3F1C2
:101730000B03B3F120020CDA0C3208DD02F1140CB9
:10174000C2F10C0201FA0CF021FA02F10CE002F1F4
:101750001402D8BFC2F1200C01FA02F120FA0CFCED
:10176000DCBF41EA0C019040E41AA2BF01EB045136
:10177000294330BD6FEA04041F3C1CDA0C340EDC34
:1017800004F11404C4F1200220FA04F001FA02F377
:1017900040EA030021FA04F345EA030130BDC4F135
:1017A0000C04C4F1200220FA02F001FA04F340EA2A
:1017B0000300294630BD21FA04F0294630BD94F0DB
:1017C000000F83F4801306BF81F480110134013DC2
:1017D0004EE77FEA645C18BF7FEA655C29D094EA33
:1017E000050F08BF90EA020F05D054EA000C04BFB1
:1017F0001946104630BD91EA030F1EBF002100209C
:1018000030BD5FEA545C05D14000494128BF41F03A
:10181000004130BD14F580043CBF01F5801130BD9E
:1018200001F0004545F0FE4141F470014FF0000029
:1018300030BD7FEA645C1ABF194610467FEA655CDA
:101840001CBF0B46024650EA013406BF52EA03357C
:1018500091EA030F41F4002130BD00BF90F0000F6A
:1018600004BF0021704730B54FF4806404F13204A6
:101870004FF000054FF0000150E700BF90F0000F5F
:1018800004BF0021704730B54FF4806404F1320486
:1018900010F0004548BF40424FF000013EE700BF56
:1018A00042004FEAE2014FEA31014FEA02701FBFE6
:1018B00012F07F4393F07F4F81F06051704792F0B8
:1018C000000F14BF93F07F4F704730B54FF4607432
:1018D00001F0004521F0004120E700BF50EA01027D
:1018E00008BF704730B54FF000050AE050EA01022A
:1018F00008BF704730B511F0004502D5404261EB9A
:1019000041014FF4806404F132045FEA915C3FF4DA
:10191000DCAE4FF003025FEADC0C18BF03325FEA73
:10192000DC0C18BF033202EBDC02C2F1200300FA28
:1019300003FC20FA02F001FA03FE40EA0E0021FA4D
:1019400002F11444C1E600BF70B54FF0FF0C4CF437
:10195000E06C1CEA11541DBF1CEA135594EA0C0FED
:1019600095EA0C0F00F0DEF82C4481EA030621EA28
:101970004C5123EA4C5350EA013518BF52EA033563
:1019800041F4801143F4801338D0A0FB02CE4FF015
:101990000005E1FB02E506F00042E0FB03E54FF045
:1019A0000006E1FB03569CF0000F18BF4EF0010E3D
:1019B000A4F1FF04B6F5007F64F5407404D25FEA39
:1019C0004E0E6D4146EB060642EAC62141EA5551EC
:1019D0004FEAC52040EA5E504FEACE2EB4F1FD0C2E
:1019E00088BFBCF5E06F1ED8BEF1004F08BF5FEAAC
:1019F000500E50F1000041EB045170BD06F000465E
:101A000046EA010140EA020081EA0301B4EB5C040A
:101A1000C2BFD4EB0C0541EA045170BD41F4801102
:101A20004FF0000E013C00F3AB8014F1360FDEBF27
:101A3000002001F0004170BDC4F10004203C35DA03
:101A40000C341BDC04F11404C4F1200500FA05F386
:101A500020FA04F001FA05F240EA020001F0004227
:101A600021F0004110EBD37021FA04F642EB06019D
:101A70005EEA430E08BF20EAD37070BDC4F10C04C7
:101A8000C4F1200500FA04F320FA05F001FA04F28B
:101A900040EA020001F0004110EBD37041F1000177
:101AA0005EEA430E08BF20EAD37070BDC4F1200582
:101AB00000FA05F24EEA020E20FA04F301FA05F2EA
:101AC00043EA020321FA04F001F0004121FA04F292
:101AD00020EA020000EBD3705EEA430E08BF20EA62
:101AE000D37070BD94F0000F0FD101F0004640009C
:101AF00041EB010111F4801F08BF013CF7D041EA1E
:101B0000060195F0000F18BF704703F00046520021
:101B100043EB030313F4801F08BF013DF7D043EAF2
:101B20000603704794EA0C0F0CEA135518BF95EAA8
:101B30000C0F0CD050EA410618BF52EA4306D1D12F
:101B400081EA030101F000414FF0000070BD50EA4E
:101B5000410606BF1046194652EA430619D094EAD8
:101B60000C0F02D150EA013613D195EA0C0F05D1C2
:101B700052EA03361CBF104619460AD181EA030116
:101B800001F0004141F0FE4141F470014FF00000CE
:101B900070BD41F0FE4141F4780170BD70B54FF069
:101BA000FF0C4CF4E06C1CEA11541DBF1CEA1355E9
:101BB00094EA0C0F95EA0C0F00F0A7F8A4EB0504CB
:101BC00081EA030E52EA03354FEA013100F08880C2
:101BD0004FEA03334FF0805545EA131343EA12638B
:101BE0004FEA022245EA111545EA10654FEA002640
:101BF0000EF000419D4208BF964244F1FD0404F5F9
:101C0000407402D25B084FEA3202B61A65EB030554
